:020000040000FA
:040000006FD00400B9
:101000006F00907D00000000000000009020002094
:10101000AA220020A9BDF9F56C23002000000000E1
:10102000000000006C230020902000200000000041
:101030000000000090200020000000009020002010
:101040000000000090200020902000209020002030
:101050009020002090200020482F00208224002093
:101060000000000090200020902000200C24002090
:1010700090200020D22300209020002090200020EB
:101080009020002090200020902000209020002020
:101090009020002001A04111B7170040985F3AC688
:1010A000945F3247E39CE6FE3245410182800111A4
:1010B00013078008F337078093F787083EC20100C3
:1010C0000100B7170040930570052380B70413068D
:1010D00080FA2380C7040100010083C6B70493F699
:1010E000F60DA385D704238007049246F3A6068055
:1010F0000100010093760502D5CEF336078093F602
:10110000860836C4010001002380B7042380C70489
:1011100001000100B70614007D89558D88C70100C4
:1011200001000100010023800704A246F3A6068007
:101130000100010073370780137787083AC6010062
:1011400001002380B7042380C704010001000100CF
:1011500001003727004093061005A303D7802380A2
:101160000704B247F3A70780010001009307800836
:10117000F3B7078093F787083ECE01000100B71749
:101180000040130770052380E704130780FA2380CB
:10119000E7040100010003C7B70413670708A3852C
:1011A000E70423800704F247F3A70780010001004A
:1011B0000561828093760504BDC6F336078093F6F9
:1011C000860836C8010001002380B7042380C704C5
:1011D00001000100B7061400938606047D89558D31
:1011E00088C7010001000100010023800704C246F6
:1011F000F3A6068001000100733707801377870884
:101200003ACA010001002380B7042380C70401000B
:1012100001003727004093062005A303D7802380D1
:101220000704D24781B773370780137787083ACC12
:10123000010001002380B7042380C70401000100DE
:1012400098471367070C98C723800704E24719BF24
:101250000111814601468145114506CE97000000E7
:10126000E780405793078008F3B7078093F7870814
:101270003EC601000100B717004013077005238028
:10128000E704130780FA2380E7040100010003C785
:101290006704136717002383E70423800704B2471A
:1012A000F3A7078001000100F2400561828041112F
:1012B000814601468145114597000000E780805135
:1012C00013078008F337078093F787083EC40100AF
:1012D0000100B7170040130670052380C70493066A
:1012E00080FA2380D70401000100FD552396B70240
:1012F00023800704A245F3A5058001000100733790
:101300000780137787083AC6010001002380C704CD
:101310002380D7040100010003C767041367170087
:101320002383E70423800704B247F3A70780010063
:10133000010001A0B1473305F50201007D1575FDDF
:101340008280411122C426C206C6AA8401446317C2
:101350009400B24022449244410182800504130566
:10136000803E420497000000E78000FD4180C5B741
:101370009305000273A04580824573901534924016
:101380002242B2424243D2436244F2440255925551
:101390002256B2564257D2576258F25806499649D9
:1013A000264AB64A464BD64B664CF64C065D965DD1
:1013B000265EB65E465FD65F09617300203041113C
:1013C000B7170040985F3AC6945F3247E39CE6FE49
:1013D000324541018280B71700401307000323887C
:1013E000E7028547171700002326F74673002030D1
:1013F000411122C406C637040020976000E0E78050
:10140000A03D1C408297976000E0E780E03CF5B784
:1014100037370040834747009146BD8B639ED70214
:10142000B73600401306F00F973500009385851FEF
:101430009737000083D7072F03C7A6001377F70F4E
:101440001DE3B7E70400BC4F0946894517150000A6
:101450000345C5F7829731A099466394D700834727
:1014600057007300203003C786001377F70FE3653A
:10147000F6FC13851700AE97173800002314A82A2E
:101480002380E70075B7B787004003C76700098B63
:101490006309071003C77700930600031377070358
:1014A000630DD708173800000348987A17360000F4
:1014B000130606770547B30606012380E60083C5B9
:1014C0007700173700001307A777429793F5F50FBA
:1014D0002300B70003C58700973500009385457545
:1014E000C2951375F50F2380A500034707008945B2
:1014F0001377F703630CB70C63E7E50A6306071A73
:101500008545630CB7129737000083C7777433079C
:10151000F600034707001377F70F19CB850793F7FA
:10152000F70F3D476363F71A17370000A302F772FE
:10153000B787004009472383E700B787004083C788
:101540007700E207E18763DE07049737000083C76F
:101550003770173700001307A76C3E9785462300A6
:10156000D700173700001307A76D3E9793060003B7
:101570002300D700173700001307876B3E97A1465B
:1015800085072300D70093F7F70F3D476364F714EF
:1015900017370000A30EF76AB78700400947238377
:1015A000E70073002030930610026300D70E930605
:1015B00020026305D70693060002E316D7F403C79B
:1015C00027021377C70F13672700D5A803C7670043
:1015D0001377070465CB03C7A70217380000130869
:1015E000A845173500001305E53C13470708238578
:1015F000E70203C7A7021377370F13678700238516
:10160000E702814713070004B305F5008C41B306D8
:10161000F80091078CC2E399E7FEF5B503C7A7026E
:10162000134707042385E70203C7A7021377C70FF1
:10163000136727002385E702F9B503C7670013770F
:10164000070449C303C7670217380000130888322C
:10165000173500001305C529134707082383E70240
:1016600003C767021377370F136787002383E702E7
:10167000814713070004B305F5008C41B306F80059
:1016800091078CC2E399E7FEBDBD03C7670213470C
:1016900007042383E70203C767021377C70F1367A3
:1016A00027002383E70285B503C767001377070484
:1016B00011CB03C727021377370F136787002381E6
:1016C000E70291B5238006003DBD97370000A38156
:1016D0000758B9BD97370000A38C075675BD230383
:1016E000048015472303E48001002302A480828044
:1016F00083076480E3CE07FE230304808280830790
:101700006480E3CE07FE03454480828083076480C3
:10171000E3CE07FE2302A4808280411126C44AC280
:101720004EC006C61377F50BAD47AA892E8995449E
:10173000630CF700194597000000E78080FA9700D6
:101740000000E78020FB8D444E8597000000E78075
:1017500040F9FD59FD1463983401B240A244124986
:10176000824941018280135509011375F50F9700D5
:101770000000E780E0F92209F1BF011126CC06CE76
:10178000B704080097000000E780C0F615459700F1
:101790000000E78000F597000000E78080F69700E2
:1017A0000000E78000F62AC697000000E78080F47A
:1017B00032459377150089EB136515001375F50F06
:1017C000F240E24405618280FD14E9F00145CDBF9D
:1017D000397126DC4ADA4ED852D656D45AD25ED067
:1017E00006DE62CE66CCB7E700E07D5783AA07002D
:1017F00022C603AA470023A0E71823A2E718B717B9
:101800000040130770052380E704130780FA238044
:10181000E70483C74704930B75FFB684E20793FB85
:10182000FB0F8546AA892E8B328937240040E18739
:10183000015763FA76016308D50089461307000251
:101840006313D5000157D98F93F7F70FB71C0040EA
:101850002382FC0411472303E4801305F00F970053
:101860000000E78000E8094C97000000E78080E86E
:1018700063657C15B7050700DA953787070079554A
:1018800063FEE504B3879500636AF704370B08002D
:10189000A94733EB65016395F90881E88144970016
:1018A0000000E78020E5268515A8DA850945970020
:1018B0000000E780C0E605090345F9FFFD14050BAC
:1018C00097000000E780C0E481C49377FB0FE5F741
:1018D00097000000E780A0EA69F17D55B717004046
:1018E000130770052380E704130780FA2380E704B9
:1018F00003C74704418B2382E704F250B7E700E0B7
:1019000023A0571123A24711E25432445259C2591D
:10191000325AA25A125B825B724CE24C2161828085
:10192000A547639BF90685691309F00FB306990073
:10193000B3742B01B6941349F9FFB3749900856B06
:1019400033796901416B9387F9FFB3F7270199E375
:1019500063FC340193D94900C147E3E637FF3DBF3B
:101960000569C1697D19D9B71305800D63886901BF
:10197000130500026384790113051008CA859700D6
:101980000000E780C0D997000000E78040DF31D534
:101990004E99B38434416DBFDA852D459700000020
:1019A000E780E0D7CA94E30B99EE050997000000A1
:1019B000E78020D5A30FA9FEFDB79387F9FF93F722
:1019C000F70F636DFC0C83C71C0413073008631505
:1019D000F706370708006361EB06B3079B00B706FD
:1019E000100063FBD704334BEB0089476399F9067A
:1019F0008980D549E38404EADA8509459700000027
:101A0000E780E0D111090327C9FF91472320E48033
:101A100003076480E34E07FE23033481FD17EDFBCB
:101A2000FD14110B81C49377FB0FE9FF97000000B1
:101A3000E780E0D461F155B5B717004003C75704FC
:101A4000B70708001377070219E3B787070079552E
:101A5000E376FBE833079B00E3F9E7F841B58547F8
:101A6000E380F9F0DA852D4597000000E78020CB70
:101A70009389F4FFE38404E297000000E78060C8E4
:101A800093F7390091EB832604800327090093071D
:101A90004900E396E6E03E89CE84D9BFB547639915
:101AA000F9001305900B97000000E78080C3FDB399
:101AB000B1471305B00AE388F9FE99476397F90423
:101AC000B7050800B365BB002D4597000000E7800F
:101AD00000C581448D4BA14997000000E78060C29A
:101AE00063967401832704802320F9008504E3951D
:101AF00034FF8327048013172B016355070023123B
:101B0000F90069BB2322F90051BB9D47639FF9028D
:101B100081451305B00497000000E78040C0BD4434
:101B20002320090023220900FD5997000000E780C7
:101B300040BD93F77400CA9703C70700FD14398DA1
:101B40002380A700E39334FF91BBA1476397F90675
:101B500097000000E780A0C28144630D0B008D4711
:101B60009304C0036308FB009304000563048B0126
:101B7000930440041375C507E30295D219459700F5
:101B80000000E78000B697000000E780A0B605459A
:101B900097000000E780E0B4268597000000E7800A
:101BA00020B7094597000000E78080B69700000045
:101BB000E780E0BCE31405CE0DB39147639FF900C5
:101BC0001305600697000000E780A0B197000000B1
:101BD000E78040B213059009F9B5E38109CCF154CF
:101BE0007DB9BD660147173600001306E6239386CC
:101BF00006A685458347060093F7F70F91C38280B9
:101C00000507E3F9E6FE97370000238FB720DDB71D
:101C10007D166206618693178601E18763D407000B
:101C200001458280931726003307F500AE971843CD
:101C30009C4363E7E7007D16E37FF7FC7D558280D8
:101C400005458280FD15E205E185139785016187D1
:101C500093F7F50F63480700FD15139725002A97A2
:101C6000584365D713851700620561858280330864
:101C7000B5021C4283A80600B335B502C29733B53E
:101C80000701AE98469585486367B5006394A50043
:101C900063E3070181480C43C6950CC388C21CC28C
:101CA000828081471397870161876343B7008280F1
:101CB000139727002A97232007008507E5B7814758
:101CC000014793968701E18663C5B6001335170077
:101CD000828093962700AA9694428507558FD5B7A0
:101CE00093D755408A07AA979C4305453315B500FD
:101CF0007D8D828017F3FFDFE702A33D2A849700E2
:101D00000000E78060F405C5931725003E94032783
:101D1000C4FF814711EB7D1516053E9542054185AF
:101D200017F3FFDF6700233D05838507E5B701450E
:101D3000C5BF81471397870161876343C7008280CE
:101D400013972700B386E50094422A97850714C3AA
:101D5000D5B77D1662066186014793178601E18734
:101D600063D5070013351700828093172600B3064A
:101D7000F500AE9794429C437D16B58F5D8FF1BF01
:101D80008A05AA9501476363B500828083A6C5FFD3
:101D9000F11593D71600D98F9CC11397F601E5B7BB
:101DA0002A830148014701456343D7008280B387F6
:101DB000050183A80700B30706019C43C697AA97AD
:101DC0006384F80033B517010507B3080301620700
:101DD00023A0F80061871108C1BF2A83014781470A
:101DE000014563C3D70082803388E500832808005B
:101DF000330EE600032E0E003388A8403308C84196
:101E00006384080133B508018507B308E300E207DE
:101E100023A00801E1871107E9B717F3FFDFE70205
:101E2000432B0111B286B2842E86AA850A859700BB
:101E30000000E780C0FA2A84A6850A859700000082
:101E4000E78020E833348000060413351500018D47
:101E5000056117F3FFDF6700032A17F3FFDFE702CF
:101E6000C3244111AA89AE8A328BB68402C202C44D
:101E700002C60144131C8401135C8C4163499C021B
:101E8000939B1400FD1B0549138CF4FFF15C330494
:101E90008901620461846340740792478E04CE9482
:101EA00023AEF4FE410117F3FFDF6700832313190C
:101EB0002400B30B2B01014A93172A00D69783A560
:101EC0000B00884378003400500097000000E78042
:101ED00040DA050A93178A01E187F11BE35EFCFCF7
:101EE00092474E9905042320F900A2473EC2B2470B
:101EF00002C63EC441B7131A8901135A8A41131D01
:101F0000240093178A01E18763CF970092470A0460
:101F10004E941CC0A24705091379F90F3EC2B2477F
:101F200002C63EC4ADB7B3079A0313152A005695EF
:101F30000841780034005000050AEA97DA978C438C
:101F400097000000E780E0D26DBF0000197106C263
:101F500012C416C61AC81ECA22CC26CE2AD02ED229
:101F600032D436D63AD83EDA42DC46DECAC0CEC2D9
:101F7000D2C4D6C6DAC8DECAE2CCE6CEEAD0EED209
:101F8000F2D4F6D6FAD8FEDA971500009385058CC0
:101F90008841E700050092402242B2424243D243C8
:101FA0006244F244025592552256B2564257D257D5
:101FB0006258F25806499649264AB64A464BD64BCD
:101FC000664CF64C065D965D265EB65E465FD65F55
:101FD0000961730020300000972100209381810265
:101FE000175100201301018217F5FFFF1305C501EA
:101FF0009705002093850501171600201306C6FDDE
:1020000063FAC5008322050023A055001105910540
:10201000E3EAC5FE170502001305854E971500205B
:102020009385C5FB171600201306C66563FAC50025
:102030008322050023A0550011059105E3EAC5FEA2
:102040001715002013050564974500209385852901
:102050006377B500232005001105E36DB5FEFD4251
:10206000739002BC8D4273904280B722000093822D
:10207000828873900230970200209382A2F893E244
:1020800032007390523097520000938222917390E5
:1020900012346FB0F47673002030397101436EC68C
:1020A00019A0397141536AC866CA62CC5ECE19A0C4
:1020B000397101535AD056D252D44ED64AD826DA64
:1020C00022DC06DE33016140828241114AC026C211
:1020D00022C406C68282B24D4101024D924C224C6E
:1020E000B24B4101024B924A224AB2494101024994
:1020F00092442244B240410182803D432A87637367
:10210000C3029377F700BDEFADE5937606FF3D8AF6
:10211000BA960CC34CC30CC74CC74107E36BD7FE40
:1021200011E28280B306C3408A06970200009696A9
:102130006780A6002307B700A306B7002306B700F1
:10214000A305B7002305B700A304B7002304B70015
:10215000A303B7002303B700A302B7002302B7000D
:10216000A301B7002301B700A300B7002300B70005
:10217000828093F5F50F93968500D58D9396050192
:10218000D58D61B7939627009702000096968682B8
:10219000E78086FA9680C1171D8F3E96E374C3F8D8
:1021A000A5B73367B500FD530D8B79E7B7877F7F00
:1021B0009387F7F710419441B372F6003363F6004A
:1021C000BE92B3E262006397720C6318D606504168
:1021D000D441B372F6003363F600BE92B3E26200FC
:1021E0006398720A631BD60410459445B372F600D7
:1021F0003363F600BE92B3E262006391720A631E1B
:10220000D6025045D445B372F6003363F600BE9251
:10221000B3E26200639A72086311D60210499449CE
:10222000B372F6003363F600BE92B3E262006393CA
:1022300072085105D105E30FD6F6131706019397DF
:102240000601631CF7001357060193D706013305F7
:10225000F7409375F50F91E982804183C18333057F
:10226000F7409375F50F91E182801377F70F93F79D
:10227000F70F3305F74082800346050083C605004B
:10228000050585056313D60065FA3305D6408280BF
:1022900011059105E312D6FE014582802105A105B5
:1022A000E31CD6FC014582803105B105E316D6FC5E
:1022B000014582804105C105E310D6FC01458280BD
:1022C000B717004003C777051377E70FA38BE70421
:1022D000130700F8A38DE7043D47238CE704130799
:1022E0005003A38CE70403C7A7051377D70F238DEB
:1022F000E7048280B717004003C7E7020D89411148
:102300001377C70F498F93068008F3B6068093F6BC
:10231000860836C601000100930670052380D704A5
:10232000930680FA2380D704010001002387E70287
:1023300023800704B247F3A7078001000100410191
:10234000828041112A83014E930E407E130F0019A3
:10235000930F400663E56E129308001913034006BD
:10236000B3781503854E0D4FA14F337365020D8968
:102370001335150063EFBE121308F6FF7946729805
:102380004208135808013307C70213D61700BE07C7
:1023900032976146B3F6C60213068070B386C60252
:1023A0003697A166F58F42075D8FB716004083C749
:1023B000F60293F70708A303F1000346710083C7F1
:1023C000F60293F70708E394C7FE83477100B71638
:1023D000004093F7F70F6388071293078008F3B75D
:1023E000078093F787083EC401000100B71700403B
:1023F000930670052380D704930680FA2380D704C0
:102400000100010023AA070383C6170393E6060809
:10241000A388D70223800704A247F3A707800100FF
:1024200001001166B71700407D16D45BC85F938525
:102430004703A98EF18EF5FA93068008F3B606805D
:1024400093F6860836C601000100930670052380C6
:10245000D704930680FA2380D7040100010098C1B5
:1024600003C7170313670704A388E7022380070441
:10247000B247F3A7078001000100410182807D136C
:102480003368E3039308E016630E08003368F30330
:102490009308D016630808009378330093B81800A7
:1024A0009388D81633081E01131E0801135E0E010F
:1024B00055B56393E5030548638608000148630347
:1024C00003002A8871087298FD15131E0801C205C1
:1024D000135E0E01C18179BD13F8150063F4BF00CE
:1024E0007908D5B713381800E5BF83C7F60293F70C
:1024F0000708A303F1000346710083C7F60293F7B0
:102500000708E394C7FE8347710093F7F70FF1DFE5
:10251000E9B531714AD966CB06DF22DD26DB4ED71D
:1025200052D556D35AD15ECF62CD6AC96EC7AA8C36
:1025300002D897100000E78020B12A89930780080D
:10254000F3B7078093F787083EDA01000100B71759
:102550000040130770052380E704130780FA2380E7
:10256000E7040100010003C7F7021377770FA38781
:10257000E70203C7F70213678700A387E7022380F8
:102580000704D257F3A70780010001000545970013
:102590000000E78060D6130780C13347E902116A63
:1025A00093070AE893065002BD69930BA004814A81
:1025B000014B13048008930470057D1AB347F90298
:1025C0003307D7023EC0FD873ECC938709A6930907
:1025D000803E3347F7023AC27D873AC43347390316
:1025E0008549B399990193D93940B306D702B30B02
:1025F0007703B3C6F602B3CBFB0236C6FD8636C8F8
:1026000093D6FB4136CEB7460F0093860624334956
:10261000D9028566938606FAB3969601B389E902D4
:10262000130760553309D90293060010B389E902F4
:102630003349D902B3C9F9029316390036CA37199A
:102640000040FD8636D0930D090493D7F9413ED260
:10265000F336048093F6860836DC01000100930708
:1026600070052380FD00930680FA2380DD000100C1
:1026700001008346390593F6860FA309D9048346E2
:10268000390593E61600A309D90423800D00E2560C
:10269000F3A6068001000100130C80FA116DF336D9
:1026A000048093F6860836DE01000100930770056A
:1026B0002380FD0023808D01010001008346390540
:1026C000216693E60602A309D90483560905B3E6F9
:1026D000A6012318D90483560905D18E2318D904DD
:1026E00023800D00F256F3A6068001000100834608
:1026F000390593F606026381061A03463905218AD5
:102700006DDE081897100000E7800098733604808B
:1027100013768608B2C20100010023809D00238049
:102720008D0101000100B717004003C6370513767D
:10273000F60DA389C70403C6370513660602A389ED
:10274000C704835609052166B3E6A6012318D904F8
:1027500083560905D18E2318D90423800D0096468F
:10276000F3A60680010001008346390593F60602B0
:10277000638B061483463905A18AEDFE970000207D
:10278000E7806091AA8636D497000020E780A09069
:10279000A256E30AD5FE835609054255B3E6A601C3
:1027A0002318D90497100000E780C08F83463905AD
:1027B000A18AEDDE03560905834629058247337653
:1027C000CA00B306DA0293D5F641B296B388F64052
:1027D000E24733B8C6002E983308F840A247B3B694
:1027E00016013308D84063C70701631DF8009247FC
:1027F00063FA1701C247634FF80E63950701B247AA
:1028000063EAF80E894663E9660FF24693151800ED
:1028100013D3F8015E8613951800B365B30042D652
:1028200046D497C00100E780E0E23258050B137BE5
:10283000FB0F63470001631A0838A2586387083802
:1028400013081500B336A800B69513D6F5013298D3
:10285000B336C800AE9613581800FE06B3E606015C
:102860007336048013768608B2C601000100238007
:102870009D0023808D01010001000356C902B2961C
:10288000C206C1822316D90223800D00B646F3A6E4
:1028900006800100010021B5F336048093F6860816
:1028A000B6C00100010023809D0023808D0101003E
:1028B00001008346390593E60602A309D904238063
:1028C0000D0086460DB5F336048093F68608B6C42F
:1028D0000100010023809D0023808D010100010083
:1028E0008346390593E60602A309D90423800D0027
:1028F000A646BDB5E30B0BF0F336048093F68608CD
:10290000B6C801000100930680FA23809D00238051
:10291000DD00010001008346390593F5FC0F93F6B5
:10292000860FA309D90483463905CD8EA309D9049E
:1029300023800D00C646F3A60680010001001305A2
:1029400080FA03463905930639051D8A631C9629CA
:102950007336048013768608B2CC0100010013069A
:1029600080FA23809D002380CD000100010003C672
:1029700006001376F60D2380C60003C60600136614
:1029800006022380C600835609051166D18E2318DE
:10299000D904835609052166D18E2318D9042380D2
:1029A0000D00E646F3A6068001000100130680FA3A
:1029B0008346390593F60602638006268346390569
:1029C000130C3905A18AFDDA081897000000E7808A
:1029D000A06BF336048093F68608B6D001000100A0
:1029E000930680FA23809D002380DD000100010012
:1029F00083460C00116693F6F60D2300DC00834637
:102A00000C0093E606022300DC0083560905D18EF4
:102A10002318D904835609052166D18E2318D904B9
:102A200023800D008656F3A60680010001001306E0
:102A300080FA8346390593F60602638A06208346A8
:102A40003905A18AEDFE97F0FF1FE780C0642A8C4C
:102A500097F0FF1FE7802064E30C85FF835609058C
:102A600011664255D18E2318D90497000000E780E3
:102A700060638346390513063905A18AFDDAF3360A
:102A8000048093F68608B6D401000100930680FA0C
:102A900023809D002380DD000100010083460600A5
:102AA00093F6F60D2300D60023800D00A656F3A65C
:102AB0000680010001008356090503462905D24717
:102AC000B376DA003306CA021305800C9355F6413B
:102AD0003696330DF6408257333CD6002E9C333663
:102AE000A601330CFC40330CCC40330885039256CE
:102AF0004E86B335A5033305A503C29597C00100E3
:102B0000E78040B563468001631E0C16630C0D160A
:102B1000130615003335A6002E959356F50136960B
:102B2000B335D600AA959396F50105828585D18E99
:102B30006346B000639D051A638B061A0356C902EB
:102B400015823305D6003336C500B2956348B00010
:102B5000639105241306F00F637DA622894663F373
:102B6000561593078008F3B7078093F78708BED6FA
:102B70000100010037170040930770052300F70498
:102B8000930780FA2300F704010001008356C7026F
:102B900089678117D58FC207C1832316F7022300E7
:102BA0000704B657F3A7078001000100FA506A54E2
:102BB000DA544A59BA592A5A9A5A0A5BFA4B6A4C59
:102BC000DA4C4A4DBA4D296182801308F5FF33353E
:102BD000A800FD152E951356F5013298B336C8009E
:102BE000AA9695B9F336048093F68608B6CA010012
:102BF000010023809D002380AD0001000100834679
:102C00003905CD8EA309D90423800D00D646F3A63D
:102C100006800100010035B3F336048093F6860880
:102C2000B6CE0100010023809D002380CD0001006D
:102C300001008346390593E60602A309D9042380DF
:102C40000D00F646F3A606800100010095B3F336A9
:102C5000048093F68608B6D20100010023809D000F
:102C60002380CD00010001008346390593E606026A
:102C7000A309D90423800D009656F3A6068001000F
:102C8000010045BB9306F5FF33B5A600FD152E9553
:102C90009355F501AE96B3B5B600AA951396F50116
:102CA000858269B5F336048093F68608B6D80100AC
:102CB0000100930680FA23809D002380DD0001003F
:102CC00001008356C9020566011693F6F60FD18EF0
:102CD000C206C1822316D90223800D00C656F3A670
:102CE000068001000100850A93FAFA0F95B233E6D7
:102CF000B60045C20356C9023305D0403338A000A0
:102D0000B305B040B385054115826345B000D1E1FC
:102D10006371A608894663F0560593078008F3B7E8
:102D2000078093F78708BEDA01000100B71700405B
:102D3000130770052380E704130780FA2380E70454
:102D40000100010003D7C7027D8B2396E702238091
:102D50000704D65781BDF336048093F68608B6DCA7
:102D600001000100930680FA23809D002380DD008E
:102D7000010001008356C9020566011693F6F60F9D
:102D8000D18EC206C1822316D90223800D00E656D9
:102D9000B9B793078008F3B7078093F78708BEDEBB
:102DA0000100010037170040930770052300F70466
:102DB000930780FA2300F704010001000356C702BD
:102DC00093975600B297C207C1832316F7022300D8
:102DD0000704F657C1BB914763EEB70217D701004E
:102DE0001307C7728A05BA959C41BA978287B717AD
:102DF000004003A7470B1345F5FF698F23AAE70A95
:102E000003A7070B698F23A8E70A03A7070A798D91
:102E100023A0A70A8280B717004083A6470B134759
:102E2000F5FFF98E23AAD70A83A6070B558D23A891
:102E3000A70A83A6070A758F23A0E70A8280B7171F
:102E4000004003A7470B498F23AAE70A03A7070BF4
:102E50001345F5FF45BFB717004083A6470B13473F
:102E6000F5FF758F23AAE70A03A7070A598D4DB707
:102E7000B717004003A7470B498FEDB7914763EEA3
:102E8000B70217D701001307A7698A05BA959C41B5
:102E9000BA978287B717004003A7470D1345F5FF80
:102EA000698F23AAE70C03A7070D698F23A8E70CF6
:102EB00003A7070C798D23A0A70C8280B7170040C9
:102EC00083A6470D1347F5FFF98E23AAD70C83A6D7
:102ED000070D558D23A8A70C83A6070C758F23A07B
:102EE000E70C8280B717004003A7470D498F23AA3C
:102EF000E70C03A7070D1345F5FF45BFB7170040C3
:102F000083A6470D1347F5FF758F23AAE70C03A788
:102F1000070C598D4DB7B717004003A7470D498FD0
:102F2000EDB7797122D43714004026D24AD0035924
:102F300024028354040206D64209C2044ECE52CC67
:102F400056CA13590901C1802DE11379F9F793F499
:102F5000F49F4209C20413590901C18093078008F4
:102F6000F3B7078093F787083EC401000100930779
:102F700070052300F404930780FA2300F404010091
:102F80000100231124032310940223000404A24708
:102F9000F3A7078001000100B25022549254025955
:102FA000F249624AD24A45618280B7F507008146FC
:102FB0003000B105194597000020E7806081A247E5
:102FC00013972701E34A07FC1369090893E40440B7
:102FD00093098008F3B7098093F787083EC0010082
:102FE0000100930A700523005405130A80FA230098
:102FF000440501000100231124032310940223003F
:1030000004048247F3A7078001000100294597F0D7
:10301000FF1FE7802032F3B9098093F989084EC277
:1030200001000100230054052300440501000100B4
:103030008357040293E707202310F40223000404BB
:103040009247B9B7B7170040884742054181937747
:10305000050491EB9377F5013755E80113050580D9
:103060003345F50282809377050C130700046397BC
:10307000E7009377F50137459C1CCDB72165130513
:1030800005D0828037E700E01C435443A183E20669
:10309000D58F1CC1FD572320F7182322F7188280F3
:1030A00013178500B7E700E023A0E710618123A292
:1030B000A7108280B7F700E08847CC47828081471D
:1030C00037370040A14663C4C7003285828003457C
:1030D000B740E38EA6FE3385F5000345050085075E
:1030E0002304A740CDB797070020938727EF9C4381
:1030F000173700201307071F3E95636EE50017374B
:103100000020130727506368A70017070020232714
:10311000A7EC3E858280FD57EDBF8280411122C41D
:1031200006C62A8497000000E78000F22947B3070B
:10313000E502B2408D83B3D7870222449507B3D707
:10314000E70237370040C207C1832316F700410169
:103150008280411137150E0006C697000000E780F7
:1031600020FCB7370040130770F82381E7000D47B4
:10317000A381E70013070004A380E7000547238726
:10318000E700B24041018280B737004003C7170013
:1031900019C9D98DA380B70003C70700136787003B
:1031A0002380E700828093C5F5FFF98DA380B700E7
:1031B0008280AE872A87B7360040214637380040E4
:1031C00089E717030000670083F583C8B600E309A9
:1031D00016FF05078348F7FFFD17C20723041801F0
:1031E000C183F9BF411122C406C62A84970000009A
:1031F000E78080E52947B307E502B2408D83B3D766
:10320000870222449507B3D7E70237370040C20749
:10321000C1832316F7404101828071654111130576
:10322000052006C697000000E78000FCB737004085
:10323000130770F82381E7400D47A381E740130788
:103240000004A380E74005472387E740B2404101DF
:103250008280CC41411106C6328503C6150083C564
:10326000050022064D8E42068D654186138875A2A3
:10327000630C0611634BC804138845A26300060D56
:10328000634AC800938535A26301B60823900600FF
:1032900029464DA0138855A26305060D938565A2A6
:1032A000E316B6FE8D451D4663E6E5081146198E08
:1032B00063F3C7003E86B7E704002390C600FC47CF
:1032C00097D50100938505289DA0138895A26303D7
:1032D0000611634E060D1388A5A26300061393859D
:1032E00005A5E315B6FA99451D4663E5E504198E73
:1032F00063F3C7003E86B7E704002390C600FC478F
:10330000970500209385C5D71DA09D451D4663E305
:10331000E5022146198E63F3C7003E86B7E7040035
:10332000FC472390C6009705002093852536BA9563
:1033300082970146B240328541018280AD451D46EB
:10334000E3EAE5FE3146198E63F3C7003E86B7E730
:1033500004002390C600FC4797D501009385052102
:10336000F9B7B1451D46E3E7E5FC3546198E63F331
:10337000C7003E86B7E704002390C600FC4797D5F8
:1033800001009385A51F65B78D451D46E3E4E5FA69
:103390001146198E63F3C7003E86B7E704002390F9
:1033A000C600FC4797D501009385851A49B78D451E
:1033B0001D46E3E1E5F81146198E63F3C7003E862A
:1033C000B7E704002390C600FC4797D5010093851A
:1033D000A51CB1BFA5451D46E3EEE5F42946198EAF
:1033E00063F3C7003E86B7E704002390C600FC479E
:1033F00097D50100938585161DBFB5451D46E3EBA6
:10340000E5F23946198E63F3C7003E86B7E704003C
:103410002390C600FC4797D501009385A51101BFF5
:10342000B7E7040003A3071397060020938646C45A
:103430004146A54517050020130585BA02832D4591
:103440005DE703C505000947631FE50803A84500BC
:10345000411106C6034718003285034608002207BB
:103460004168518F930828FE6307170563E9E80058
:1034700005186303070323900600294591A8130646
:1034800048FE630AC7041518E31707FF15463E8771
:10349000637BF600154701A8130600023E8763749C
:1034A000F60013070002B7E704002390E600FC478C
:1034B0001316070111A83E8691C30546B7E704001D
:1034C000FC472390C6004206CC45418282970145C5
:1034D000B24041018280130600083E87E375F6FC86
:1034E00013070008C9B72390060005458280828033
:1034F000416779176304E504411122C406C6854774
:103500002A84639FF500B7E7040022852244B24075
:1035100003A387139705002093858531410102831A
:1035200089476399F500B7E7040083A7070B854532
:10353000829771D9B24022444101828082807971A0
:1035400026D252CCAE842A8A97D501009385C5062F
:1035500017D501001305C50806D63AC622D44AD0AD
:10356000368432894ECE97B00100E780E059A285BB
:1035700017D501001305C50797B00100E780C058B3
:10358000294597B00100E780005D83C7840093F769
:103590000702F9E383C9040089470545324763966A
:1035A000F908D44083C7160083C60600A207D58F4A
:1035B000C166138616FE638CC7028D16638FD7060D
:1035C0008D669386269029456391D706B7E7040058
:1035D000A286225403A34714B250F2494A86A68514
:1035E000025992545285624A8547456102832D45AE
:1035F0000DEF93070002354563E98702B7E7040042
:10360000FC47C84413060002CA8582978149970780
:1036100000209387A7229C43014581CB9C4391C7FF
:103620004E852286CA8582970145B2502254925413
:103630000259F249624A456182802D457DF7930720
:10364000700F3545E3E387FEB7E70400FC47C84445
:103650002286CA85829765BF2145C1BF411122C418
:1036600037E404008327841326C2AA84416506C672
:10367000970500209385C51B7D1582978327C40A73
:1036800017050000130505E78588829795C0032379
:1036900004132244B2409244970600209386C6AF9A
:1036A0004146C545170500201305059E41010283CB
:1036B000B2402244924401454101828019C59707D6
:1036C000002023ADA7160145828045458280114721
:1036D000636AA70A97D601009386C6EC0A05369559
:1036E0001841411106C63697AE87B2850287130787
:1036F00000026145639DE700B7E70400FC4713063D
:103700000002170500201305E5F882970145B24035
:103710004101828005476145E39BE7FEB7E704006E
:10372000FC470546170500201305C5F8F9BF130728
:10373000700F6145E39DE7FCB7E70400FC47130603
:10374000700F17050020130525F7C1B713070008F0
:103750006145E39EE7FAB7E70400FC47130600085B
:10376000170500201305C5044DB715476145E390C3
:10377000E7FAB7E70400FC471546170500201305D4
:10378000650B61B709458280411126C2B7E4040088
:1037900083A7C41322C44AC006C62E8497050020FE
:1037A000938505092A898297058905C59707002011
:1037B0009387878D83D7A70BA28503A3440D23107E
:1037C000F4002244B24092444A8502490146410134
:1037D0000283B24022449244024949454101828019
:1037E00097070020238E07049707002023AC0704C7
:1037F000B717004003A7070CB706C0FFFD16758F6B
:1038000023A0E70C03A7070DB7064000558F23A898
:10381000E70C03A7070C3D9B23A0E70C03A7070DAC
:103820001367070123A8E70C8280B717004003A5A0
:10383000470C83A7470C598113451500C18B058997
:1038400099E3136525009707002083C767FF63800E
:10385000A702970700202385A7FE11C9970700201C
:10386000938747FE03A3070063030300028382805C
:10387000114517F3FFFF670003CA41119396250016
:10388000AA852D4506C697F0FF1FE78060F4B24079
:10389000014541018280011122CC06CE371400403F
:1038A00026CA4AC84EC652C483447405034AB405A6
:1038B000834984050349940597F0FFFFE78080A0C2
:1038C0008347A40593F4F40F137AFA0F93E71700D4
:1038D000230DF40493F9F90F1379F90FB71700408A
:1038E00003C7A705058B6DFF03D5C705A38D470546
:1038F000238C3705A38C2705A38B9704F2406244E1
:10390000D2444249B249224A0561828041119397CB
:10391000050122C406C626C2C1872E8463DC0700C7
:10392000B7E40400FC54829719C1BC548297216506
:10393000218D15A893F7150013C515008DE793F792
:1039400025009DC797000000E78060EEB7E7040000
:10395000BC4F1306000A894517050020034505EFF3
:10396000829713452400B240224492444101828050
:103970009397250163D80702B7E4040083A7C41E08
:10398000829797000000E780E0EEBC4C37560700B6
:1039900013060630896517050020034525EB82973D
:1039A000096579B7939715010145E3DE07FA17D545
:1039B00001001305E5CB97B00100E780C02CB7E705
:1039C0000400BC4F130600649165170500200345F1
:1039D000E5E782971165A9BF2D71232A9110FD7427
:1039E000E98C232C811023282111232631112A84CC
:1039F000AE893289930600100A86A6852D45232EAE
:103A0000111097F0FF1FE780A0DC13154401B7E702
:103A10000400FC4751810A0513962900CA850A95BE
:103A20008297A68585660146254597F0FF1FE780AA
:103A300020DA0A86A68593060010294597F0FF1F15
:103A4000E78000D98320C11103248111832441110F
:103A5000032901118329C11015618280B7F707007E
:103A600003C70701411106C622C426C24AC0A547A2
:103A7000631DF70097000000E78040F6B240224443
:103A80009244024901454101828013942500AA8491
:103A90003289A286AA850146254597F0FF1FE78057
:103AA00020D3A2864A86A685294597F0FF1FE78086
:103AB00020D2E9B71D71A2CC37E404005C5C485801
:103AC00086CE494697D50100938505B6829711E9C0
:103AD00017D50100130585B697B00100E780A01A3D
:103AE00001A0B7F600E0795798CAFD57DCCA056710
:103AF000B7E700E023A0E7101306F00290C223A06E
:103B0000E7180100010037070020184713060004DA
:103B100081459706002023A9E6D24157A38AE740B2
:103B20003C4408088297970700209387276F3EC878
:103B3000856713870740231AE1001D673ACC3707D2
:103B40000105130707103ACE938757D11307B00F1B
:103B50002310E1022312F102054797F7FFFF938735
:103B6000A7552301E1023ED817070000130727D10C
:103B700097070000938767D2B7F50700BAC23EDC0B
:103B8000170700001307C7ED97070000938787CE3C
:103B900081463000E1051945BAC43EDE97F0FF1FAB
:103BA000E78000C318088147994630003E960346D7
:103BB000060085070507A30BC700E398D7FEC24799
:103BC00091C70357410185676373F70001A0B7E709
:103BD000040083A7470A08088297AA8511C917D548
:103BE00001001305E5A697B00100E780E0F101A010
:103BF000F640664425618280411126C2B7E4040084
:103C000083A7040806C622C417050000130545D083
:103C1000829717040020130464C32300A4009700B4
:103C20000000E780800297000000E780A0BB03450A
:103C30000400224403A38405B240924413060032D8
:103C4000896541010283797106D622D41307800861
:103C5000F337078093F787083EC201000100B717CA
:103C60000040930570052380B704130680FA238073
:103C7000C7040100010083C6F70293F6A60FA387CD
:103C8000D702238007049246F3A6068001000100B4
:103C900073370780137787083AC401000100238037
:103CA000B7042380C7040100010003C7F7021367AC
:103CB0002700A387E70223800704A247F3A7078012
:103CC00001000100054597E0FFFFE780E0629700F3
:103CD0000000E78020BA01478146814705468545B7
:103CE0001305407E97E0FFFFE780E06537E40400BE
:103CF0003C446800514681458297B707C0A83EC83A
:103D0000B787E803938707D03ECA97E7FF1F9387DB
:103D1000076B3EC67C5868008297B25022544561BA
:103D20008280411197D501009385C5FA17D501000E
:103D30001305058B06C697B00100E780E0DC17D5B8
:103D400001001305E51197B00100E780E0DBB24008
:103D50002945410117B301006700E3DF411197D501
:103D60000100938565F817D501001305658706C620
:103D700097B00100E78040D917D501001305050D64
:103D800097B00100E78040D8B2402945410117B300
:103D90000100670043DC411122C406C683470500C9
:103DA0002A849DC797D501009385C5F917D50100D1
:103DB0001305058397B00100E78000D54C4017D567
:103DC00001001305251897B00100E780E0D33DA05E
:103DD00058410DEF97D501009385C5F617D5010021
:103DE0001305058097B00100E78000D217D50100C8
:103DF0001305C51697B00100E78000D12244B240F8
:103E00002945410117B301006700E3D4A1679386F8
:103E1000D7036313D70297D501009385A5F217C581
:103E200001001305E57B97B00100E780E0CD17D5D1
:103E300001001305A5137DBFED0797D501009385FC
:103E400065F017C501001305A579631BF70097B04E
:103E50000100E78060CB17D501001305651259BF3B
:103E600097B00100E78040CA4C4017D50100130508
:103E7000251391BF411197D50100938525E817C5FA
:103E800001001305E57506C697B00100E780C0C7BD
:103E9000B2402945410117B301006700C3CB7971D6
:103EA00022D426D24AD02E842A898145B284480061
:103EB000714606D697E0FFFFE780602497F7FF1F63
:103EC0009387874EDC4783D70700231421012313F0
:103ED000F10097500000E78080E39547A305F100CB
:103EE0009307401F3EC6FD572305A100230AF1009A
:103EF00097500000E780E0F52686A285480097509D
:103F00000000E780A0E3B250225492540259456168
:103F1000828097270020239F078297170020238FF6
:103F2000076EB7E70400BC47411106C6414681450C
:103F3000170500201305051D829797200000E780D4
:103F4000805E97200000E780E04201459750000026
:103F5000E780C070170700200347C71C9307F00ACB
:103F60006315F7029307F0F889451705002013053C
:103F7000651B170700202307F71A97070020A38364
:103F8000071A97600000E780009897600000E780BC
:103F900060C48145370504009707002023A2071657
:103FA00097070020239C07149707002023890714F4
:103FB000970700202398070C970700202396070AED
:103FC00097070020239B07129707002023940714CC
:103FD00097300000E7804021014597600000E780AE
:103FE000809B97D501009385E5D317C50100130584
:103FF000255F97B00100E78020B117D501001305B8
:10400000650097B00100E78020B0B240294541012A
:1040100017B30100670023B4411122C406C626C2AB
:1040200093F715002E84638F0710814617F6FF1F44
:104030001306C6348545170500200355A50297C011
:104040000000E780201E15C997D50100938545CE55
:1040500017C501001305C55897B00100E780C0AA35
:1040600017C501001305856F97B00100E780C0A94F
:10407000294597B00100E78000AE97D501009385F0
:1040800025CB17C501001305A55597B00100E780A2
:10409000A0A717C501001305A56D97B00100E78023
:1040A000A0A6294597B00100E780E0AA17F5FF1FF9
:1040B0001305852F5C4505472390E70097400100D5
:1040C000E780A0CE97D50100938585C617C501006E
:1040D0001305055197B00100E78000A317C5010043
:1040E0001305456A97B00100E78000A2294597B003
:1040F0000100E78040A6930710F81707002023036C
:10410000F7029707002083D7A7F517070020A30B16
:10411000F700170500201305E500A1839145170757
:1041200000202302F70097070020A38E07FE975078
:104130000000E780407D13451400B24022449244C1
:104140004101828093F72500E1C71707002003573C
:10415000E7FA45CF97060020938686FA944297D7D0
:104160000100938727EC17060020034646F9814596
:1041700017050020130505F997700000E780E02976
:1041800097F7FF1F2396A712AA8441C197D5010074
:104190009385C5C017C501001305854497B001007C
:1041A000E7808096A68517C501001305255F97B0A7
:1041B0000100E7806095294597B00100E780A0994C
:1041C00097070020239C07F2930710F81707002099
:1041D000230AF7F49707002083D787E81707002002
:1041E000A302F7F4A18317070020230EF7F29145ED
:1041F0008D47170500201305E5F217070020A304DB
:10420000F7F297500000E78000701345240035B79F
:1042100093F74500D1C397D50100938525B817C5FD
:1042200001001305E53B97B00100E780E08D17C55D
:1042300001001305655897B00100E780E08C29451F
:1042400097B00100E7802091930720F8170700201E
:10425000230AF7EC9707002083D7C7E2170700204F
:10426000A302F7ECA18317070020230EF7EA854786
:1042700017070020A309F7EA97500000E78060BD08
:1042800017050020130505EA914597500000E780C7
:1042900080671345440055B593F78500A9C797D5A6
:1042A00001009385A5AF17C501001305653397B0CD
:1042B0000100E780608517C501001305255197B0FF
:1042C0000100E7806084294597B00100E780A0885D
:1042D00097070020239407E297700000E780C0232F
:1042E0001345840099BD93F70501D1C38545170592
:1042F0000020035525D997600100E780E0D597D5C8
:1043000001009385A5A917C501001305652D97A088
:104310000100E780607F17C501001305654C97A079
:104320000100E780607E294597B00100E780A08208
:10433000930730F8170700202306F7DE97070020C1
:1043400083D747D417070020A30EF7DC17050020FA
:10435000130545DDA1838D45170700202305F7DCF4
:1043600097500000E780205A13450401F9B393F7F2
:104370000502D1C797D50100938545A217C5010055
:104380001305052697A00100E780007817C50100F6
:104390001305454797A00100E7800077294597A0BE
:1043A0000100E780407B930740F817070020230BAC
:1043B000F7D69707002083D727CB17070020A30342
:1043C000F7D6A18317070020230FF7D485471707D7
:1043D0000020A30AF7D497070020239707C8975017
:1043E0000000E78000A7170500201305A5D391451D
:1043F00097500000E7802051134504023DBB93F71E
:104400000504FDC397D501009385459917C50100A3
:104410001305051D97A00100E780006F17C5010077
:104420001305C53F97A00100E780006E294597A0BE
:104430000100E78040729707002083C7A7CE1307CB
:10444000700A6386E7061307800A638CE708130780
:10445000600A6393E704930760F8170700202303BB
:10446000F7CC9707002083D747C917070020A30B75
:10447000F7CAA183170700202307F7CA8547170744
:104480000020A306F7CAB14517050020130585C90A
:1044900097500000E780204797500000E780609B1E
:1044A0001345040497070020239907C479B19307A3
:1044B00070F8170700202307F7C69707002083D757
:1044C000C7C317070020A30FF7C4A1831707002055
:1044D000230BF7C4854717070020A307F7C49945A6
:1044E00065B7930780F8F1B793F705080145E386B0
:1044F00007C497D501009385658A17C50100130588
:10450000250E97A00100E780206017C50100130564
:10451000653297A00100E780205F294597A0010040
:10452000E78060639307A0F817070020230CF7BE0D
:104530009707002083D707BE17070020A304F7BE04
:10454000A183170700202300F7BE85471707002027
:10455000A30BF7BC97070020239E07BA97500000D3
:10456000E780208F170500201305C5BB91459750A4
:104570000000E780403913450408C1B6411122C448
:1045800097C501009385457D2A8417C50100130551
:10459000250506C697A00100E78000574C4017D5B7
:1045A00001001305A59797A00100E780E055294574
:1045B00097A00100E780205A034704009307F00FFB
:1045C000631FF70297C501009385057917C50100A0
:1045D0001305050197A00100E78000534C4017D553
:1045E00001001305A59497A00100E780E051224443
:1045F000B2402945410117A301006700C355B240ED
:10460000224441018280B1C1411122C417C5010079
:10461000130505FD2E8497C501009385E56E06C63A
:1046200097A00100E780404EA28517D50100130531
:10463000259B97A00100E780204D2244B2402945E8
:10464000410117A30100670003518280411122C478
:1046500026C22E84AA8497C501009385A56B17C531
:1046600001001305E5F706C697A00100E780C049E1
:1046700017D501001305859797A00100E780C04872
:10468000294597A00100E780004D97C5010093855B
:104690006568970700202397979C17C501001305AD
:1046A00025F4854497070020239C879A97070020CC
:1046B0002399979A97170020239E870897A00100B7
:1046C000E78080449715002083D5C50817D50100E1
:1046D0001305459297A00100E7800043294597A064
:1046E0000100E780404797170020238997F2972021
:1046F0000000E78020C8228597500000E78000F680
:10470000054597500000E780002997F7FF1F938722
:10471000A7C9DC4703D70700C167FD176312F7027B
:104720002244B7E70400B240924403A3870517F57B
:10473000FF1F034525121306000A85454101028328
:10474000B2402244924441018280011122CC37E4DC
:1047500004005C5C06CE354697C5010093858571E3
:1047600017D501001305853F829711E917C5010090
:104770001305C5EC97A00100E780E05001A097F772
:10478000FF1F9387E70D3EC4B7F507008567938742
:104790000780814617F6FF1F1306060CE105194531
:1047A0003EC697E0FF1FE780A0027C44194697F5BC
:1047B000FF1F9385650A170500201305E58C829776
:1047C000340017F6FF1F1306260997D501009385BD
:1047D000E5BB17D501001305E5BC97700000E78025
:1047E000C0982A841DCD97C501009385255A17C509
:1047F00001001305E5DE97A00100E780E030A28507
:1048000017C501001305056897A00100E780C02FB8
:10481000294597A00100E7800034F2406244056119
:10482000828097E00000E78020FB17C50100130598
:10483000655C97600000E780008D97A00000E7802E
:10484000604F97600100E780E0B317F5FF1F130585
:1048500025B297600100E780809C17C50100130511
:10486000655A97600100E78060B42A849760000071
:10487000E78040F397100100E780C08B978001002C
:10488000E780E02497700000E780804B976000008D
:10489000E780406997300100E780204D97C501000F
:1048A0009385C54E17C50100130585D319C897A078
:1048B0000100E7806025A28517C501001305C55ECC
:1048C000A1B797A00100E780202417C501001305B8
:1048D000E55F97A00100E7802023294597A001000C
:1048E000E780602797300100E780002997F00000FB
:1048F000E780C04755C9854537050400973000005B
:10490000E780808E97C501009385454817C5010053
:10491000130505CD97A00100E780001F17C5010012
:104920001305455C97A00100E780001E294597A06C
:104930000100E780402297F7FF1F9387679683D790
:104940000700171700202317F7E0854717170020E7
:104950002306F7CC97200000E780A0B59720000041
:10496000E78040A1171500200355C5DE97500000D1
:10497000E780C0CE054597500000E780C00197C58D
:1049800001009385A54017C50100130565C597A0D3
:104990000100E780601717C501001305E55697A0D1
:1049A0000100E7806016ADB597C501009385053E0F
:1049B00017C501001305C5C297A00100E780C01408
:1049C00017C501001305056497A00100E780C01317
:1049D000294597A00100E7800018014569BF4111F2
:1049E00022C437E404008327041A06C6829797502E
:1049F0000000E78060CA8327040817F5FFFF13054E
:104A0000E561829797F7FF1F2386A7E417F5FF1F3D
:104A10001305859997400000E78040762244B24014
:104A2000410117030000670083D2B7E70400FC4789
:104A30001171A2DDCAD986DFA6DBCED72E843289DA
:104A40002E86AA8517F5FF1F1305C56D829717F7E8
:104A5000FF1F1307276D8347070093068002938784
:104A6000E70793F7F70FE3ECF610BA898A0717C741
:104A70000100130727C0BA979C43BA9782878D47D6
:104A800097C501009385C53217C50100130545B5CB
:104A9000630FF40097A00100E780000717C501002D
:104AA0001305C5EF97A00100E7800006BDA497A0FD
:104AB0000100E780600517C501001305A5EF97A069
:104AC0000100E7806004294597A00100E780A00865
:104AD000930720F8114697F5FF1F9385A5644A8533
:104AE00017F7FF1F2300F76497F7FF1FA38D0762D7
:104AF00097F0FFFFE780E03A2A841DC997C50100BF
:104B00009385052B17C50100130585AD97A00100FE
:104B1000E78080FFA28517C50100130565ED97A00A
:104B20000100E78060FE294597A00100E780A00210
:104B300097C501009385C52717C50100130545AA30
:104B400097A00100E78040FC17C50100130585EB25
:104B500097A00100E78040FB294597A00100E7806E
:104B600080FF4165930730FA054697F5FF1F93854F
:104B7000655B7D1517F7FF1F2306F75A97F0FFFFB8
:104B8000E78020322A841DC997C5010093854522FC
:104B900017C501001305C5A497A00100E780C0F662
:104BA000A28517C501001305A5E497A00100E780C1
:104BB000A0F5294597A00100E780E0F9B7E70400D8
:104BC000BC4F0566130606C8A14517F5FF1F034530
:104BD00065C88297FE506E54DE544E59BE5911611D
:104BE000828091476303F40297C501009385451CB9
:104BF00017C501001305C59E97A00100E780C0F00E
:104C000017C50100130545E371BDB7E70400FC4F6C
:104C1000914517F5FF1F0345E5C3829797C501002E
:104C20009385051917C501001305859B97A0010001
:104C3000E78080ED17C501001305C5E197A00100CD
:104C4000E78080EC294597A00100E780C0F09740FD
:104C50000000E7800020914535A485476303F402F6
:104C600097C501009385C51417C501001305459725
:104C700097A00100E78040E917C50100130505DF93
:104C800015B597F7FF1F239F273FB7E70400056679
:104C9000BC4F130606C8C1450DBF8D476303F40220
:104CA00097C501009385C51017C5010013054593ED
:104CB00097A00100E78040E517C501001305C5DC9A
:104CC000D5B3930740F8114697F5FF1F93858545A7
:104CD0004A8517F7FF1F2307F74497F7FF1FA384A1
:104CE000074497F0FFFFE780C01B2A84E30405EE2A
:104CF00097C501009385C50B17C501001305458EA7
:104D000097A00100E78040E0A28517C501001305C8
:104D100025CE97A00100E78020DF294597A001005C
:104D2000E78060E345BD9147E31CF4F6B7E7040074
:104D3000FC4F9305000217F5FF1F0345A5B18297AD
:104D400097C501009385C50617C501001305458960
:104D500097A00100E78040DB17C50100130545D48B
:104D6000F1BD894763E3870297C501009385450438
:104D700017C501001305C58697A00100E780C0D8BC
:104D800017C50100130505D331BB97F4FF1F83C47A
:104D9000843997F7FF1F83C7F73897C501009385BC
:104DA0002501A20417C5010013058583DD8C97A09A
:104DB0000100E78060D5A28517C501001305C5D0A5
:104DC00097A00100E78040D4C204294597A00100C4
:104DD000E78060D8C1849305D4FF93960401C18213
:104DE0004A8693F5F50F17F5FF1F1305D533972066
:104DF0000000E7802043E35F90DC930750F817F74B
:104E0000FF1F2301F73283C73900228697F5FF1F62
:104E10009385453185074A8517F7FF1FA305F730AE
:104E200097F0FFFFE780E0072A84E30505DA97C5DE
:104E300001009385E5F717B501001305657A97A082
:104E40000100E78060CCA28517C501001305451855
:104E5000C9B5894763E3870297C50100938545F586
:104E600017B501001305C57797A00100E780C0C9F9
:104E700017C50100130505C735B197400000E7804D
:104E800040FDA28517F5FF1F1305C52997500000A7
:104E9000E78060A781B38D476303F40297C50100E3
:104EA000938505F117B501001305857397A00100DF
:104EB000E78080C517C50100130585C4E5B6B76650
:104EC00002000146B7750200054597E0FF1FE78025
:104ED0002090930760F817F7FF1F2305F72497F733
:104EE000FF1FA38207249307000617F7FF1F230D58
:104EF000F722894717F7FF1FA308F72297F7FF1F2D
:104F00002385072297F7FF1FA3810722C14717F7C1
:104F1000FF1F230DF720930720F917F7FF1FA307A3
:104F2000F720314697F7FF1FA383A72097F5FF1FB0
:104F30009385451F4A8597F7FF1F238A071E97F021
:104F4000FFFFE78000F62A84E30605C897C5010045
:104F5000938505E617B501001305856897A0010044
:104F6000E78080BAA28517C501001305E5BA55B3DD
:104F7000B1476303F40297C50100938565E317B554
:104F800001001305E56597A00100E780E0B717C5AC
:104F90000100130525BA39B6B7E70400FC4F9305A5
:104FA000000417F5FF1F0345E58A8297974000002C
:104FB000E78020EAB145F9B5914763E3870297C5D9
:104FC00001009385E5DE17B501001305656197A023
:104FD0000100E78060B317C50100130565B7D9B4B8
:104FE00097F4FF1F83C4441497F7FF1F83C7B713B9
:104FF000A204DD8C8E04B77702006D14BE94228665
:10500000A68517C501001305E5B597A00100E78047
:10501000A0AFB7E70400FC47228697F5FF1F9385F2
:10502000B5102800829793160401C1823000A6852E
:10503000094597D0FF1FE780A0792A8409C917C5C1
:1050400001001305E5B397A00100E780C0C39307F3
:1050500070F8194697F5FF1F9385C50C4A8517F719
:10506000FF1F2301F70C97F7FF1FA38F870A97F005
:10507000FFFFE78000E32A84E30E05B497C5010033
:10508000938505D317B501001305855597A0010039
:10509000E78080A7A28517C50100130565AF95B904
:1050A0009947630BF41297C50100938565D017B536
:1050B00001001305E55297A00100E780E0A417C5A1
:1050C0000100130565AEF9BA914763E3870297C5FE
:1050D00001009385E5CD17B501001305655097A034
:1050E0000100E78060A217C50100130565AD5DBA38
:1050F00097F4FF1F83C4440397F7FF1F83C7B702CA
:10510000A204DD8C8E04B77702006D14BE94228653
:10511000A68517C501001305E5AB97A00100E78040
:10512000A09EB7E70400FC47228697F5FF1F9385F2
:10513000B5FF2800829793160401C1823000A6852E
:105140000D4597D0FF1FE780A0682A8409C917C5BD
:1051500001001305E5A997A00100E780C0B29307FD
:1051600080F8194697F5FF1F9385C5FB4A8517F709
:10517000FF1F2309F7FA97F7FF1FA38787FA97F016
:10518000FFFFE78000D22A84E30605A497C501004B
:10519000938505C217B501001305854497A001004A
:1051A000E7808096A28517C501001305A5A595B6D1
:1051B00099476303F40297C50100938565BF17B54E
:1051C00001001305E54197A00100E780E09317C5B2
:1051D00001001305A5A4F9B0B7E70400FC4F93053F
:1051E000000417E5FF1F0345E5668297974000001E
:1051F000E78020C6994579B18D476303F40297C5CE
:1052000001009385E5BA17B501001305653D97A028
:105210000100E780608F17C501001305A5A159B0F3
:1052200017C50100130505A297A00100E780A0A5FE
:105230001305C01297D0FF1FE780A010014597E02B
:10524000FFFFE78060E40D4597100000E78080A035
:10525000294597D0FF1FE780C00E97D0FF1FE7803A
:1052600020FF8DBA99476303F40297C50100938527
:1052700025B417B501001305A53697A00100E780F6
:10528000A08817C501001305A59C29B817F7FF1FB3
:10529000034797E997F7FF1F83C707E922075D8F49
:1052A0009166BA96C2061166C1821306F6EF8D4763
:1052B0006365D60297E7FF1F9387070F9C4B17F68E
:1052C000FF1F034656E69386C7002DC203D607008C
:1052D00069CA8907E39CD7FE89471307A0F81146DE
:1052E00097F5FF1F938505E44A8597F6FF1F238BEB
:1052F000E6E217F7FF1FA308F7E297F0FFFFE7804A
:1053000040BA2A84E308058C97C50100938545AA15
:1053100017B501001305C52C97900100E780C07EEA
:10532000A28517C501001305E593E5B203D6070072
:10533000630EE60A8907E39BF6FE8D4779BF914726
:105340006304F40297C50100938585A617B5010093
:105350001305052997900100E780007B17C5010020
:105360001305C5916FF00FF4B7E70400FC4F9305E8
:10537000000817E5FF1F0345E54D8297C9B897C59B
:1053800001009385E5A217B50100130565259790E7
:105390000100E780607717C501001305A58F6FF046
:1053A0006FF02390E70017E5FF1F1305E5FF973027
:1053B0000100E780E0A197C501009385659F17B5BF
:1053C00001001305E52197900100E780E07317C500
:1053D00001001305258D97900100E780E0722945B3
:1053E00097900100E78020778147C5BD2390070093
:1053F00017E5FF1F130545FB97300100E780409D2F
:1054000097C501009385C59A17B501001305451D81
:1054100097900100E780406F17C501001305058ACA
:105420005DBF411122C406C6834705002A849DC77B
:1054300097C501009385859317B501001305451A9B
:1054400097900100E780406C4C4017C501001305A0
:1054500065BE97900100E780206BC9A85841B70747
:10546000CF009387777D6312F70897C50100938576
:10547000E58F17B501001305A51697900100E78089
:10548000A0681C448356E4008355C40003C607008B
:1054900017C50100130585BB97900100E780C06622
:1054A000294597900100E780006B0357E4009707B8
:1054B000002083D7272A630EF7008355C4000844D1
:1054C000854717070020230EF72497300000E78058
:1054D000E0370356E4008355C40008442244B24038
:1054E000410117F3FFFF67008354B707CC00938790
:1054F000777D6315F70497C501009385258717B558
:1055000001001305E50D97900100E780E05F1C4462
:105510008356E4008355C40003C6070017C5010085
:105520001305C5B297900100E780005E2244B240A7
:1055300029454101179301006700E361B707CE00D9
:105540009387777D6304F70297C5010093850582F1
:1055500017B501001305C50897900100E780C05AF0
:105560004C4017C501001305A5A3E5B5B240224480
:1055700041018280B7E70400FC4741112E8606C630
:1055800022C426C24AC02E842A89AA8517F5FF1F85
:10559000130545B9829797C501009385258317B5F3
:1055A00001001305E50397900100E780E05597F5AA
:1055B000FF1F83C525B717B501001305252997904F
:1055C0000100E7806054294597900100E780A058CA
:1055D00097F4FF1F938404B583C704004147938762
:1055E000070693F7F70F636EF75A17B70100130713
:1055F000A7128A07BA979C43BA9782879D47630789
:10560000F40297B501009385657C17B50100130579
:1056100025FD97900100E780204F17B50100130585
:10562000652397900100E780204E8DA497F7FF1F18
:1056300083C757AFDDCB17F7FF1F0347D7AE97F7E9
:10564000FF1F83C747AE22075D8F97F7FF1F83C7F2
:10565000A7ADC2075D8F97F7FF1F83C7F7ACE207BF
:10566000D98F17F7FF1F232DF7A883C7640097B5BD
:1056700001009385A57517B50100130565F617F7A9
:10568000FF1F230EF7A697900100E780E04797F7EA
:10569000FF1F9387E7A68C4317F6FF1F034626A636
:1056A00017B501001305C51C97900100E780C045A0
:1056B000294597900100E780004A97F7FF1FA383D1
:1056C00007A62244B24092440249930700F817F714
:1056D000FF1F2309F7A49D4517F5FF1F130585A498
:1056E0004101174300006700032297600000E78034
:1056F00020F297F7FF1F2388A7A29357850017F77B
:10570000FF1FA302F7A2935705012A8417F7FF1F73
:10571000230CF7A093578501014517F7FF1FA30539
:10572000F7A097600000E78060EF97F7FF1F238ED8
:10573000A79E97B501009385656917B5010013050C
:1057400025EA97900100E780203C17F6FF1F0346EB
:10575000C69DA28517B5010013050513B1B7CD4746
:105760006303F40297B501009385456617B5010000
:10577000130505E797900100E780003917B5010090
:105780001305051279BD37E404007C44414697F5C2
:10579000FF1F9385359917F5FF1F1305A59682976F
:1057A00097F7FF1F83C7279917F7FF1F034797989E
:1057B000A20703238405D98F17F7FF1F2310F7943F
:1057C0001306000A89452244B2409244024917E573
:1057D000FF1F03452508410102838D476303F4023F
:1057E00097B501009385855E17B50100130545DF68
:1057F00097900100E780403117B501001305051AA5
:105800000DB517F4FF1F0344049297F7FF1F83C7DA
:10581000779197B501009385655B220417B5010068
:10582000130505DC5D8C97900100E780E02DA285D3
:1058300017B501001305450897900100E780C02CBB
:10584000294597900100E78000310D4697F5FF1F2D
:105850009385458D228597E0FFFFE7808064AA84C9
:1058600021C197B501009385655617B50100130551
:1058700025D797900100E7802029A68517B501005C
:105880001305C50497900100E78000282244B24028
:105890009244024929454101179301006700A32B57
:1058A00097E7FF1F2390877EB7E70400116603A3E5
:1058B0008705130606E8914539B78D476303F4025F
:1058C00097B501009385855017B50100130545D1A3
:1058D00097900100E780402317B501001305C51A12
:1058E00089B317F4FF1F0344048497F7FF1F83C78E
:1058F000778397B501009385654D220417B50100A4
:10590000130505CE5D8C97900100E780E01FA2850E
:1059100017B501001305C5FC97900100E780C01E74
:10592000294597900100E78000230D4697E5FF1F6A
:105930009385457F228597E0FFFFE7808056AA8404
:105940001DC197B501009385654817B50100130582
:1059500025C997900100E780201BA68517B5010097
:10596000130545F905B797E7FF1F239F876EB7E734
:105970000400116603A38705130606E893050002D9
:1059800099B5894763E3870297B50100938505447C
:1059900017B501001305C5C497900100E780C01634
:1059A00017B5010013050511ADB997E4FF1F83C4B6
:1059B000847797E7FF1F83C7F77697B50100938534
:1059C000E540A20417B50100130585C1DD8C979051
:1059D0000100E7806013A68517B50100130505F3E4
:1059E00097900100E7804012294597900100E780D9
:1059F0008016228697E5FF1F9385C572268597E05E
:105A0000FFFFE780004A2A84630E051A97B501005C
:105A10009385C53B17B50100130585BC9790010020
:105A2000E780800EA28517B50100130565EF99BDCB
:105A3000854763F98718834519002244B240924490
:105A40000249B335B00097E7FF1F2387B76417B546
:105A50000100130525EE4101179301006700C30AF9
:105A6000A2852244B24092444A850249410117036B
:105A700000006700632499476303F40297B50100AF
:105A80009385C53417B50100130585B597900100BE
:105A9000E780800717B501001305851B59B617E489
:105AA000FF1F0344446897E7FF1F83C7B76797B595
:105AB00001009385A531220417B50100130545B2F5
:105AC0005D8C97900100E7802004A28517B5010046
:105AD0001305C5E797900100E780000329459790DB
:105AE0000100E7804007194697E5FF1F938585630E
:105AF000228597E0FFFFE780C03AAA841DC197B5D1
:105B000001009385A52C17B50100130565AD97908D
:105B10000100E78060FFA68517B50100130505E4C5
:105B200095B397E7FF1F2397875EB7E704001166D9
:105B300003A38705130606E89305000869B18547A6
:105B400097B501009385852817B50100130545A970
:105B5000630BF40097900100E78000FB17B501008C
:105B6000130505E17DBC97900100E780E0F917B5CA
:105B70000100130565E197900100E780E0F82945F1
:105B800097900100E78020FD2244B24092440249F0
:105B900097E7FF1F23940756410117630000670032
:105BA000A39797B501009385652217B501001305EA
:105BB00025A397900100E78020F517B50100130594
:105BC000650D85B4B240224492440249410182806D
:105BD000411106C622C497E0FFFFE780802C21CD4B
:105BE00097E7FF1F83D7674B85072A8417E7FF1FB7
:105BF0002315F74A97B501009385C51E97E7FF1F48
:105C0000239EA74817B501001305859D97900100B5
:105C1000E78080EFA28517B501001305653B9790DB
:105C20000100E78060EE2244B2402945410117930C
:105C30000100670043F297E7FF1F83D74746B24052
:105C40002244850717E7FF1F231BF7444101828089
:105C5000411122C491462A8417E6FF1F1306865A73
:105C60009D652D4506C697D0FF1FE78060B6B7F744
:105C7000070003C70701A5476313F70001A09306B8
:105C8000001001469D65254597D0FF1FE78040B471
:105C900097E7FF1F238887562244B240914617E6B4
:105CA000FF1F130626569D652945410117D3FF1F87
:105CB000670003B21171CED7B7E9040083A7C90406
:105CC000CAD917E9FF1F1309E945A2DD2E8686DF31
:105CD000A6DB2E84AA854A85829797E7FF1F83C794
:105CE00067441307700A6385E710636DF7001307B5
:105CF000600A6385E704FE506E54DE544E59BE5967
:105D0000116182801307800A6385E7161307900AE2
:105D1000E393E7FE8D476306F41C97B50100938576
:105D2000653E17B501001305A58B97900100E7802C
:105D3000A0DD17B501001305253A25A08D47630C9A
:105D4000F40297B501009385E53B17B501001305F3
:105D5000258997900100E78020DB17B50100130526
:105D6000E53097900100E78020DA294597900100FF
:105D7000E78060DE49B7854717B501001305C530D8
:105D800017E7FF1F230AF73097900100E780A0EF85
:105D9000B7750200B76602000146054597D0FF1FA0
:105DA000E78000A3930760F817E7FF1F230CF7367F
:105DB00097E7FF1FA38907369307002617E7FF1F02
:105DC0002324F736E5779387072117E7FF1F231F63
:105DD000F734B14597E7FF1F238B073497E7FF1F81
:105DE000A387A7344A8597000000E780E01621B713
:105DF000914763E3870297B501009385A53017A506
:105E000001001305E57D97900100E780E0CF17B50D
:105E1000010013056529B1B797E4FF1F83C4C4309F
:105E200097E7FF1F83C73730A204DD8C83A7C9041F
:105E30006D14228697E5FF1F9385152F2800829702
:105E40008E0493160401B7750200C1823000A69536
:105E5000094597D0FF1FE780A097930770F817E7D1
:105E6000FF1F2301F72C994597E7FF1FA38EA72A51
:105E700095BF914763E3870297B501009385852815
:105E800017A501001305C57597900100E780C0C7ED
:105E900017B501001305C522E9B597E4FF1F83C4B8
:105EA000A42897E7FF1F83C71728A204DD8C83A7C8
:105EB000C9046D14228697E5FF1F9385F5262800F7
:105EC00082978E0493160401B7750200C1823000D8
:105ED000A6950D4597D0FF1FE780808F930780F828
:105EE000BDBF17B501001305652097900100E7803D
:105EF00080D9930790F82304F100834719008D455A
:105F00002800A304F100834729002305F10097002E
:105F10000000E78060041305C01297C0FF1FE780F0
:105F20004042014597D0FFFFE78000160D459700DE
:105F30000000E78020D2294597C0FF1FE78060401E
:105F400097C0FF1FE780C0307DB397E7FF1F23A3F3
:105F5000A72C828097E7FF1F9387C72B03A3070017
:105F6000630303000283174300006700C3994111D4
:105F70004AC097F6FF1F83D6E67D328917D6FF1FEA
:105F80000356A64422C426C206C62A84AE849700BD
:105F90000000E780C05F35C12DC0994763FF9704BB
:105FA0008347140003470400A207D98F1397870083
:105FB000A183D98FC2073167C1831307C755639E79
:105FC000E70297D7FF1F83D74740A301F400A183BF
:105FD0002302F40097F7FF1F83D7C77791C7A30267
:105FE000F400A1832303F400A68517B5010013056F
:105FF000651597900100E78020B197F7FF1F83C7D1
:10600000E761B9CF97D5FF1F83D5253C17B50100B0
:106010001305051597900100E78000AF2686A2853D
:1060200017D5FF1F0355653A97000000E78080BA37
:106030006301090497E7FF1F83C7071E9DCB95C81F
:1060400097E7FF1F83C747058DE722852244B240AB
:106050000249A68592444101174300006700A38AC4
:1060600017B501001305C51097900100E780A0C186
:10607000C1B7B24022449244024941018280834721
:1060800055008345450017B501001305650AA207B1
:10609000DD8D17930100670023A717B501001305D5
:1060A000250817930100670003BE8D4763FBB70AFD
:1060B000011126CA06CE22CC0344350097E4FF1F07
:1060C00083C4941597B501009385450BB3378000C1
:1060D00017E7FF1FA302F71409C497B501009385C2
:1060E000A50A17B501001305A50A97900100E780DE
:1060F000A0A197E7FF1F83C7371263869700970019
:106100000000E780E02E97E7FF1F83C7F7108DC7D9
:1061100085472306F100B7E7040083A747177000FF
:10612000854513055030829717B5010013054507C3
:1061300097900100E78020B59967938757EE231663
:10614000F100680085479145A30781002307F1000E
:1061500097000000E78040E0F2406244D2440561CD
:1061600082808280894763F7B708011122CC06CE6E
:1061700026CA8344250085472A84639DF4049147F9
:1061800063F5B704034545008347340022055D8D60
:1061900097D7FF1F239BA72297000000E7800048A6
:1061A0009967938767EE2314F10083473400230532
:1061B0009100A305F100834744009545280023067C
:1061C000F10097000000E78020D9F2406244D244F9
:1061D00005618280FDF89967938767EE2314F100CB
:1061E00097D7FF1F83D7671EA305F1002305010082
:1061F000A183E1B782800111996722CCD51717F4EA
:10620000FF1F1304A4412314F1008347040026CA8E
:1062100097F4FF1F938404542305F10083D70400EF
:1062200028009545A305F100A18306CE2306F100C1
:1062300097000000E78040D203D6040083450400A5
:1062400017B50100130545F797900100E780C08B53
:10625000F2406244D244056182809D677971D9170A
:106260002316F10097F7FF1F83C7473B06D6230786
:10627000F100A9C3B7E70400FC47414697E5FF1FBB
:10628000938545E81305F10082976800CD45970096
:106290000000E78060CC97F5FF1F83C5253817B550
:1062A0000100130565F497900100E780E085B25086
:1062B00045618280B7E70400BC474146814513052C
:1062C000F1008297D9B745C5411106C622C493078C
:1062D00050FA2300F5009307A005A300F5008947B5
:1062E0002301F5009147A301F5009307D002A30213
:1062F000F50097F7FF1F9387673283C707002302D4
:1063000005002A842303F50097E7FF1F9387D7F042
:1063100083C70700414697E5FF1F9385A5DEA303CA
:10632000F50097F7FF1F83D7E7422304F500A18309
:10633000A304F50097D7FF1F83D727092305F5008E
:10634000A183A305F500B7E70400FC473105829758
:106350002285F14597000000E780601F230EA4000E
:106360002181A30EA400B240224441018280828098
:106370005D710A8586C6A2C497000000E780E0F43C
:1063800037E404007C448A850810794682973C44AF
:106390001305E10309468145829710109305000219
:1063A000014597D0FFFFE780C032B64026446161C7
:1063B0008280411122C426C24AC02A84AE84328916
:1063C000AA8585660146254506C697C0FF1FE7805A
:1063D0002040A2852244B240CA86268602499244C1
:1063E0002945410117C3FF1F6700833E0111B7C74D
:1063F000A55A22CC9387C73317E4FF1F1304D4E1B7
:106400003EC4834704002C002146196506CE3EC6D3
:1064100097000000E78020FA8345040017B50100CB
:10642000130545ED97800100E780006EF24062445D
:10643000056182800111A146300099652D4522CC6D
:1064400006CE97C0FF1FE780A038A24737C4A55AE1
:106450001304C43363958702B24517B501001305D1
:10646000A5DCB335B00097E7FF1FA387B7DA9780A5
:106470000100E7806069F2406244056182809165B5
:10648000A1463000938505F02D4597C0FF1FE7809A
:106490002034A247E38287FC854717E7FF1FA30D3F
:1064A000F7D6854517B50100130545DAC9B77971E7
:1064B000D146700091652D4522D406D697C0FF1FA6
:1064C000E7800031B24737C4A55A1304F435639806
:1064D0008702B7E70400FC4717E5FF1F130585C2D5
:1064E00041460C08829717B50100130525DC9780FB
:1064F0000100E7804079B250225445618280916565
:10650000D1467000938505E82D4597C0FF1FE780B1
:10651000202CB247E38F87FA17B50100130505DB7E
:10652000F9B74111856601469165254506C697C0B4
:10653000FF1FE780E029B24017B50100130505CD24
:1065400041011783010067000374C16769768146C2
:10655000FD1705061397060141836364B7003E8566
:1065600082803307D50003470700B98F214713F80E
:106570001700858363050800B18FC207C1837D17AB
:106580001377F70F6DF78506F1B741C5A5470547A6
:1065900063F2B70883471500034705003168A20777
:1065A000D98F13978700A183D98FC207C18313089E
:1065B000C855054763900707411106C622C426C285
:1065C00003442500914763F087049307540063EC6C
:1065D000F502A301C50021822302C5009304340003
:1065E00091C6A302D500A1822303D5002A84A685E3
:1065F00097000000E780A0F526942300A4002181E5
:10660000A300A4000147B240224492443A854101CC
:10661000828005473A8582800111B7C7A55A22CCEE
:106620009387E7342A842AC621462C00156506CEB6
:106630003EC497000000E78000D8A28517B501008E
:10664000130545CD97800100E780004C97000000BE
:10665000E78040D2F2406244056182800111A14688
:10666000300095652D4522CC06CE97C0FF1FE780F0
:106670002016A24737C4A55A1304E4346395870251
:10668000B24517B50100130565BE97D7FF1F239EBE
:10669000B7D2C205C18197800100E780E046F24091
:1066A0006244056182809165A1463000938505EEC4
:1066B0002D4597C0FF1FE780A011A247E38287FC0A
:1066C000D14717D7FF1F2312F7D0D14517B50100C7
:1066D0001305C5BBC9B797B701009387A7C713D7E1
:1066E000C5003E97034707001105230EE5FE13D7AB
:1066F00085003D8B3E9703470700A30EE5FE13D7A9
:1067000045003D8BBD893E97AE970347070083C781
:106710000700230FE5FEA30FF5FE82808145B30736
:10672000B5008387070089E717230000670003127D
:106730008505C205C181E5B7011122CC06CE26CA66
:106740004AC84EC693F715002E84638E0716AD67B0
:106750009387A7AA371700401CC397F7FF1F83C76B
:1067600047FC99EF97F7FF1F83C7E7FE850793F76D
:10677000F70F1D47636AF70217F7FF1F230DF7FC9A
:10678000B7E70400BC4F13060019854517D5FF1F56
:10679000034585C3829713451400F2406244D244F6
:1067A0004249B2490561828097F7FF1F238507FAA6
:1067B000B75720419304D0039387777497F5FF1F51
:1067C00083D545F917F5FF1F130515F613090002C8
:1067D00017F7FF1F2328F7F497F7FF1F238697F477
:1067E00097000000E78060EF2300250197F7FF1F67
:1067F00083C7C7E2B337F00093870703A301F5000F
:106800009309000593072004A30035012301950097
:1068100023022501A302F5002303950097D5FF1F4E
:1068200083D545B81D0597000000E78000EB2300E5
:106830002501A3003501930750042301F500A301AE
:10684000950097D5FF1F83D5A5A6110597000000D9
:10685000E780A0E89307B0042300250123019500F9
:10686000A300F50097E7FF1F83C7C789A20797E535
:10687000FF1F83C53589DD8D0D0597000000E7807A
:10688000C0E597E7FF1F83C70788A20797E5FF1FAB
:1068900083C57587DD8D97000000E78000E4B5476C
:1068A0002300F500A947A300F5009305250017F57F
:1068B000FF1F130525E7898DC205C18197200000C0
:1068C000E780E00175BD93F7250081CB97F7FF1FA7
:1068D000239807E413C52500C9B593F74500014582
:1068E000E38D07EA17B50100130585A49780010021
:1068F000E780603997300000E780802F134544001F
:1069000069BD411122C437E404005C5C06C635460B
:1069100097A501009385055617B5010013050524B9
:10692000829711E917B50100130545A19780010071
:10693000E780603501A08327041C82972A840545DF
:1069400097C00000E780A0E897600100E780C06D75
:1069500097600100E780C04297B00000E78020FA0E
:106960002285B2402244410182801567B71700405A
:106970001307575598C3D8439D66558FD8C3D8433E
:10698000FD76758FD8C3D8431367F70FD8C3356723
:106990001307C7CC98C382800111054506CE22CCCF
:1069A00026CA4AC84EC697C0FFFFE780C0571305E6
:1069B000A00497B0FF1FE780806F757585457D1532
:1069C00097C0FFFFE78060417D7585451305F5366B
:1069D00097C0FFFFE780C04A371400408327840A2E
:1069E0008D451305002093E707202324F40A97C060
:1069F000FFFFE780803E97D0FFFFE7804082B7E748
:106A00000400C85B97800100E780E02717B501000C
:106A10001305C51497800100E780E0268327840CC6
:106A20008545414593E707082324F40C97C0FFFFF1
:106A3000E78000458D451305000897C0FFFFE780FC
:106A4000204497C0FFFFE780007137A507001305BA
:106A5000051297C0FFFFE780A06C9D45014597C0D8
:106A6000FFFFE780A072B7E700E03707000423A02C
:106A7000E7180100010097D0FFFFE780E00397D0FF
:106A8000FFFFE780A01797000000E780C0E79700AE
:106A90000000E780609A9304C05D97000000E780E3
:106AA00020BC014997000000E78040279309700C43
:106AB000294497200000E780E0D17D1413054006AB
:106AC0001374F40F97C0FF1FE780C0867DF09720F6
:106AD0000000E780C0D619C505094209135909010C
:106AE00063E62901FD14C204C180F9F0970000009B
:106AF000E780E0E717B50100130505879700000060
:106B0000E78000C297E0FFFFE780A0ED17B5010026
:106B10001305C58697000000E78080C037E40400B5
:106B200097000000E780E00A8327040817050000AB
:106B30001305C5C0829797D7FF1F2387A7883C4CB2
:106B4000130600648545829797C0FF1FE780408A3F
:106B500001458280B7F7070003C70701A547AE8646
:106B60006316F7009397450191C301A0AA850146DA
:106B7000254517C3FF1F6700A3C54111B2862E86A6
:106B8000AA852D4506C697C0FF1FE78060C4B240A6
:106B90000145410182809307000463E8C7021D712B
:106BA000A2CC2A84080886CE32C697800100E780EE
:106BB00040EAB2461008A285294597C0FF1FE7802A
:106BC00020C1F6406644256182803955828041119A
:106BD0000D658D4506C697C0FFFFE7800020B717FB
:106BE00000408D6623A6D70A17F5FF1F1305C5B60B
:106BF0001387C70A9387870A1CC15CC585668967A6
:106C00005CC958C114C518C9B7E70400B24003A352
:106C1000871E410102838145B307B50083870700C2
:106C200089E717230000670063C28505C205C1819B
:106C3000E5B797B701009387E78D1357C5003E97D7
:106C400003470700011106CE2304E1001357850016
:106C50003D8B3E970347070023060100A304E10094
:106C6000135745003D8B3D893E97AA970347070080
:106C700083C7070028002305E100A305F100970062
:106C80000000E78080F9F24005618280411126C250
:106C9000E97797F4FF1F9384A4BC22C49387A75578
:106CA0002E842381B4002E86AA8517F5FF1F1305B5
:106CB00065BB06C62390F400A38104009780010001
:106CC000E78020D993052400C205C18117F5FF1F75
:106CD000130525B997000000E7806087B38784001B
:106CE0002382A7002181A382A70093056400224488
:106CF000B24026859244C205C1814101172300009C
:106D00006700C3B409C99307800263E6B70017039D
:106D100000006700E3F7828097F7FF1F83C727B75C
:106D200099EF411106C697200000E78020A9B240E4
:106D3000854717F7FF1F230CF7B44101828082803B
:106D40006301054A638F05485D71CAC04EDE86C681
:106D5000A2C4A6C252DC56DA5AD85ED662D466D233
:106D60006AD0B9472A89AE8963F9B706394697A52B
:106D700001009385E56797800100E78020CB31ED26
:106D80008347E900130710036394E702854717F769
:106D9000FF1F2305F7AC17A501001305656697F7DC
:106DA000FF1F239C07AA97000000E78000E771A05F
:106DB0001307000317A5010013058567E395E7FE98
:106DC00097F7FF1F238C07A897F7FF1F239707A8A4
:106DD00017A5010013054564F9B797F7FF1F83C78F
:106DE000E7A763870722BD6AB96B938CFA55014AFE
:106DF00017FBFF1F130B0B98138CEB65938AFA6636
:106E000005A8B307490183C6070097F7FF1F83D77B
:106E1000C7A4B1E39307A005639BF600854717F766
:106E2000FF1F231CF7A297F7FF1F2385D794050A9E
:106E300093170A01C183E3E637FDB6402644964422
:106E40000649F259625AD25A425BB25B225C925CAA
:106E5000025D61618280054D639BA7039307500A21
:106E6000639EF600894717F7FF1F2318F79E9307C5
:106E700050FA17F7FF1FA30FF78E55BF9307A00512
:106E8000E387F6FA97F7FF1F2399079C4DB71387FF
:106E900017004207DA9741832380D70017F6FF1FB8
:106EA000231DE69A8D47E3F4E7F817F4FF1F034428
:106EB000948C97F7FF1F83C7078C22045D8C930780
:106EC000F4FFC207C1839306F00DE3EDF6FA9307D2
:106ED0006400C207C183E31CF7F493052400C205D4
:106EE000C18117F5FF1F1305058997F0FFFFE780A4
:106EF000006633078B008347570003474700A2070C
:106F0000D98F17F7FF1F231A07946318F50E8144D2
:106F1000630CA40197F4FF1F83C40486A20497F7AF
:106F2000FF1F83C77785DD8C170500001305C5DDBE
:106F300097F0FFFFE780A00163878407636D9C02E1
:106F40009387EB556382F40497F7FF1F83C7C782CB
:106F500005476389E70681CB1387A7051377F70FEA
:106F60008D4663F2E6081307F0072300E100A30053
:106F7000F10089459DA063829405E39754FD97F045
:106F8000FFFFE780C02D11A8A28517E5FF1F13059D
:106F9000A57E97F0FFFFE7808011014597F0FFFF86
:106FA000E780E0FA69B5A28517E5FF1F1305C57CE8
:106FB00097F0FFFFE780401BCDB797F0FFFFE7801A
:106FC000C023E1BF930710F8130511002300F1005F
:106FD00097F0FFFFE780602FFD450A8597000000CE
:106FE000E78000CB5DBFA28517E5FF1F1305C578BD
:106FF00097F0FFFFE78040CC4DB79307F007894536
:107000000A852310F10097000000E78060C805B5ED
:10701000BD4763F83717414697A50100938585431F
:107020004A8597800100E78060A0631C051417A5BE
:1070300001001305654397000000E78000BE17E5D7
:10704000FF1F0355257197000000E780C0BE97E73A
:10705000FF1F83C7A75C17A501001305653889E7E3
:1070600017A501001305453897000000E780E0BA36
:1070700017A501001305C54097000000E780E0B99F
:1070800017C5FF1F0355053297000000E780A0BA1F
:1070900017A501001305053F97000000E780E0B742
:1070A00017C5FF1F0355653297000000E780A0B8A1
:1070B00017A501001305853D97000000E780E0B5A6
:1070C00017D5FF1F0355A5FD97000000E780A0B668
:1070D00017A501001305053C97000000E780E0B309
:1070E00017D5FF1F035565FB97000000E780A0B48C
:1070F00017A501001305853A97000000E780E0B16D
:1071000017D5FF1F035585F997000000E780A0B24F
:1071100017A501001305C53897000000E780E0AF10
:1071200017C5FF1F0355C51897000000E780A0B0E2
:1071300017A501001305453797000000E780E0AD73
:1071400097D7FF1F83C707FCA20717D5FF1F03456B
:1071500075FB5D8D97000000E780E0AD97D7FF1FBE
:1071600083C767FAA20717D5FF1F0345D5F95D8DC1
:1071700097000000E78020AC17A50100130505A7C4
:107180001DB1C147E3FB37CB414697A5010093856D
:10719000E5314A8597800100E7804089E31F05C8F3
:1071A0008347090113071003639CE700854717E72E
:1071B000FF1F230FF75A17A5010013056530E5B629
:1071C0001307000317A5010013058532E39DE7BCF3
:1071D00097E7FF1F238E075817A501001305C52F3A
:1071E000D9B68280411126C2AE848D4522C406C61E
:1071F0002A8497C0FFFFE780A0C8B717004099C84E
:1072000003A5C70C418D23A6A70CB240224492448B
:107210004101828003A5870C418D23A4A70CF5B7FB
:107220008347050003471500A207D98FC20761777E
:10723000C18713072720639AE70083452500370598
:10724000040017030000670023FA828017E6FF1F7F
:10725000130646648147B2861303F00FA94833082A
:10726000F6000348080013F7F70F6307A80C63063E
:1072700068008507E39517FF2947B387E600238059
:10728000A70097E7FF1F9387A7615DA8411113D758
:1072900065001347170006C693F63500058B954722
:1072A00091CA054699476387C60009469D4763838F
:1072B000C600A14713F645003336C00093F6850398
:1072C000050685C2A145638BB604E145638AB60411
:1072D000930580026388B604930580036393B60028
:1072E000914697F5FF1F2382F58297F5FF1F238DA7
:1072F000C58097F5FF1FA389D580BE8517A501001E
:107300001305452597800100E7800080B24085473E
:1073100017E7FF1FA30BF77E410182808546D1B797
:107320008946C1B78D4675BF17A501001305052510
:10733000177301006700437D17E7FF1F13074756C8
:10734000BA972380B700E147E302F5F49307700290
:10735000E30CF5FC82802A8723800500814717E52E
:10736000FF1F130525531308F00F2946B306F50038
:1073700083C606006396E60297E6FF1F9386465291
:10738000B69783C7070005452380F5009947636ECC
:10739000F7029D4763FDE700E147630DF700828038
:1073A000638506018507E393C7FC0145C5B72380C4
:1073B00005008280B737004003C7370083C7050048
:1073C00093F70704D98F2380F50082805D7152DC2A
:1073D00056DA5ED6716A97FBFF1F938B2B848D6AFA
:1073E000A6C24EDE62D486C6A2C4CAC05AD866D22D
:1073F0006AD06ECEC1495E8C97E4FF1F9384044B24
:10740000130A0A20938A7ADC17F9FF1F03490984BB
:10741000B3872B0183C7070093F7F70FC9EFB7872F
:10742000004003C76700058BE310077C03C76700B4
:10743000118BE30D077E83C75700918B99E36F1083
:10744000200317F7FF1F0347878085476304F70072
:107450006F10400197E7FF1FA389E76A97E7FF1FB7
:107460002386075097E7FF1F2384075C97E7FF1FDA
:107470002382076897E7FF1F238F076697E7FF1FA1
:10748000A386074E97E7FF1FA384075A97E7FF1FBE
:10749000A382076697E7FF1FA38F076497E7FF1F85
:1074A000A386076697E7FF1FA383077AB787004085
:1074B00011476F0070779307190093F7F70F3D4757
:1074C0006364F70617E7FF1F2302F77897E7FF1FAC
:1074D0009387C776CA9783C707001307100293F7ED
:1074E000F703638EE71E6366F70405446385871C14
:1074F000E38C07620947638EE71013070002E384F9
:10750000E74EB7E700E03707400023A0E718010087
:107510000100629923000900FD1923A0E71093F9E7
:10752000F90FE39309EEE5BD97E7FF1F238007728C
:1075300071BF130730026388E70C63E8E71613078F
:107540004002638CE70A13070003E39CE7FA97E71E
:10755000FF1F9387A76DCA9703C70700A14713773B
:10756000F70FE31BF71483C7640097E6FF1F23851B
:10757000F65897E7FF1F83C7D73391C7FD5797E6A4
:10758000FF1F238BF65697E5FF1F83C5353297E71C
:10759000FF1FA383B75697E7FF1F83C7273113FB4E
:1075A00007089306000493F70706639FD74C9307D9
:1075B000A009638DF51663EAB7129307F005638699
:1075C000F54A930750096384F52A014497E7FF1FA2
:1075D00083C797521547E392E736B7E700E03707CE
:1075E000400023A0E71801000100B7860040238077
:1075F0008602130680FC6F00500EFD5717E7FF1F31
:10760000230BF74EFDBDFD5717E7FF1F2304F74E71
:10761000CDBD17A501001305E50797700100E780B0
:10762000806697E7FF1F93876760CA9703C40700C8
:10763000014B97ECFF1F938CEC3F1374F40F17ADC5
:107640000100130DAD0563478B04294597700100B8
:10765000E7806050854717E7FF1FA30BF73C17E74C
:10766000FF1F2308873C17E7FF1F2301F74A37E76F
:1076700000E0B70640002320D7180100010037863C
:1076800000408347A60293F7370F2305F602232015
:10769000D71085BDB3876C0183C507006A85050BCC
:1076A00097700100E780404679BF854717E7FF1FC5
:1076B0002300F738B9B517E7FF1F130727574A9775
:1076C0000347070097E6FF1FA382F62A97E6FF1FEE
:1076D000238FE62817E7FF1F230AF7421DB58547CA
:1076E00017E7FF1F2304F72829BD9307400A638982
:1076F000F5349307200B6384F5369307100AE3965D
:10770000F5EC838724000144E3D207EC97E7FF1FE1
:1077100083C7F71993F63700638A061A0546638A0A
:10772000C62209466395C61A1D4755A217E5FF1FD5
:107730000345E517C94797ECFF1F83CC5C1797E516
:10774000FF1F83C5E51617E4FF1F03447416631576
:10775000F510CD476392FC1093077008639CF50207
:107760001307300FB7170E006308E4001307900DDE
:10777000B7B704006314E40817E7FF1F2324F738A2
:10778000BE8517A501001305E5F197700100E7809C
:10779000A03725BD93078008639DF500B30780409F
:1077A00013F4F70FB7774600938787CDB3D78702D7
:1077B000E1B793079008639AF500B307804013F48C
:1077C000F70F91679387C766D5B79307A008639BA8
:1077D000F500B307804013F4F70FB7173D00938708
:1077E0000790E9B79307B008639AF500B3078040A4
:1077F00013F4F70F9167938797D04DBF93F5F50773
:107800008D47639BF500B307804013F4F70FB797DC
:107810005B00938707D859BF8947639BF500B3077F
:10782000804013F4F70FB7770B009387071BBDBF9A
:107830008547639AF500B307804013F4F70FDD67BF
:10784000938767E3A5B7D28785F9B307804093F79D
:10785000F70FB3D7FA020DB797000000E780409FFB
:10786000A285668597000000E780809EB9BB9305DE
:10787000610017E5FF1F0345850317E4FF1F03445D
:10788000140397000000E78040AD93057100228546
:1078900097000000E78060AC3C0017E7FF1F232D36
:1078A000F736834761002304F10083477100A30486
:1078B000F100894717E7FF1F2300F7248357810052
:1078C00017E7FF1F2314F7FE094409B3154793F682
:1078D0004700B336D00093F78703850685C321465A
:1078E000638BC7066146638AC706130680026388F6
:1078F000C706130680036393C700914717E6FF1F6F
:107900002304D62097E6FF1FA380F62097E7FF1FEA
:10791000238DE71E17E7FF1F034787F993760704B8
:1079200097E7FF1F83C7D7F88DEE1377770C930681
:107930007008630CD7021377F7078D466312D70CD4
:10794000B307F040B7955B0093F7F70F938505D821
:1079500049A81947ADBF854755B7894745B78D47F2
:1079600071BF930670086311D7021307300FB71564
:107970000E006389E7021307900DB7B50400638317
:10798000E7021307700845BF9306800C6311D70206
:10799000B307F040B775460013F7F70F938785CD0F
:1079A000B3D5E70297E7FF1F23AEB714D9BB930601
:1079B000900C631CD700B307F04093F5F70F916765
:1079C0009387C766B3D5B702F1BF9306A00C631DBA
:1079D000D700B307F040B7153D0093F7F70F938535
:1079E0000590B3D5F5027DBF9306B00CE315D7F42F
:1079F000B307F04093F5F70F9167938797D0D9B706
:107A00008946631BD700B307F040B7750B0093F7A7
:107A1000F70F9385051BF1B78546631AD700B307A7
:107A2000F040DD6593F7F70F938565E35DBFD28581
:107A300035FBB305F04093F5F50FB3D5BA029DB70A
:107A400083C72400C18B99C7854717E7FF1F230809
:107A5000F70AA5BE97E7FF1F2383070ABDB6854730
:107A600017E7FF1FA303F70A8DB63C0017E7FF1FB8
:107A70002324F71A0947930700032314F10097E61C
:107A8000FF1F238BE6062DBD63940756A94763E5C8
:107A9000B74217A70100130727A98A05BA959C4189
:107AA000BA97828717E4FF1F034474E0894C63068A
:107AB000940D63E68C0685476303F4089307F00F83
:107AC00017E7FF1F0347470363F6E70017E7FF1FAA
:107AD0002304F70297ECFF1F83CC0C0293070004EA
:107AE00013F4FC0F63F497011304000497E7FF1FDE
:107AF0009387871203AD070022862685EA85B38C1B
:107B00008C40229D97700100E780A0F497E7FF1F4B
:107B1000238497FF97E7FF1F23A0A71145BC8D473C
:107B2000630CF40A9947E31BF4F897A701009387C5
:107B300027A617E7FF1F2321F70EA94751B717E71D
:107B4000FF1F0347C71097E7FF1F9387E7FC4946CE
:107B500097A501009385C5AC6306870097A5010032
:107B6000938505A83E8597700100E78080EE17E7B2
:107B7000FF1F2323A70AC947A1B797E6FF1F83C6A4
:107B8000060D054797E7FF1F938707F96394E60201
:107B90003E851306700297A501009385E5A59770B1
:107BA0000100E78000EB17E7FF1F2327A7069307D5
:107BB000700239B73E851306300497A501009385FE
:107BC000E59D97700100E780C0E817E7FF1F2325B8
:107BD000A70493073004EDB597E5FF1F83C525CDB6
:107BE00017A50100130545AD97700100E780C0F1AE
:107BF000054D97EDFF1F83CD8D0597E5FF1F83C5CD
:107C000005CB17A50100130525AB6398AD0B977045
:107C10000100E78060EF97E7FF1F83C747C9B5CB37
:107C2000E36EF4E817A401001304C4A3638CB70146
:107C300017A40100130484A36386970117A401000D
:107C4000130444A4228597700100E780800C13750B
:107C5000F50F93071500860717E7FF1F230EF7EAB6
:107C60008D4717E7FF1FA309F7EA97E7FF1F9387E1
:107C7000A7EA0147BE861376F70F89076365A60258
:107C800097E7FF1F23AAD7F897E7FF1F83C7C7E827
:107C900005BD97A701009387E79517E7FF1F232DE1
:107CA000F7F6914731BD3306E40003460600A38092
:107CB000070005072380C7007DBF97700100E7809C
:107CC000A0E497E7FF1F83C787BEE1D7E368F4DE30
:107CD00017A4010013040496638CA70117A40100E4
:107CE0001304C4956386970117A4010013048496B6
:107CF000228597700100E780C0011375F50F930787
:107D00001500860717E7FF1F2308F7E08D4717E7E1
:107D1000FF1FA303F7E097E7FF1F9387E7DF014704
:107D2000BE861376F70F8907E37CA6F43306E400DA
:107D300003460600A380070005072380C700D5B7C8
:107D400097E5FF1F83C5A5B617A501001305859705
:107D500097700100E78040DB97E7FF1F83C797DB41
:107D600093E7470017E7FF1FA306F7DA83C724004E
:107D700017E7FF1FA30EF7D889B817A50100130551
:107D8000A59597700100E78000F097E7FF1F9387A4
:107D900027D883C7070017E7FF1F2309F7B017E4A9
:107DA000FF1F034464D5333480000DB017A50100D4
:107DB0001305C59397700100E780E0EC97E7FF1F7C
:107DC00083C757D593E7070117E7FF1FA304F7D42D
:107DD00083C7240017E7FF1F230CF7D26FF0EFFED5
:107DE00017A501001305C59197700100E780A0E970
:107DF00003C704007D8B51EFB787004003C76702BC
:107E00001377C70B136727002383E70203C7A70273
:107E10001377C70B136727002385E70203C7E70221
:107E20001377C70B136727002387E70203C72703CE
:107E30001377C70B136727002389E702854717E7E6
:107E4000FF1F2305F7B217E7FF1F2303F7BE17E74E
:107E5000FF1F2301F7CA17E7FF1F230EF7C897E795
:107E6000FF1FA38507B097E7FF1FA38307BC97E712
:107E7000FF1FA38107C897E7FF1FA38E07C697E7D9
:107E8000FF1FA38507C897E7FF1FA38207DC6FF0DA
:107E9000CFF389476312F70297E7FF1F83C747A114
:107EA0009146638CD70863E0F604638EE70C636940
:107EB000F70A05476380E70EFD5717E7FF1FA30D7D
:107EC000F7C237074000B7E700E023A0E71801003A
:107ED0000100B78600401306F0FC2381C60223A0F0
:107EE000E7106FF00FE2130720086382E708636270
:107EF000F70213071008E391E7FC37870040834738
:107F0000670293F7C70B93E727002303F7026FF08D
:107F1000CFEB130730086389E70213074008E39D9E
:107F2000E7F8378700408347270393F7C70B93E7AA
:107F300027002309F7026FF04FE937870040834796
:107F4000270393F73707F5B7378700408347E702E2
:107F500093F7C70B93E727002307F7026FF0EFE6CD
:107F6000378700408347E70293F73707F5B737872E
:107F700000408347A70293F7C70B93E72700230529
:107F8000F7026FF08FE4378700408347A70293F72B
:107F90003707F5B7378700408347670293F73707FE
:107FA000ADB7179501001305A57697700100E7801E
:107FB00080CD97E7FF1F238B078ED5B31795010060
:107FC0001305057697700100E780E0CB97E7FF1F68
:107FD000239E078C97E7FF1F938707B203C4070010
:107FE000894763F3870009441374F40F6FF00FDEC1
:107FF00013070002E392E7EC631B0B0A638FF500A3
:10800000930720026383F508179501001305C574D3
:1080100097700100E78040AF45B517950100130543
:10802000E57097700100E78000C60144179D0100CC
:10803000130D0D71A14CB387840083C507006A85B9
:10804000050497700100E78020ACE31694FF1795B4
:1080500001001305A5BF97700100E780C0C217E4B7
:10806000FF1F0344E48401E897E7FF1F2382078290
:10807000014B6FF0AFD58947E310F4E4854717E76C
:10808000FF1F2307F7806FF04FD417E6FF1F03464B
:10809000168297E5FF1F83C585811795010013059B
:1080A000A56A97700100E78020A66FF00FD2638069
:1080B000F50693071002E399F5F497D5FF1F83C5E2
:1080C000257F179501001305256A97700100E78049
:1080D000A0A397E7FF1F23A197B497E7FF1F9387FC
:1080E00067A2944383D7470017E7FF1F0347E7A121
:1080F00017D6FF1F232CD67A1D4497D6FF1F23992E
:10810000F67A97D7FF1F2386E77A6FF02FCC97D5A3
:10811000FF1F83C5E5791795010013056566977004
:108120000100E780609E97D7FF1F2383077697D7CC
:10813000FF1F239D07766FF02FF92547638FE7C850
:108140009946378700406394D70223008702B7E738
:1081500000E0B706400023A0D71801000100130675
:1081600000FC2301C70223A0D7106FF08FB993063C
:10817000100A639FD70023008702B7E700E0B70625
:10818000400023A0D71801000100130680FCD1BFD6
:108190009306A009E381D7FE9306400AE38DD7FC3E
:1081A00093062002639DD700B7E700E0B7064000C2
:1081B00023A0D7180100010023008702F9B78546E4
:1081C000E384D7FE93070008E300FBFEB7E700E077
:1081D000B706400023A0D71801000100130620FCB9
:1081E00023008702BDBF17E7FF1F0347F790630215
:1081F000F71E63E7E70295476300F7109947630AA4
:10820000F704B786004023800602B7E700E037078F
:10821000400023A0E718010001001306A0FC75B977
:108220009307F005630AF700930750096306F70008
:1082300093071002E317F7FCB7E700E037074000A9
:1082400023A0E71801000100B7860040130620FCB8
:1082500069B117EBFF1F034B2B8A930700045A8D5C
:1082600063F46701130D000497E7FF1F9387C79A14
:1082700083AC07001374FD0F2286E6852685976080
:108280000100E780007DB3078B40669417E7FF1F6E
:108290002304F78697E7FF1F23A08798B78700403E
:1082A000630C0B022380A703B7E600E0370640000B
:1082B00023A0C6180100010003C7270213470704C3
:1082C0002381E70203C727021377C70F2381E70241
:1082D00023A0C6106FF0EFA22380070237E700E06B
:1082E000B70640002320D71801000100130620FC28
:1082F0002381C7026FF0AFB937870040834737004B
:1083000097E6FF1F83C6D68093F70708D58FA30192
:10831000F700B7064000B7E700E023A0D718010038
:1083200001001306A0FC35BD97E7FF1F9387079058
:10833000CA9783C7070093F7F70FC1CF97E7FF1FCF
:1083400083C7E790D9E717D7FF1F0347F77A93074B
:1083500000026310F70883AD040017DDFF1F034D13
:108360002D5597DCFF1F83CCBC5417DBFF1F034B3D
:108370004B54E6876A87DA866E8697D5FF1F83C5DA
:108380002551179501001305254197600100E780ED
:10839000A07797D7FF1F23A7B77797D7FF1F23850E
:1083A000A77797D7FF1FA381977797D7FF1F238EB4
:1083B000677597D7FF1FA38C874CB7E700E0370797
:1083C000400023A0E71801000100B78600406FF0CD
:1083D0004FA2B7E700E03707400023A0E7180100ED
:1083E0000100B786004015BD97E6FF1F83C62686AD
:1083F0000547639CE60429472381E7020947238355
:10840000E7022385E70297D7FF1FA381077097E74D
:10841000FF1FA38E0782B7870040A381070017D7ED
:10842000FF1FA307076E05472383E700B6402644D6
:1084300096440649F259625AD25A425BB25B225CB8
:10844000925C025DF24D6161828029472381E702DF
:1084500009472383E7022385E7022387E70223896D
:10846000E70255B717D7FF1FA303F7426FE01FFFBF
:10847000854717D7FF1F230BF74E17D7FF1F230979
:10848000F75A17D7FF1F2307F76617D7FF1F2304D5
:10849000F7666FE0BFFE854717D7FF1F2308F74C2D
:1084A00017D7FF1F2306F75817D7FF1F2304F764BA
:1084B00017D7FF1F2301F76417D7FF1FA308074A29
:1084C00017D7FF1FA306075617D7FF1FA30407627E
:1084D00097D7FF1FA38107628280411106C69700CC
:1084E0000000E78080FBB787004023800700130768
:1084F00040FC2386E7001307C004A386E70017D7D4
:10850000FF1F1307A73A2398E70017D7FF1F13078A
:10851000E73D239AE70017D7FF1F13076749239CFE
:10852000E70017D7FF1F1307E754239EE7002947EB
:108530002381E70209472383E7022385E702238794
:10854000E7022389E702A3810700930600F8A380CE
:10855000D700930690022380D700FD562383D700CF
:108560002381E7009306000537E700E0230BD7409F
:10857000B70640002320D71003C717001367170062
:10858000A380E700B24097D7FF1F2393075841010C
:108590008280411106C697000000E78000F0B7878F
:1085A000004023800700130700FC2386E7003147C3
:1085B000A386E70017D7FF1F1307472F2398E7006D
:1085C00017D7FF1F13078732239AE70017D7FF1F1C
:1085D0001307073E239CE70029472381E702094749
:1085E0002383E7022385E702A3810700930600F8AF
:1085F000A380D700930690022380D700FD562383E3
:10860000D7002381E7009306000537E700E0230B3E
:10861000D740B70640002320D71003C717001367C1
:108620001700A380E700B24097D7FF1F2392074EA1
:1086300041018280F1679387072017D7FF1F23230B
:10864000F74C854717D7FF1F2310F74CA14717D7C3
:10865000FF1F230CF74A97D7FF1FA388074A97D716
:10866000FF1F2385074A97D7FF1F2383072297D72A
:10867000FF1FA38E0720814717D5FF1F13058521F4
:10868000FD5517D6FF1F1306A6212947B306F5008F
:108690002380B600B306F600238006008507E39723
:1086A000E7FE97D7FF1FA38A074497D7FF1FA3882A
:1086B000074497D7FF1F2383074497D7FF1F238EB5
:1086C000074297D7FF1F238D074297D7FF1FA38726
:1086D000074297D7FF1F23840742814717D6FF1F02
:1086E0001306C6534147B306F600238006008507EC
:1086F000E39BE7FE828017D7FF1F03474755854757
:108700006316F700170300006700E3E81703000093
:108710006700E3DC411122C406C617D7FF1F0347D9
:10872000075385472E8613F4F50FAA856317F704C0
:1087300017D5FF1F1305C52B97600100E780603137
:1087400097D7FF1F2386072EB78700402384870211
:10875000B7E600E03706400023A0C618010001007C
:1087600003C7A7021377C70F2385E702B24022444D
:1087700023A0C61001454101828017D5FF1F1305B4
:10878000E51A97600100E780C02C97D7FF1F238F61
:10879000071CB787004023828702B7E600E0370650
:1087A000400023A0C6180100010003C76702137729
:1087B000C70F2383E7025DBF411106C69700000083
:1087C000E78080E7B2404101170300006700E3F251
:1087D000411106C697F0FFFFE78080BF97D7FF1FC4
:1087E00083C7D718A1CB97D5FF1F83C5451889C963
:1087F00017D5FF1F1305C51797E0FFFFE7808054CB
:1088000097D7FF1FA384071697D7FF1F2380073032
:1088100037E700E0B70640002320D7180100010029
:10882000378600408347660293F7370F2303F6022B
:108830002320D710B2404101828017D5FF1F034586
:10884000252D3335A000828041C9D9C597D7FF1F98
:1088500083C7072CD1C3011122CC4AC84EC656C2C9
:108860005AC006CE26CA52C42E89AA890144930A48
:108870000004371B030063772403B3078940C20752
:10888000C183BE8463F4FA0093040004C204C1806F
:10889000130A1BD497D7FF1F83C7470D9DE37D1A8B
:1088A000631C0A00F2406244D2444249B249224A5F
:1088B000924A024B0561828097F0FFFFE78040B14A
:1088C000D1BF338589002694A68542049700000015
:1088D000E78080E4418045B78280411106C622C40A
:1088E00029C12E8495C997D7FF1F83C7672295CBCF
:1088F00097D7FF1F83C787078DC713070004AE876D
:108900006374B70093070004139407014180A285A4
:1089100097000000E78040E02285B24022444101F8
:1089200082800144D5BF97D7FF1F9387E735184250
:108930009C4383D645000345070083C5C700035603
:1089400046006396A50083D5E700638DD50201112B
:1089500006CE2386A7002397D700B705CF00DC4BB0
:108960009385757D05077D162EC2230001003AC44C
:108970002316C1002317D10099C30A858297F240BC
:10898000056182808280DC4DDC4B81CFB7E704003B
:10899000904503A38705914517D5FF1F0345052F74
:1089A000028382806D713C083EC6B707E500232232
:1089B00091103EC8AA843C083285232611103ECA75
:1089C00023248110232021112E8997300000E78075
:1089D000005E2A8497950100938585DF1785010045
:1089E000130505C097600100E7800012A285179566
:1089F0000100130565EE97600100E780E01029454E
:108A000097600100E7802015B705CB009385757D41
:108A1000680097100000E7802067A2856800973003
:108A20000000E780204B014781467000CA852685FB
:108A300097200000E780A08A05CD2A849795010041
:108A4000938505D917850100130585B99760010045
:108A5000E780800BA285179501001305A5E89760B4
:108A60000100E780600A294597600100E780A00EB9
:108A70008320C11003248110832441100329011095
:108A80005161828097D7FF1F9387072018429C432C
:108A9000797122D406D60348070083C807012A84C7
:108AA00083D64500035546006396080183D8270105
:108AB000638DD8022388070105072399D70037085B
:108AC000CC00DC4B1308787D3ACC1307F5FF42CA83
:108AD00023080100231EE100231FD10099C70808C5
:108AE00032C62EC482973246A245228597000000E6
:108AF000E78080EBB2502254456182806D713C0862
:108B00003EC0B707E5003EC23C083EC42326111014
:108B10002324811023229110231701002318010020
:108B200023190100231A0100231B010097B7FF1F1F
:108B300083D7078C99E3C167FD172316F10097B718
:108B4000FF1F83D7078B91EB97D7FF1F9387C7131F
:108B50009C439C43DC4783D7070017B4FF1F1304D3
:108B60002489584C2317F10083574400484B23189D
:108B7000F10031E197950100938585CC17850100BF
:108B8000130505A697600100E78000F8179501001E
:108B9000130545CC97600100E78000F729459760F1
:108BA0000100E78040FB8320C1100324811083244F
:108BB00041105161828097B7FF1F83C7D78389EB2C
:108BC000B7E70400BC5782975C4C23AA0700E1BFBB
:108BD000FD1797B6FF1FA380F68203560701834750
:108BE00004014C470A85230BF10097300000E78011
:108BF000802B97D7FF1F938727099C430147814606
:108C000088430A866C0097100000E780406DAA84B4
:108C100029C1979501009385A5C217850100130509
:108C2000259C97600100E78020EEA685179501003E
:108C3000130505C397600100E78000ED29459760A3
:108C40000100E78040F1584CB7E70400BC57484B9F
:108C50009DBF97A7FF1F83C7177AF5D7B7E7040013
:108C6000BC4F1044854517D5FF1F03452502829749
:108C70001DBF5C4EDC4BB9CFB1CD411122C417856D
:108C800001001305E5952E8497950100938585B91C
:108C900006C697600100E78020E7A28517950100CE
:108CA0001305C5BE97600100E78000E6294597607F
:108CB0000100E78040EAB7E704002244B24003A382
:108CC000870517D5FF1F034565FC13064006914530
:108CD000410102838280411122C417A4FF1F1304A3
:108CE000E46E1C4C06C689C7DC4399C34C48829786
:108CF000584CB7E70400BC57484B82975C4CB240D5
:108D0000224423AA07004101828017A7FF1F1307EF
:108D1000E76D834707009306F00B850793F7F70F7E
:108D200063E9F60097A6FF1F2382F66C0345070050
:108D30008280930700F8FDB78357450063860710CC
:108D400001114AC817A9FF1F1309896A52C4032ACF
:108D5000C90106CE22CC03274A0126CA4EC656C2F6
:108D6000F15735E31307D00DFD57636EC704B7E91C
:108D7000040083A709072A84130586004205418160
:108D8000B284AE8A8297232AAA000325C9015C49CE
:108D9000A9E7979501009385E5A6178501001305BE
:108DA000258497600100E78020D617950100130500
:108DB00025B697600100E78020D52945976001001E
:108DC000E78060D9DD57F2406244D2444249B2495B
:108DD000224A924A3E850561828093874400B70506
:108DE000CF002319F5009385757D3105971000009C
:108DF000E78080290325C901834564003105973048
:108E00000000E780200D0325C9012686D68531059F
:108E100097300000E78020097146A2854A85976057
:108E20000100E78000C3504419CA83A7890585451E
:108E300017D5FF1F034585E58297814769B79700DE
:108E40000000E780E0CBD5BFFD573E858280411111
:108E500026C297A4FF1F9384A459D84C22C437E498
:108E600004003C54484B06C68297DC4C0323C405DF
:108E70002244B240924423AA070017D5FF1F03459E
:108E8000E5E0854541010283411126C297D4FF1FC9
:108E9000938484DF9C4006C622C44AC0D5C3DC4309
:108EA000C5C35CC12300B5002A8497950100938552
:108EB000A590177501001305A57297600100E78062
:108EC000A0C4294597600100E780E0C89C4023A426
:108ED000070023A2070097A7FF1F9387274FDC4FA8
:108EE000DC4B91C7295597000000E78000DF97A76A
:108EF000FF1F9387E74FDC4FDC4B89C797000000CB
:108F0000E78020F537E904008327C905894517D58F
:108F1000FF1F0345A5D782978327C905914517D51C
:108F2000FF1F0345A5D682979C4003A34701630911
:108F3000030022852244B240924402494101028347
:108F4000B24022449244024941018280011132859B
:108F500006CE22CC26CA2E8497300000E78020055A
:108F6000AA849795010093856588177501001305FC
:108F7000256797600100E78020B903078400035646
:108F8000640083554400A6861795010013050592D9
:108F900097600100E78040B7294597600100E780AE
:108FA00080BB97A7FF1F83C7C742639D97000145FA
:108FB00097000000E78060D281450A859700000095
:108FC000E780C0ECF2406244D244056182806D715A
:108FD00023248110232611102322911093F745009A
:108FE0002E84638707143C083EC0B707E5003EC2E5
:108FF0003C083EC423170100231801002319010077
:10900000231A0100231B010097A7FF1F83D7073CEA
:1090100099E3C167FD172316F10097A7FF1F83D7B8
:10902000073B91EB97D7FF1F938707C69C439C4351
:10903000DC4783D7070017A7FF1F1307273923171C
:10904000F100544F835747002318F100DC4AA1E791
:10905000978501009385C57D177501001305455857
:1090600097600100E78040AA178501001305857EFF
:1090700097600100E78040A9294597600100E780DB
:1090800080AD134544008320C11003248110832444
:1090900041105161828097A7FF1F83C797332555E1
:1090A000D9C3FD1717A6FF1FA305F63203D6060185
:1090B00083470701CC460A85230BF1009730000057
:1090C000E78060DE97D7FF1F938707BC9C4317A7F5
:1090D000FF1F1307A72F978601009386A67A884360
:1090E0000A866C0097100000E780601FAA8451D99F
:1090F000978501009385C573177501001305454ECB
:1091000097600100E78040A0A68517850100130540
:10911000257597600100E780209F29459760010031
:10912000E78060A3268597000000E78000BB91BF21
:1091300093F725009DC7B7E70400BC47414681452A
:1091400028088297255597000000E78000B9280875
:109150009305F00F97000000E78040D313452400EB
:109160001DB793F71500014599DF97000000E780D0
:1091700020991345140001BF5C4D411106C688C3F8
:1091800017D7FF1F2322F7B0B7E7040083A707080C
:10919000170500001305E5E38297B24097D7FF1F3C
:1091A0002386A7AE01454101828001113335A0001D
:1091B000A307A100B7E7040083A7471706CE13064D
:1091C000F1008545130550308297F2400561828099
:1091D0008280411122C406C697D7FF1F83C787AC80
:1091E000014489EF97B7FF1F83C71703054499E729
:1091F00017C4FF1F034484421344140022859700C0
:109200000000E780C0FA178501001305257C09E4FA
:10921000178501001305857C2244B2404101176384
:1092200001006700638E797122D4A30F010037E437
:1092300004008327841726D24AD006D6AA842E8912
:10924000130550309305F10132C6829732468347A9
:10925000F10193150601C18185CB01452EC697000A
:109260000000E780C0F483274417B2454A8626856C
:109270008297054597000000E78060F3B2502254C2
:109280009254025945618280832744174A86268575
:109290008297EDB741119397050122C406C626C2F5
:1092A000C1872E8463D40702B7E40400FC5417A5D9
:1092B000FF1F0345E516829719C1BC5482972165AB
:1092C000218DB240224492444101828093F71500DF
:1092D0008DC7B7E7040083A7471A17A6FF1F130619
:1092E000261397D5FF1F9385259B17A5FF1F0345C1
:1092F0002513829713451400E9B793F7250099CFFA
:10930000B7E70400BC4F13060064894517A5FF1F8B
:109310000345051182971345240065B793F785002F
:1093200085CF97D7FF1F83C7A79885E7B7E70400C6
:1093300003A8871A1307401F97A7FF1F83C7470E6D
:10934000814613064006994517D5FF1F0355C5955D
:10935000029813458400B5B793F745000145B5D38E
:10936000B7E4040083A7041817D5FF1F0355C5935E
:109370008297BC4C13060064914517A5FF1F034557
:10938000250A8297134544002DBF97D7FF1F83D727
:10939000A7916398A70217D7FF1F2318B79017D775
:1093A000FF1F2315C79017D7FF1F2312D7902E86B4
:1093B000178501001305C567BE85175301006700B7
:1093C000A374178501001305256817630100670062
:1093D000838B0357450097D7FF1F83D7E78C631E06
:1093E000F704C1674111F91722C417D7FF1F232DB6
:1093F000F78A37E4040097D7FF1F23A9078A97D776
:10940000FF1FA381078A97D7FF1F2383078A7C4CFE
:1094100006C6894517A5FF1F0345850082977C4C2A
:10942000914517A5FF1F0345A5FF82972244B2402F
:10943000410117030000670003DA178501001305D7
:10944000A56017630100670003847D15954763E2FB
:10945000A71C17870100130727550A053A951C41D9
:10946000011122CC06CEBA972E848287178501007F
:109470001305055E97600100E780E080A1A203C7A5
:10948000250099476311F7022E8597000000E780B9
:1094900080F483456400178501001305655C9750CF
:1094A0000100E780606697B7FF1F238707D61785FF
:1094B00001001305A55C7DBF03C72500954763190F
:1094C000F702C16717C7FF1F0357077EF91703D5B8
:1094D000A5006309F702B7E7040083A7C7178297BF
:1094E000178501001305855A97500100E780A07980
:1094F000854717B7FF1F2301F7D217850100130512
:10950000655B8DBF97C7FF1F2390A77A83D7E500C0
:1095100097C6FF1F239BF67883D7050197C6FF1FC9
:109520002396F67883D7250197C6FF1F2391F678F7
:1095300097C7FF1FA3880776631BE502B7E7040000
:10954000BC4F096613060690A14517A5FF1F0345EA
:1095500025ED82970356E4008355A400178501008A
:109560001305055497500100E780005A51B793073F
:10957000700F2316F100B7E7040083A7870D17A625
:10958000FF1F0346E6E96C0082974DF9854717C730
:10959000FF1FA309F7705DB717850100130545523A
:1095A000D1BD83C5250091476392F502178501005F
:1095B0001305855297500100E780E06C970000008A
:1095C000E78060C1F24062440561828099476392FE
:1095D000F502228597000000E780E0DF8345640004
:1095E000178501001305C54797500100E780C0515A
:1095F000D1BF9547639AF50083471400E1F31785BF
:1096000001001305A54FBDB5178501001305854F52
:10961000E1BF8280411122C417A4FF1F130484E11B
:10962000AA86178601001306A6392285C14506C6FB
:1096300097500100E78060660357440097A7FF1F1B
:10964000938747E02393E700035764002394E700E0
:10965000B240224441018280411106C697000000B9
:10966000E78080FBB7E7040083A7871417A6FF1FD6
:10967000130646DCD54501458297B2404D4697A575
:10968000FF1F938525DC130570304101170300008F
:109690006700A3B961712324811A37E4040083278A
:1096A00004082326111A2322911A2320211B232E7A
:1096B000311917050000130525BE829717A9FF1F52
:1096C000130909D6994785442300A900231CF100FA
:1096D000978501009385C5329307400617750100F1
:1096E000130505F0231CF1082308910097C9FF1FFB
:1096F0009389490697500100E780004183D509000E
:10970000178501001305C52E97500100E780C03F63
:10971000294597500100E780004403D50900896975
:1097200097000000E78040EF832744171008854525
:109730001305503082978327441717A6FF1F13067F
:1097400066D0CD451305703082978327441717A63E
:10975000FF1F130626CDB54513056030829783277A
:109760004417300889451305103182978327441721
:109770003009894513052031829783274415938545
:1097800009900D45829783274415938509901145CB
:109790008297A3059100230691002308910002CD32
:1097A000230C01008327841630099145130570406E
:1097B0008297832784161306B10085451305004060
:1097C0008297832784167000854513051040829781
:1097D0008327841630088545130520408297832708
:1097E0008416100885451305504082978327041579
:1097F0007D558297832744137D5582977D5597A089
:10980000FFFFE780E0E58327440C829797A0FFFFE6
:10981000E78040C18327841417A6FF1F130686C163
:10982000D5450145829789471306700F8145280960
:109830002306F1009790FFFFE780608C8D471306A9
:10984000000881452808230CF1089790FFFFE78066
:10985000008B9147230CF100977701009387C7C9CC
:10986000984383C747003AC8230AF10097D0FFFF07
:10987000E78040B070008545054597A0FFFFE78071
:1098800040E530099305700F094597A0FFFFE78079
:1098900040E43008930500080D4597A0FFFFE780DE
:1098A00040E310089545114597A0FFFFE78060E26F
:1098B000C16717C7FF1F1307273FF9171CC32322D0
:1098C000070017A5FF1F130565B597A0FFFFE780E9
:1098D00020DF8327C41D17C5FF1F1305653B829733
:1098E0003C4803450900854582978320C11A03241B
:1098F000811A8324411A0329011A8329C1195D6140
:109900008280C16717C8FF1F0358083AF91763011F
:10991000F8083DCDB5CD011126CAB7E4040083A7F0
:10992000841222CC2E862315B10006CE2A8401474C
:109930008146ED45428582972AC611ED17850100C3
:109940001305050D97500100E780E033F2406244B3
:10995000D24405618280FC440356A100A28582970F
:109960002C0017C5FF1F0355253497A0FFFFE78084
:10997000E0E169DD178501001305C50A9750010074
:10998000E780603083A7C412ED45280082977DBF31
:109990008280411106C61DC9854717A7FF1FA3086E
:1099A000F7A8354697A5FF1F9385C5A71305603017
:1099B00097A7FF1F238E07A697000000E780E08689
:1099C000B2404101170300006700E38097A7FF1F23
:1099D000A38F07A4F9B797C7FF1F83C7672DA9EF08
:1099E000C16717C7FF1F0357272CF9176306F70432
:1099F0004111854722C417C7FF1F230BF72A37E4FD
:109A000004007C4C06C6A14517A5FF1F034545A1D0
:109A100082970323841A2244B24097A7FF1F83C76B
:109A200027A017C5FF1F035525281307401F814690
:109A3000314699454101028382806D712324811052
:109A40002326111023229110328401CD8947630A05
:109A5000F5028320C1100324811083244110516139
:109A60008280178501001305A50AAE849750010076
:109A7000E7806021A285268597C0FFFFE780C0AF01
:109A8000C9BFB7E70400FC4728008297178501008B
:109A90001305C50897500100E780E01E8347810049
:109AA00039C41307000B6380E7021387A7051377F8
:109AB000F70F8D4663EDE602A285280097C0FFFFF1
:109AC000E780801F79B78547E3F587F883459100E4
:109AD00017750100130505E6B335B00097A7FF1F02
:109AE000238CB75A97500100E78000029DB70347C7
:109AF0009100A207D98F35671307D7556385E7080B
:109B00006368F7022D671307B7556387E706316768
:109B10001307C755638AE70429671307A75563949A
:109B2000E702A285280097C0FFFFE780405715B7DE
:109B300039679306E7656381D70863E9F600130781
:109B4000E7556384E706A28528003DB73D67930685
:109B5000F755638AD7061307F766E396E7FE97C0C3
:109B6000FFFFE780C06FF5B50146A285280097C0CA
:109B7000FFFFE7800040F1BDA285280097C0FFFFEE
:109B8000E7802050F9B58947E3F587EC970000009E
:109B9000E780A0E49305E4FFC205C1811305A1009D
:109BA0009790FFFFE78020616DB5A285280097C0E0
:109BB000FFFFE780C04F71BDA285280097C0FFFF5F
:109BC000E780805A79B597C0FFFFE780006351B501
:109BD000C16717C5FF1F0355250DF9176307F5006A
:109BE000B7E7040003A3C71702838280854717C71E
:109BF000FF1F2309F70A014517F3FFFF6700235BE7
:109C00001783FFFFE702034B2A8408452E89B28998
:109C100019C900C1971500009385A5866105973085
:109C20000100E780800181447D5A97100000E780A1
:109C3000E03963C7A404814497100000E780003A2C
:109C400063C8A40497C7FF1F9387C7069C43DC47DC
:109C5000B307F94091872302F40063830904832743
:109C6000C900B307F4409587A302F4001C4C89C7D0
:109C70009C4799C3228582971783FFFF6700C346DD
:109C80005C44139714008504BA972390470171BF71
:109C90001C48139714008504BA972390070069BFE6
:109CA000832789000547B307F4409587A302F40092
:109CB00083570400638EE7028DC309476384E7047A
:109CC0000D47E395E7FA978701009387E7371CCCA8
:109CD000978701009387473811A8978701009387DA
:109CE00027FE1CCC97870100938787FE5CC8BDBF09
:109CF000978701009387C7E91CCC9787010093875A
:109D000027EAEDB7978701009387C7381CCC978760
:109D1000010093872739D9BF95E51783FFFFE70235
:109D2000033B004618448347940075839D8B63175B
:109D3000F70097100000E78060B448C41783FFFF66
:109D40006700233B82801783FFFFE702A336138956
:109D50003500C16442094111AA890144F114135923
:109D60000901054A2EC697100000E7802026B2455B
:109D70006348A400014541011783FFFF6700C33614
:109D800083A7090013171400BA9783D707006388C5
:109D9000B7006394970063742A010504E1B7054591
:109DA000D9BF1783FFFFE7020330AA892E89328BC0
:109DB000B6843A8ABE8A97A00000E78020FB71C96A
:109DC000268597200000E78020098D4763E7A700DC
:109DD0007D551783FFFF6700833083DB44009710B6
:109DE0000000E780A0242A8497100000E780402527
:109DF0009307740031443305850263CDA7029710A1
:109E00000000E780A02297100000E78020222A842B
:109E100097100000E780C022930774003144330597
:109E2000850263C3A70497100000E78020209307F2
:109E3000450029A897100000E7808020330585029F
:109E40001307F0179307C017E35FA7FA2D55E3C276
:109E500077F963040B02D6865286A6854A85972039
:109E60000100E78020BAB5B797100000E780401DD9
:109E7000330585029307C5FFD1BF832749001385AA
:109E8000C90083D5270097000000E78000EC61F54A
:109E900081B769553DBF97C7FF1F239FA7E097C7AD
:109EA000FF1F938727E1904381470C463307F50056
:109EB000420741836393B70082805446139847005A
:109EC0008507C2962390E600D5B797C7FF1F9387F3
:109ED00067DE9C4303C58700828017C5FF1F0355BB
:109EE000A5DD82801783FFFFE702631EC16713872A
:109EF000D7FF630BE502636AA700F1176300F50261
:109F000001451783FFFF6700C31E1387E7FF630246
:109F1000E502FD171D8D13351500E5B797500000BC
:109F2000E780C0267D15C5BF97500000E78040FB45
:109F3000D5BF97500000E78060F9EDB71783FFFFAA
:109F4000E702E3184111AA8401442EC697100000CD
:109F5000E780C008B2456348A4000145410117836A
:109F6000FFFF670003199C48131514003E958357A3
:109F70000500E385B7FE0504C9BF034855008146C7
:109F800093F7F60F63E5070181473E8582805845C8
:109F900093975600BA9703D727006316B70003D7E5
:109FA0000700E304C7FE8506E1BF8346450001477D
:109FB0009377F70F63E4D700814711A81C45131668
:109FC00057000507B29703D60700E313B6FE3E8598
:109FD00082801783FFFFE702E30D93170501C18716
:109FE00097CAFF1F938A0ACD635BF00883A70A0014
:109FF000C0479C4703570400198D4205418163689F
:10A00000F500014422851783FFFF6700E30D120569
:10A010002A94CDBFDC4713944900014A3E948347FC
:10A0200044006341FA02014A834754006349FA023B
:10A030008509C20993D9090183A70A009847E3EB70
:10A04000E9FCC1B71C4413195A00A6853E994A85FC
:10A0500097000000E780C0EE05E1050AC9B75C443F
:10A0600013195A00A6853E994A8597000000E7809B
:10A0700020ED19E1050A4DBFE30C09FA61B7AA8486
:10A0800081495DBF1783FFFFE70263041C452A84F3
:10A0900081E79307C5001CC51C44231204001CC0A3
:10A0A0009307F00F63EDB70093F5F50F2285972026
:10A0B0000000E78020E21783FFFF6700830393948B
:10A0C0000501C167C18063F9F500A6852285972047
:10A0D0000000E78040E5C5B7C18193F5F50F228503
:10A0E00097200000E78000DFA685228597200000EA
:10A0F000E78040E0C9B797C7FF1F9387A7BB884396
:10A1000082801C4599C797C7FF1F23A5A7BA0145A1
:10A1100082807D55828097C7FF1F9387A7B9984398
:10A1200083474500484792073E9582801783FFFF8B
:10A13000E702E3F9617100451C183EC6B7078001CC
:10A140003EC81C183ECA8357440002CE02D002CC3F
:10A15000231EF100834784002A8902D22301F102E1
:10A160003C083ED402D697000000E78000FB8357EE
:10A1700005002316F10297500000E78060C4230712
:10A18000A1025C4003556400F18313F71700834775
:10A19000F10252055181F99BD98FA307F102971063
:10A1A0000100E780807539CDAA840355050097A08A
:10A1B0000000E78080BC83D704002AD26800231CFB
:10A1C000F10083D72400231DF1001C4803D647006B
:10A1D0008C4397200000E78000CD8347B400CA86F7
:10A1E00017860100130646948117A305F4006C003E
:10A1F000481097200100E780E0805D611783FFFF32
:10A20000670023EF2155D5BF1C45B1CF03C5A7007B
:10A21000894613576500630BD7028D46630ED7023C
:10A2200085466300D702130740063305E50203C7DE
:10A23000B700418B15CB83C7B700BD8B3355F540B5
:10A2400082801375F5031307803EC5B70967137540
:10A25000F50313070771D1BF372709001375F503FD
:10A260001307077CD9B7014582801783FFFFE702F8
:10A2700003E603A98500630C09048347B900AE8493
:10A2800093F7070E85C303459900930520030D81BD
:10A290000505B305B5028844610597300100E780E4
:10A2A000E0A935A02E8597000000E78020F62A84DB
:10A2B00019CD97000000E780605C8325C900B307D3
:10A2C000B54063FA87002E94B305A440E9F51783DF
:10A2D000FFFF670003E285457DBF1783FFFFE702AD
:10A2E00003DF2A8403D50500011132C636C43AC201
:10A2F0002EC002CA02CC02CE97A00000E780E0A7E1
:10A3000082452ACA22852ECC97000000E780E0E033
:10A3100003570500231EE10097500000E78040AA84
:10A32000A24632469247230FA10036874C08B286D8
:10A330002285014697000000E780E0A605611783AB
:10A34000FFFF670003DB1783FFFFE70243D861715C
:10A350001C183EC6B70780013EC81C183ECA3C0800
:10A3600000453ED4AA8402CC02CE02D002D202D64C
:10A3700097000000E78060DA8357050035592316FF
:10A38000F10297500000E780A0A32307A10209C4AF
:10A390008357440081EB21594A855D611783FFFF94
:10A3A000670023D5035564005205518197100100C1
:10A3B000E780A0542A8965D18347B40093F7070E3C
:10A3C00099C71305840197300100E780609983578E
:10A3D0004400231EF100834784002301F1025C4006
:10A3E00003550900D98313F7070883471102231C7B
:10A3F000A10093F7F707D98FA300F1028357290033
:10A40000231DF1005C40F18313F717008347F1022D
:10A41000F99BD98FA307F10297A00000E780E09590
:10A420002AD235D983479400680013975700834791
:10A43000B400FD8BD98FA305F4001C4803D6470058
:10A440008C4397200000E78000A6A68717770100BD
:10A450001307876D740005464C1026859700000091
:10A46000E78060942A890DD98347B400A685FD8BC7
:10A47000A305F40097000000E78060DF31BF178379
:10A48000FFFFE702C3C4832485FE2A844111268589
:10A4900097000000E78080D7834734FF93F7070ECB
:10A4A0008DCB2AC6268597000000E78060C809CDBD
:10A4B000834734FFB245FD8BA309F4FE91C5228585
:10A4C00097300100E780808741011783FFFF670015
:10A4D00043C27DD98327C4FF2685829775F58347BC
:10A4E00034FF93F7070E91C7228597300100E7806C
:10A4F0002087032584FE97000000E78000E5E9B788
:10A500001783FFFFE702A3B99C4141112A8903C7C2
:10A51000070089472E84935667006380F6040D4632
:10A520006388C6049307F0076304F7022E8597201B
:10A530000000E780C0A7AA848149C16B130C4900C1
:10A5400097B7FF1F938707779C43984763E4E90415
:10A5500041011783FFFF670043B803D745008547D4
:10A56000E3F8E7FE2E8597200000E780A0A9E1B779
:10A5700003D74500E3FEE7FC2E8597200000E78027
:10A5800000A3AA84228597200000E78060A4C2046B
:10A59000C98C5DB7DC470355A900139A49003E9A60
:10A5A00093170501C187635DF00083570A00639725
:10A5B000A70263E774038327CA00034D5A002DA046
:10A5C000A1672167A98F1307F7EFE374F7FE63977D
:10A5D000090097000000E780209161FD85098DB793
:10A5E00083278A00034D4A00835DA9000357690051
:10A5F000216A138BC7003AC6814A33CA4D01631ED4
:10A600005D0197B7FF1F9387676B9C43E1DBA286D1
:10A610006286814526858297D1B7A1679387F7EF38
:10A62000930C4BFF63F24703B2455A8597F0FFFF47
:10A63000E780A0710DC103278B00104709CE10439E
:10A640006382C4023107D5BFEE856685970000009E
:10A65000E780008F71F993861A0093FAF60F130BB7
:10A660000B0271BF835644005C43E3E9F6F6228592
:10A670003AC697100000E780807DA1679387D704D2
:10A680002A8A035D4400324763E897008347D90074
:10A6900093E707F8A306F9001C4766852286E28542
:10A6A0008297C1670844FD17337AFA00529508C0B3
:10A6B0002312A40125B797B7FF1F9387A75F98437D
:10A6C000814715C31447814763FFD5009397450021
:10A6D0004C47BE9519C903C7550081476375E6000D
:10A6E000DC451606B2973E85828003C74500814748
:10A6F000E37BE6FE16069C45F5B71783FFFFE702EE
:10A70000639BAA892E8A814497BAFF1F938A8A5A2B
:10A7100083A70A00984763E6E4001783FFFF6700FA
:10A72000A39CDC471394440001493E9413BB1400DE
:10A7300083474400634BF900014913BB140083476E
:10A740005400634FF9008504E1B70844931759009A
:10A750005287DA860146A2853E9582990509C9BFCE
:10A760004844931759005287DA860546A2853E95DC
:10A7700082990509E9B71783FFFFE70243958145F1
:10A7800017F5FFFF1305054897B7FF1F23960752DC
:10A7900097000000E780A0F61783FFFF670063952E
:10A7A00097B7FF1F938707519C4395C31783FFFFFC
:10A7B000E702E391814517F5FFFF1305A5449700D4
:10A7C0000000E780C0F31783FFFF67008392828059
:10A7D0001783FFFFE702038E37E404008327841208
:10A7E00041112315E100AE893289368A3A868146C5
:10A7F0000147ED45AA8482972AC621C90356A100C4
:10A80000D28597400100E780C0248327C413CE85FA
:10A8100026858297058905C98327440D23142101C4
:10A8200001462C00268582972A8401C9B7E70400D7
:10A8300083A7C712ED45280082972285410117831F
:10A84000FFFF6700638A4944D5B76554FDB75C4193
:10A85000FD175CC182801783FFFFE7024387B7E7DC
:10A860000400FC5F829795473305F50281450D8111
:10A870001783FFFF6700E3871783FFFFE702238546
:10A88000B7E70400FC5F829795473305F5020D8119
:10A890001783FFFF6700E3851783FFFFE70223832A
:10A8A000B7E7040083A7870B03550500829717833A
:10A8B000FFFF670003841783FFFFE702438103550F
:10A8C00005003287AE861796FF1F0356C6BD97B5A3
:10A8D000FF1F9385E53E97000000E780A0EF1783F8
:10A8E000FFFF670003811773FFFFE702437EB7E7AF
:10A8F000040083A7C71782971773FFFF6700637F62
:10A900001773FFFFE702A37CB7E7040083A7871351
:10A9100097B5FF1F9385C53A829701451773FFFFCF
:10A920006700237D1773FFFFE702637AB7E7040030
:10A9300083A7C71F81451795FF1F0355C5B282978F
:10A940001773FFFF6700E37A1773FFFFE7022378AF
:10A95000B7E7040083A7871397B5FF1F9385453793
:10A96000829701451773FFFF6700A3781773FFFFF6
:10A97000E702E375B7E7040083A7C71F8145179572
:10A98000FF1F035545B482971773FFFF6700637677
:10A990001773FFFFE702A3732E8597800000E780FF
:10A9A000E0AF97800000E780E0EC1773FFFF6700DF
:10A9B00043741773FFFFE702837197800000E780FD
:10A9C000E0F61773FFFF6700C3725C49E1175CC9CB
:10A9D0005CC583572501A1072319F500835705019D
:10A9E000A1072318F5008280F1473305F50297B7D8
:10A9F000FF1F9387E72F9C433E9582808D47631509
:10AA0000F60803D74600854763F0E7081773FFFF92
:10AA1000E702E36B368536842E8997100000E780C5
:10AA2000005929C98357440093140501C18063E389
:10AA30009704228597100000E7806057FD142312C9
:10AA400094009307A0026300F5029307B002630726
:10AA5000F50293079002631FF5002285970001001D
:10AA6000E780C08501A80146CA85228597A000001D
:10AA7000E78060B01773FFFF6700A3672285971018
:10AA80000000E780C003FDB7828097B6FF1F938662
:10AA900066269C42014599CF9843D44217B6FF1FC2
:10AAA000232AE6246396D70097B6FF1F23A6E62441
:10AAB0001385C7FE82801773FFFFE702436197008B
:10AAC0000000E780A04B71443305850291459790C3
:10AAD0000000E78020E911E565551773FFFF670067
:10AAE000436197B7FF1F23A3A72097000000E780CB
:10AAF000E04833058502914597900000E78080E6A5
:10AB000061DD97B7FF1F23A5A71E97000000E78010
:10AB1000E04697B7FF1F2395A71C97000000E7802A
:10AB2000E04597B7FF1F239EA71A977701009387E9
:10AB3000E70417B7FF1F2329F71A97070000938729
:10AB400007E917B7FF1F232FF718014579B71773C8
:10AB5000FFFFE702C357AA8517B5FF1F1305451866
:10AB600097100000E780C05B1773FFFF6700635812
:10AB70001773FFFFE702A35597000000E78060FD11
:10AB800097100000E780405B97B7FF1F93878716F9
:10AB90009C4391CF1387C7FE19CB83D5C7FF17B549
:10ABA000FF1F1305A51597200100E78020191773D3
:10ABB000FFFF670003541773FFFFE702435197003D
:10ABC0000000E780C0EC09CD834785002A8493F715
:10ABD000070499EB0355E50097000000E78080F932
:10ABE0001773FFFF6700E3508347C50093044501D7
:10ABF00017B9FF1F1309091085E3832709005CC9F2
:10AC000097B7FF1F23A8970E83274900F1FB97B73B
:10AC1000FF1F23A3970EE9B7FD172306F500610573
:10AC200097800000E780C0D68307840063CB0704C9
:10AC30008347840093E707F82304F400B7E7040090
:10AC40009C5F82974205A94741813375F50283478E
:10AC5000840093F707FCC98F2304F4008347D400D2
:10AC60003E951C402318A40089CF984319CB8347F5
:10AC7000C4005040814585073305F50242054181F6
:10AC80000297832709005CC897B7FF1F23A4970684
:10AC90008327490089E797B7FF1F23AF97048347AE
:10ACA000C4009DDF8355040117B5FF1F130505057B
:10ACB00097200100E780800825B71773FFFFE702A0
:10ACC000034197B7FF1F9387A7289C4701448583BB
:10ACD000858B85E3AE84B2853A8697100000E780C5
:10ACE000804B2A8419C597100000E780C0418294E8
:10ACF00008CC22851773FFFF6700A33F1773FFFF80
:10AD0000E702433B41112E8932C6AA899700000011
:10AD1000E780C031324713060502CA869705000056
:10AD20009385C5CC17B5FF1F130585FB9700000061
:10AD3000E780E0F82A8425C99304C5009700000045
:10AD4000E780E0411946AA85268597100000E78034
:10AD500080158545268597100000E78060111775DE
:10AD60000100130565DF4E95834505002685971084
:10AD70000000E78020165C4831468145A1075CC889
:10AD80005CC483572401E1172319F400835704019D
:10AD9000E1172318F4001C4C3E859770FFFFE780F5
:10ADA0000036A3042501228541011773FFFF6700C8
:10ADB000A3331773FFFFE70283314111AA842EC624
:10ADC00032C497100000E7806036004DB24522463D
:10ADD000834784000CC050C093F7F70393E7070440
:10ADE0002304F40023180400268597100000E78050
:10ADF000803183479400A9462317A40013D7370056
:10AE000005073307D7029D8B85072306F400A306A9
:10AE1000E40083C70401D8488507230FF7FE17B75E
:10AE2000FF1F130727ED5843232A0400930744010B
:10AE300029E317B7FF1F2321F7EC17B7FF1F232BB9
:10AE4000F7EA17B4FF1F130464EB22859720010073
:10AE5000E78000E11C44858B5D8D19E581452285E5
:10AE600097200100E78080ED41011773FFFF670025
:10AE700043281CC317B7FF1F2320F7E8D9B7177360
:10AE8000FFFFE702C32497050000938565B70145DE
:10AE900097000000E78000B001451773FFFF6700CF
:10AEA00043251773FFFFE702832297000000E78026
:10AEB00080B01773FFFF6700C3238347C500A5E376
:10AEC0001773FFFFE702A3202A840355E5009700CC
:10AED0000000E78000C821C18347840093F7F7FB97
:10AEE0002304F4001C4091C7DC4381C74C4001455A
:10AEF000829797000000E78080B917B5FF1F130500
:10AF0000E5DF97200100E780A0E50355E400970006
:10AF10000000E78020C61773FFFF6700831D828053
:10AF20001773FFFFE702A31A97B7FF1F938787DC0A
:10AF300097050000938565C817B5FF1F130505DC4D
:10AF400023A0070023A2070097200100E780E0CE9E
:10AF50001773FFFF6700E3191C4D91CFDC4381CFCE
:10AF60001773FFFFE702A316834507008297177345
:10AF7000FFFF67000318828097B7FF1F938747DAA8
:10AF80009C4303C50700828097B7FF1F938747D96B
:10AF90009C4303C51700828097B7FF1F938747D84C
:10AFA0009C4303C52700828097B7FF1F938747D72D
:10AFB0009C4303C54700828097B7FF1F938747D6FE
:10AFC0009C4303C53700828097B7FF1F938747D5FF
:10AFD0009C4303C55700828097B7FF1F938747D4D0
:10AFE0009C4303C56700828097B7FF1F938747D3B1
:10AFF0009C4303C57700828097B7FF1F938747D292
:10B000009C4303C58700828097B7FF1F938747D172
:10B010009C4303C59700828097B7FF1F938747D053
:10B020009C4303C5A700828097B7FF1F938747CF34
:10B030009C4303C5B70011E11D45828097B7FF1FF0
:10B04000938707CE9C4303C5C700828097B7FF1F35
:10B05000938707CD9C4303C5D700828097B7FF1F16
:10B06000938707CC9C4303C5E700828097B7FF1FF7
:10B07000938707CB9C4303D50701828097B7FF1FB7
:10B08000938707CA9C4303C52701828097B7FF1F98
:10B09000938707C99C4303D54701828097B7FF1F59
:10B0A000938707C89C4303D56701828097B7FF1F2A
:10B0B000938707C79C4303D58701828097B7FF1FFB
:10B0C000938707C69C4303C5A701828097B7FF1FDC
:10B0D000938707C59C4303C5B701828097B7FF1FBD
:10B0E000938707C49C4303C5C701828097B7FF1F9E
:10B0F000938707C39C4303C5D701828097B7FF1F7F
:10B10000938707C29C438857828097B7FF1F938716
:10B1100027C19C4303D5C702828097B7FF1F93873F
:10B1200027C09C4303D5E70219E11305800C8280F8
:10B1300097B7FF1F9387C7BE9C4303C50703828051
:10B1400097B7FF1F9387C7BD9C43C85B828097B7A3
:10B15000FF1F938767BC8843828097B7FF1F938741
:10B16000E7BB8843828019E17D558280F5DE9842F5
:10B1700065DFFDD917B7FF1F130787DD1847AA87BB
:10B180007155058B631D072403C507001547E37D33
:10B19000A7FC03C737001305F0057D171377F70FDA
:10B1A000E364E5FC03C35700E30003FC83C86700C6
:10B1B000E38C08FA03C77700494579171377F70F2F
:10B1C000E364E5FA03C7A70011481305F7FF1375F9
:10B1D000F50FE36BA8F803CE97000D481305FEFFAB
:10B1E0001375F50FE362A8F803C8B70063090800F8
:10B1F00065181378F80F1305600DE36705F703C5AD
:10B20000C700794879151375F50FE36FA8F403C8E3
:10B21000D7000D457D181378F80FE36705F503D8BF
:10B220000701930E40175118420813580801E3ED27
:10B230000EF303C8E7007D181378F80FE36605F3F3
:10B2400003C827017D181378F80FE36F05F103C8D1
:10B250008700C54E75181378F80FE3E70EF103D891
:10B260006701856E938EBEE06D1842081358080181
:10B27000E3EC0EEF03D847016D184208135808019C
:10B28000E3E40EEF03D88701791842081358080148
:10B29000E36C05ED03C8A7017D181378F80FE3658B
:10B2A00005ED03C5B7011D487D151375F50FE36D59
:10B2B000A8EA03C5D701714879151375F50FE36541
:10B2C000A8EA03D5E7011308E00F7D154205418187
:10B2D000E36CA8E803C50702494879151375F50F13
:10B2E000E364A8E8C85301C937C8340059151308E6
:10B2F00058BFE36BA8E603A8870237C534001305DF
:10B3000055BF5918E36205E717B5FF1F2328C5A0ED
:10B3100003C6050117B5FF1F2324F5A00545E375F6
:10B32000C5E403D82501D04933760603E31E06E2BF
:10B3300003C61501E30A06E217B6FF1F232EB69CCB
:10B3400083C5270001466387A50003C61700F145A2
:10B350003306B60283C707039305C00272971A0724
:10B360001307C70516031A9796084697B387B702BF
:10B3700041553E973297420741836362E80617734F
:10B38000FFFFE702C3D4368597800000E780A068FE
:10B3900097000100E78020482A8497A00000E780FA
:10B3A000805A2A9497F00000E78060262A949790AC
:10B3B0000000E780A0812A9497F0FFFFE780E06F0C
:10B3C0002A9497400000E78060932A9497700000C9
:10B3D000E780A09C22951773FFFF670083D18280CE
:10B3E0001773FFFFE702A3CE4111A307A10097A0A7
:10B3F0000000E780A0C59305F100170500001305C4
:10B40000E5B597F0FFFFE780802F014541011773F5
:10B41000FFFF670003CE1773FFFFE702C3C817B42F
:10B42000FF1F1304E4B203288400795993681800BD
:10B4300097B4FF1F23A214B31378180063100802F7
:10B44000BA84BE89368B328A2E89AA8A97F0FFFF8A
:10B45000E780E0A77D15269519E531594A851773D0
:10B46000FFFF6700C3C797F0FFFFE78040A67D1589
:10B470002695A167E353F5FE97B7FF1F938707E46F
:10B4800098433E8C814B01CB014597F00000E7804B
:10B490002044933B15004A85DA865686D2859790DC
:10B4A0000000E780C04D2A8911CD1C44F99B17B7D5
:10B4B000FF1F2323F7AA83270C00CDD3E3800BFAC9
:10B4C000829769BF268597B7FF1F23A507A897F026
:10B4D000FFFFE780809C4146CE8517B5FF1F13050F
:10B4E000A5B097300100E780C05697D00000E780F4
:10B4F00040990325040B97D00000E780009D054587
:10B5000097D00000E78000A4054597000000E78081
:10B5100060EDA9B797B7FF1F938787A39C47858BDB
:10B52000EDC71773FFFFE70283BA17B5FF1F1305B7
:10B53000E5A997B7FF1F23AD07A097B7FF1F23AB60
:10B5400007A097B7FF1F23A907A097200100E78056
:10B55000208197500000E780E0F597100100E78018
:10B56000A04C97100100E780A05297B7FF1F938768
:10B57000A79C9C4391C7054597800000E780402029
:10B5800097B7FF1F938707859C4399C741657D1532
:10B5900097700000E78040A297F00000E780E03D50
:10B5A00097D00000E780808F97B7FF1F938707AF82
:10B5B0009C43139717016356070097F00000E7803C
:10B5C00000AD97B7FF1F23A107A297B7FF1F23AFB7
:10B5D00007A097B7FF1F23AD07A097B7FF1F23ABA7
:10B5E00007A097000000E780008C97000000E7802C
:10B5F000007297F0FFFFE780401897F00000E780A7
:10B6000040D61773FFFF6700C3AE828097B7FF1F56
:10B6100093870794884382801773FFFFE70223AB69
:10B6200097800000E780607597800000E780C07712
:10B630001773FFFF6700E3AB1773FFFFE70283A7F2
:10B640002A849304140201112E85B289A68521460D
:10B6500036C63A8997300100E780403D0DE9B24691
:10B6600038082686CE851305940497500000E7809D
:10B67000604121462C084A8597300100E780003B55
:10B680001335150005611773FFFF6700E3A501453A
:10B69000D5BF1773FFFFE70283A39305450617A5E0
:10B6A000FF1F1305256897100100E78020691773B5
:10B6B000FFFF670003A41773FFFFE70243A14111D7
:10B6C0002EC697F0FFFFE780601BB24588C141019D
:10B6D0001773FFFF6700E3A11773FFFFE702839D66
:10B6E000AA842E8497800000E780006CAA89854593
:10B6F000228597000000E780E07D83C7E40113897D
:10B70000940899E313890403CE85228597000000ED
:10B71000E780407C214693051902228597000000AE
:10B72000E780607897B7FF1F938787828C432285D5
:10B7300097100000E780C08221469385840222850D
:10B7400097000000E78020761773FFFF6700C3991A
:10B750001773FFFFE7022395397197F00000E78028
:10B76000E0B49305400661E997800000E78000603F
:10B770006302051497A7FF1F83C7875C13B71700E1
:10B7800097A6FF1F238EE65A014499CFC16417A9DB
:10B79000FF1F1309E97B9309400EFD149700000079
:10B7A000E780C0866342A40A97F0FFFFE780000DA0
:10B7B0004169B7290900096AFD7A2A8B81447D19FC
:10B7C0009389F97B130A0A71938A8AC7970000004C
:10B7D000E780C08363D7A4041304400EB3878402B8
:10B7E00017A7FF1F1307C7760324070B3E94835741
:10B7F000C4016382270B18403307EB4063EAE9007A
:10B80000834744008507B3874703D6976365F708E6
:10B8100001468145094597F0FFFFE780604EAA8BFE
:10B8200029E597400000E780808385476317F50688
:10B8300089659385057117A5FF1F1305A54E971000
:10B840000100E780A04F95A0B30734030327090B3D
:10B85000BA9703D7C7016308970003C75700A382AD
:10B8600007002382E700050415BF9305C500228564
:10B8700097000000E78080E65E85228697650100DC
:10B880009385C52E97F0FFFFE780E0525E85971005
:10B890000000E780608A850415BF97A7FF1F938784
:10B8A000276B9C478D83858BC1F721611773FFFF41
:10B8B0006700E38201468545094502D002D202D4E1
:10B8C00002D697F0FFFFE780A043AA8479DD97F0C6
:10B8D0000000E780E09C1389C4002A8481454A85E2
:10B8E00097000000E780005F0C4041464A859700C2
:10B8F0000000E780405B832944006385090C4E8586
:10B9000002D802DA02DC02DE97300100E7806040F4
:10B910002ACE141005462C0808184ECC975000006B
:10B92000E780E00A1375F50F51ED8355840093E528
:10B9300025004A8597000000E780E05E11460C1064
:10B940004A8597000000E780005601469765010090
:10B9500093854522268597F0FFFFE780C045268521
:10B9600097000000E780407D5C40A1D301468545FB
:10B970000D4597F0FFFFE780A038AA841DD5484009
:10B980001389C40097300100E780A0382AC64A8591
:10B9900097000000E780404C3246636FC5004C4082
:10B9A0004A8597000000E7800050014681452685C2
:10B9B00097F0FFFFE7802040268597000000E78092
:10B9C000A077E5B583558400ADB71763FFFFE702A5
:10B9D000037097A7FF1F9387A7579C471DC193E745
:10B9E000870017A5FF1F1305E53317A7FF1F2325A2
:10B9F000F75697100100E78040321763FFFF67009A
:10BA0000436FDD9B17A7FF1F2328F75497300000D3
:10BA1000E780E0647DF117A5FF1F1305A53097109F
:10BA20000100E780E033D1BF1763FFFFE702A367A0
:10BA30004169AA892E8AB28A368BBA8B814417ACA7
:10BA4000FF1F130CEC50930C400E7D1997F0FFFF75
:10BA5000E780C05B63C4A40001443DA03384940329
:10BA600083270C0B3E948357C401638627055A87AE
:10BA7000D6865286CE851305040397000000E78022
:10BA8000E0BB01C923800B0022851763FFFF67001D
:10BA900003658347F40185C35A87D6865286CE85CF
:10BAA0001305940897000000E78040B909C5854751
:10BAB0002380FB00D1BF850451BF835745006380BD
:10BAC000071E1763FFFFE702E35E01112A84970058
:10BAD0000000E780C04D09C985476309F506056187
:10BAE0001763FFFF6700436097E00000E780007C7A
:10BAF0007DF5835744004947ED9BE392E7FEC1453E
:10BB0000228597000000E7804033AA8422859700B1
:10BB10000000E780204F0357440002CE91472A8956
:10BB2000631AF700228597000000E780A0513C08C7
:10BB30002ACC3ECE97E00000E78080765C55C5D3E6
:10BB400074084A86A6850545829751BF035744006D
:10BB5000D147E3F6E7F8032A0400C169014997AA2F
:10BB6000FF1F938AEA3E130B400EFD1997F0FFFF6B
:10BB7000E780C049634FA90E2285032A040097007D
:10BB80000000E780C042A1452A8922859700000075
:10BB9000E780A02AAA84228597000000E780804AD7
:10BBA00014402A86AA8978082685CA85970000004D
:10BBB000E780C0E7AA8405D503C7F4018947631568
:10BBC000F7008347C10181DF5546D28513856400A4
:10BBD00097300100E780E0E7014597800000E780AB
:10BBE000C01901C583D7C401A5E797A7FF1F938795
:10BBF00027369C4793551900858913D73700058B45
:10BC000001CF8983858B6399B70001452EC69700C4
:10BC10000000E780C0DBB2454E8597800000E780DA
:10BC2000601F0346C1012A849375190026859790E9
:10BC30000000E780E03935C1268597800000E78065
:10BC4000E018268511C0014597800000E780004C70
:10BC500097300000E780A0408547E312F5E883C7EE
:10BC600054001307F00FE38CE7E68507A382F40086
:10BC7000BDB5B304690383A70A0BBE9483D7C4017F
:10BC8000638B37015546D2851385640097300100D8
:10BC9000E780C0D955DD0509D1BD5DD86DB782807B
:10BCA0001763FFFFE702034197800000E780000C65
:10BCB00005C1C164014417A9FF1F1309692993092C
:10BCC000400EFD1497F0FFFFE7804034634EA40060
:10BCD00017A5FF1F1305050597100100E780E00376
:10BCE0001763FFFF67004340330534038327090BC5
:10BCF0003E958357C50163889700231205009780FE
:10BD00000000E780A00C050475BF97A7FF1F93876D
:10BD100027249C478D83858B8DE31763FFFFE70204
:10BD2000033B17A5FF1F1305E5FF97100100E780F0
:10BD300020031763FFFF6700C33B82801763FFFF89
:10BD4000E702E338970500009385C5A017A5FF1FFC
:10BD5000130545FD97100100E78020EE1763FFFFF4
:10BD6000670023391763FFFFE70263368841B7E7AF
:10BD70000400BC5B050542054181829709C58547E2
:10BD80002300F50005051763FFFF6700833683C7AF
:10BD9000F5FF2E858507A38FF5FE828083C7F5FF0B
:10BDA000FD1793F7F70FA38FF5FE99EF1763FFFFCA
:10BDB000E702E331B7E70400BC571385F5FF82972C
:10BDC0001763FFFF6700E33282801C410357450081
:10BDD0008D8FBA951CC12312B5003E85828093D702
:10BDE0008500A2051441DD8D835745001387E6FFCA
:10BDF00018C189072312F50013D685004111238F3E
:10BE0000B6FEA38FC6FE4101828018419307F7FF5B
:10BE10001CC18357450085072312F500A30FB7FE09
:10BE20008280835745008D8F2312F5001C41BE95FB
:10BE30000CC12E858280AA8703D7470008410D8F49
:10BE4000AA952392E7008CC38280184108453305E8
:10BE5000A740828083574500035765001D8F1C4112
:10BE600008453385A7403305A74082801763FFFF4D
:10BE7000E702E32541112EC62A8497000000E780DF
:10BE8000A0FDB2456373B50001A08357440008408C
:10BE9000BE952312B4003E9541011763FFFF670072
:10BEA00043251763FFFFE702832241112E84B285E9
:10BEB00032C697000000E780A0FB3246A28597308B
:10BEC0000100E78000B941011763FFFF67006322AB
:10BED0001763FFFFE702A31F2E848545970000002C
:10BEE000E78000F9230085001763FFFF67006320E8
:10BEF0001763FFFFE702A31D41112317B100894516
:10BF000097000000E780C0F68347E1002300F500BA
:10BF10008347F100A300F50041011763FFFF6700AD
:10BF2000431D1763FFFFE702831A93D78500A2051D
:10BF30004111DD8D2317B100894597000000E7808E
:10BF400020F38347E1002300F5008347F100A300BD
:10BF5000F50041011763FFFF6700A3191763FFFF97
:10BF6000E702E3161397850193D78501C16693868F
:10BF700006F0D98F13D78500758FD98FA2053707A3
:10BF8000FF00F98D4111DD8D2EC69145970000000F
:10BF9000E78000EE6C00114697300100E78060AB4F
:10BFA00041011763FFFF6700C3141763FFFFE70238
:10BFB00003121C41854503C4070097000000E78079
:10BFC00080E622851763FFFF6700A3121763FFFF58
:10BFD000E702E30F1C414111894503C7070083C7EE
:10BFE00017002307E100A307F10097000000E78096
:10BFF00080E30355E10041011763FFFF6700630F12
:10C000001763FFFFE702A30C1C414111894503C7D9
:10C01000070083C717002307E100A307F10097007B
:10C020000000E78040E08357E100410113D587001D
:10C03000A2075D8D420541811763FFFF6700630B17
:10C040001763FFFFE702A3080C4141112A84114640
:10C05000680097300100E780C09F914522859700D6
:10C060000000E78040DCB247C166938606F0139774
:10C07000870113D58701598D13D78700758F598D87
:10C08000A2073707FF00F98F5D8D41011763FFFF9E
:10C09000670023061C45BE950CC18280AE87944381
:10C0A00091E6584101EF0CC15CC1828003C7570083
:10C0B00013671700A382E700B687D5B70CC3EDB7A7
:10C0C000AA87084119CD1841D44398C36313D500FA
:10C0D000D8C32A87034657009376160081E62320AB
:10C0E00007008280944381CA8C4203A847008CC316
:10C0F00063930601CCC3799A14C3A302C7003687A1
:10C10000D1BF1C45DC471D8DB777DBB6938777DB46
:10C1100009853305F502420541818280F147B385E7
:10C12000F50248452E958280834745008507230206
:10C13000F50082801763FFFFE70263F92A8409E4B0
:10C140001763FFFF6700E3FA83474400F5DBFD1741
:10C1500093F7F70F2302F400E5F71C4403D72700F9
:10C1600005072391E700DC4399C3228582974C4859
:10C1700089CD83475400898B99E71C4422859C47CD
:10C180009C439C478297232A0400004023200400FC
:10C190007DB71763FFFFE70283F383572500411143
:10C1A0002EC681EB0144228541011763FFFF670022
:10C1B00043F4035705008147F146E305F7FEB385D5
:10C1C000D702404585072E948345440008C4F5F501
:10C1D000B247AA8481E7232A040009A81C456C0001
:10C1E00022859C439C43829748C84DDD8547231296
:10C1F000F400B24723200400231804002319F4009C
:10C200005C485CC483D72400FD172391F40061BF10
:10C210001763FFFFE702A3EB97A7FF1F938787B280
:10C2200088432326050023240500410597100100BB
:10C23000E78000B31763FFFF6700A3EB1763FFFFFF
:10C24000E702E3E817A4FF1F1304C4AF1C40411129
:10C2500099CF9C472300B5002AC65CC19700000017
:10C26000E78040FB1C40DC4399C332458297410183
:10C270001763FFFF6700E3E70347450029E3584DD5
:10C28000AA877D551DCF1763FFFFE70243E41CC358
:10C29000DC4797A6FF1F23A7E6AAF156130507015F
:10C2A0002390D700970500009385050297100100A1
:10C2B000E780A09801451763FFFF670083E37D5582
:10C2C000828082801763FFFFE70263E0011161460D
:10C2D000814528009760FFFFE78060E297A7FF1F76
:10C2E000938747A69C4328009305F00FDC473EC682
:10C2F00097000000E780C0F405611763FFFF670047
:10C3000043DF97A7FF1F9387E7A39C43D847A16705
:10C310009387C702631EF70A397106DE22DC26DA2C
:10C3200080004AD84ED652D456D23285B284970075
:10C330000000E780C0C7AA89268597000000E78033
:10C3400020C92318A4FC268597000000E78040C878
:10C350002319A4FC268597000000E78060C783D7D7
:10C3600044000A8A231AA4FC858393F7F70F230E4F
:10C37000F4FC8607BD0793F7073F3301F1408A8A33
:10C3800001498347C4FD6367F902CE85130584FC28
:10C39000232C54FD97000000E78080EA52811301AE
:10C3A00004FCF2506254D2544259B259225A925A61
:10C3B00021618280268597000000E78060C1931785
:10C3C0001900D69705092390A7001379F90F55BFD7
:10C3D000828097A7FF1F9387E7969C43D847A16762
:10C3E0009387A702631AF70A397106DE22DC26DA80
:10C3F00080004AD84ED652D456D23285B2849700A5
:10C400000000E780C0BAAA89268597000000E7806F
:10C4100020BCFD572318A4FC26852319F4FC9700A3
:10C420000000E780E0BA83D744000A8A231AA4FCFC
:10C43000858393F7F70F230EF4FC8607BD0793F768
:10C44000073F3301F1408A8A01498347C4FD63678E
:10C45000F902CE85130584FC232C54FD97000000BF
:10C46000E78000DE5281130104FCF2506254D25482
:10C470004259B259225A925A2161828026859700E8
:10C480000000E780E0B493171900D69705092390C0
:10C49000A7001379F90F55BF828097A7FF1F9387D5
:10C4A000678A9C43D847A16789076310F70A3971E7
:10C4B00006DE22DC26DA80004AD84ED652D456D286
:10C4C0003285328997000000E78060AEAA894A85EC
:10C4D00097000000E780C0AF835749000A8A2318FD
:10C4E000A4FC858393F7F70F230CF4FC8607BD07A4
:10C4F00093F7073F3301F1408A8A8144834784FDE3
:10C5000063E7F402CE85130584FC232A54FD9700CB
:10C510000000E780E0D25281130104FCF250625423
:10C52000D2544259B259225A925A216182804A8584
:10C5300097000000E780C0A993971400D697850460
:10C540002390A70093F4F40F55BF82809797FF1FA5
:10C550009387477F9C43D847A1679387E704631E6F
:10C56000F70A397106DE22DC26DA80004AD84ED678
:10C5700052D456D23285B28497000000E78020A3BF
:10C58000AA89268597000000E78080A42318A4FCD0
:10C59000268597000000E780A0A3231AA4FC268527
:10C5A00097000000E780C0A283D744000A8A2319BD
:10C5B000A4FC858393F7F70F230EF4FC8607BD07D1
:10C5C00093F7073F3301F1408A8A01498347C4FD4D
:10C5D0006367F902CE85130584FC232C54FD970074
:10C5E0000000E780E0C55281130104FCF250625460
:10C5F000D2544259B259225A925A216182802685D8
:10C6000097000000E780C09C93171900D697050992
:10C610002390A7001379F90F55BF82809797FF1FCA
:10C62000938747729C43D847A1679387C704631ACF
:10C63000F70A397106DE22DC26DA80004AD84ED6A7
:10C6400052D456D23285B28497000000E7802096FB
:10C65000AA89268597000000E7808097FD57231858
:10C66000A4FC2685231AF4FC97000000E78040967E
:10C6700083D744000A8A2319A4FC858393F7F70F14
:10C68000230EF4FC8607BD0793F7073F3301F14003
:10C690008A8A01498347C4FD6367F902CE85130581
:10C6A00084FC232C54FD97000000E78060B9528180
:10C6B000130104FCF2506254D2544259B259225A26
:10C6C000925A21618280268597000000E780409081
:10C6D00093171900D69705092390A7001379F90F2E
:10C6E00055BF82809797FF1F9387C7659C43D847A4
:10C6F000A167DD076317F7041763FFFFE702239DB8
:10C7000079713285328497000000E780408A2AC61A
:10C71000228597000000E780A08B2311A1022285CB
:10C7200097000000E780A088B2452300A1022808F6
:10C7300097000000E780C0B045611763FFFF670006
:10C74000439B82809797FF1F9387C75F9C43D8477F
:10C75000A167938787046317F7041763FFFFE70256
:10C76000039779713285328497000000E780208436
:10C770002AC6228597000000E78080852311A10248
:10C78000228597000000E7808082B2452300A10245
:10C79000280897000000E780A0AA45611763FFFF03
:10C7A0006700239582809797FF1F9387A7599C4323
:10C7B000D847A1679387A7046312F7021763FFFFA7
:10C7C000E702E39001112800814597000000E7800F
:10C7D00020A705611763FFFF6700A39182809797E9
:10C7E000FF1F938727569C43D847A167938757021B
:10C7F0006319F7021763FFFFE702638D01113285AA
:10C8000097F0FFFFE780A07A2308A1008145280068
:10C8100097000000E780C0A205611763FFFF670073
:10C82000438D82809797FF1F9387C7519C43D847BA
:10C83000A1679387E702631BF7041763FFFFE70213
:10C84000038901113285328497F0FFFFE780407839
:10C85000AA84228597F0FFFFE7808077854709E962
:10C86000228597F0FFFFE78080744205B337A00070
:10C8700028008145231891003ECA97000000E780F8
:10C88000209C05611763FFFF6700A386828097974E
:10C89000FF1F9387274B9C43D84799476313F7089B
:10C8A0001763FFFFE702A38279713285328497F024
:10C8B000FFFFE780C06F2AC6228597F0FFFFE78061
:10C8C00020712310A102228597F0FFFFE780206EE0
:10C8D0002301A102228597F0FFFFE780406DA301AD
:10C8E000A102228597F0FFFFE780606C2302A1027E
:10C8F000228597F0FFFFE780806B2313A10222853A
:10C9000097F0FFFFE780A06AB2452314A102280830
:10C9100097000000E780C09245611753FFFF670052
:10C92000437D82809797FF1F9387C7419C43D847D9
:10C93000A1679387C7036313F7081753FFFFE70245
:10C94000037979713285328497F0FFFFE7802066A2
:10C950002AC6228597F0FFFFE78080672310A10297
:10C96000228597F0FFFFE780A0662311A1022285B0
:10C9700097F0FFFFE780A0632302A102228597F0D2
:10C98000FFFFE780C062A302A102228597F0FFFFAC
:10C99000E780E0612303A102228597F0FFFFE78093
:10C9A0000061B245A303A102280897000000E780B8
:10C9B000208945611753FFFF6700A37382801753D7
:10C9C000FFFFE702C37001112A8497F0FFFFE780A1
:10C9D000005EAA84228597F0FFFFE780605F2285D2
:10C9E00097F0FFFFE780C05E035744008D4763F771
:10C9F000E700228597F0FFFFE780805D228597F0B2
:10CA0000FFFFE780E05C2800A68597000000E78034
:10CA1000208305611753FFFF6700A36D9797FF1FE2
:10CA2000938747329C43D847A167FD07631FF700F0
:10CA30001753FFFFE702A369328597000000E780E4
:10CA400040F81753FFFF6700C36A82809797FF1F64
:10CA50009387472F9C43D847A167E5076315F708DD
:10CA60001753FFFFE702A36679713285328497F08E
:10CA7000FFFFE780C0532AC6228597F0FFFFE780BB
:10CA80002055228597F0FFFFE78080542310A102F4
:10CA9000228597F0FFFFE780A053520551812311B3
:10CAA000A10222852302010297F0FFFFE7802050B8
:10CAB000A302A102228597F0FFFFE780404F2303E6
:10CAC000A102228597F0FFFFE780604EB245A303E5
:10CAD000A102280897F0FFFFE78080764561175391
:10CAE000FFFF6700036182809797FF1F9387872569
:10CAF0009C43D847A1679387E703631FF700175349
:10CB0000FFFFE702C35C328597000000E78060EB1F
:10CB10001753FFFF6700E35D82809797FF1F93879E
:10CB200067229C43D847A16793874704631EF70297
:10CB30001753FFFFE702A35979713285328497F0CA
:10CB4000FFFFE780C0462AC6228597F0FFFFE780F7
:10CB50002048B245280897F0FFFFE780606E4561E6
:10CB60001753FFFF6700E35882809797FF1F938753
:10CB7000671D9C43D847A167938787026310F7041A
:10CB80001753FFFFE702A35479713285328497F07F
:10CB9000FFFFE780C0412AC6228597F0FFFFE780AC
:10CBA0000041B2452300A102280897F0FFFFE7806B
:10CBB000206945611753FFFF6700A3538280175315
:10CBC000FFFFE702C350011197F0FFFFE780203E0F
:10CBD000AA85280097F0FFFFE7808066056117535C
:10CBE000FFFF670003519797FF1F9387A7159C438B
:10CBF000D847A167D107631FF7001753FFFFE7026C
:10CC0000034D328597000000E780A0FB1753FFFF1C
:10CC10006700234E82809797FF1F9387A7129C433C
:10CC2000D847A167C507631FF7001753FFFFE70247
:10CC3000034A328597000000E780A0F81753FFFFF2
:10CC40006700234B82809797FF1F9387A70F9C4312
:10CC5000D847A167B907631FF7001753FFFFE70223
:10CC60000347328597000000E780A0F51753FFFFC8
:10CC70006700234882809797FF1F9387A70C9C43E8
:10CC8000D847A167AD07631FF7001753FFFFE702FF
:10CC90000344328597000000E780A0F21753FFFF9E
:10CCA0006700234582809797FF1F9387A7099C43BE
:10CCB000D84789476318F7021753FFFFE70223415C
:10CCC0000111328532C897F0FFFFE780402EAA8518
:10CCD000280097F0FFFFE780A05605611753FFFF7C
:10CCE0006700234182809797FF1F9387A7059C4386
:10CCF000D847A1678D076311F7041753FFFFE702B9
:10CD0000033D01113285328497F0FFFFE780202A2E
:10CD100013066100AA844C00228597300000E7804A
:10CD2000C0232800A68597F0FFFFE78060510561CA
:10CD30001753FFFF6700E33B82809797FF1F93879E
:10CD4000A7009C4381CFDC4391CB1753FFFFE70241
:10CD5000033882971753FFFF6700A3398280175368
:10CD6000FFFFE702C33679713C08AE843ED2A1656D
:10CD7000B7070A002A843ED448103C08DD053ED699
:10CD800036C432C63AC297D0FFFFE780E02F124781
:10CD90004810BA8597F0FFFFE780C013324648106D
:10CDA000B28597F0FFFFE780E014A2464810B685F1
:10CDB00097F0FFFFE7800012501001478146A685DB
:10CDC000228597D0FFFFE780805145611753FFFF11
:10CDD000670023321753FFFFE702632F01117C0026
:10CDE0000329C501AE843ECAA165B70707002A849E
:10CDF0003ECC48087C00C5053ECE97D0FFFFE780BB
:10CE0000A0288345D900480897F0FFFFE780800CF1
:10CE1000500801478146A685228597D0FFFFE7800D
:10CE2000004C05611753FFFF6700A32C1753FFFF4A
:10CE3000E702E32983C7950093F7F707A384F5007A
:10CE400097000000E78040F91753FFFF6700632A4F
:10CE50001753FFFFE702A32779713C08AE843ED247
:10CE6000A165B70709002A843ED448103C08938581
:10CE700045043ED632C636C497D0FFFFE780C020B7
:10CE8000A2464810B68597F0FFFFE780A00432461F
:10CE90004810B28597F0FFFFE780C00550100147AA
:10CEA0008146A685228597D0FFFFE78040434561F4
:10CEB0001753FFFF6700E3231753FFFFE702232108
:10CEC00083C7950041112A8493F7F707A384F500DF
:10CED00032852EC697F0FFFFE780800F85672AC452
:10CEE0006370F50297700000E78020E92246B245A2
:10CEF00009ED11478146228597000000E78060E632
:10CF000041011753FFFF6700C31E01478346F50128
:10CF1000DDB71753FFFFE702E31901113C003ECADA
:10CF2000B7070A003ECC3C003ECE83C79500AA89D5
:10CF3000328593F7F707A384F5002E8497F0FFFF5F
:10CF4000E78000098567637DF504A165AA84938560
:10CF50008504480897D0FFFFE78000132685977067
:10CF60000000E78080E12A8929E19145480897F08F
:10CF7000FFFFE78020F6A685480897F0FFFFE780CF
:10CF800060F7CA85480897F0FFFFE780A0F40147E3
:10CF900081465008A2854E8597D0FFFFE780203458
:10CFA00005611753FFFF670023148145480897F078
:10CFB000FFFFE78020F20349090275BF1753FFFF07
:10CFC000E702430F79711C103ECAB7070F003ECC31
:10CFD000404D1C10AA84AE894808994532C636894E
:10CFE0003ECE97D0FFFFE780200A32464808B28540
:10CFF00097F0FFFFE78000EE630C0902A5454808A3
:10D0000097F0FFFFE780C0E62546CA85972001001C
:10D01000E78020A4500801478146CE85268597D019
:10D02000FFFFE780C02B45611753FFFF6700C30B6D
:10D030008355C402480897F0FFFFE780A0EB035533
:10D04000E402814505C5854785456301F502C16751
:10D05000FD179305F00F630BF5007D159770000029
:10D06000E780208E9305150093F5F50F480897F09B
:10D07000FFFFE78020E683450403480897F0FFFFA1
:10D08000E78040E583451403480897F0FFFFE780F9
:10D0900060E483552403480897F0FFFFE78080E5AC
:10D0A00083554403480897F0FFFFE780A0E49DB74D
:10D0B0001753FFFFE702A30183C79500814601468E
:10D0C00093F7F707A384F50097000000E78040EF8F
:10D0D0001753FFFF6700E3011753FFFFE70223FF2A
:10D0E00079713E841C103ECA2E89B7070F00A165D6
:10D0F0003ECCFD051C10AA84480842C03AC23ECE70
:10D1000036C432C697D0FFFFE78000F832464808A1
:10D11000B28597F0FFFFE780E0DBA2464808B685BE
:10D1200097F0FFFFE78000DD12474808BA8597F0C7
:10D13000FFFFE78020DC0248630C080291454808A5
:10D1400097F0FFFFE780C0D21146A285972001002B
:10D15000E7802090500801478146CA85268597D0F0
:10D16000FFFFE780C01745611753FFFF670063F8B3
:10D170008945480897F0FFFFE78080CF8347040088
:10D180002300F50083471400A300F500E1B717530F
:10D19000FFFFE70223F283C7950001112A8A93F764
:10D1A000F707A384F5003285AE8432C697F0FFFFFF
:10D1B000E78000E232462A89328597F0FFFFE78058
:10D1C00000DF85676373F902AA894A8597700000BA
:10D1D000E780A0BA2A8419ED114781464A86A685C0
:10D1E000528597000000E780C0B705611753FFFF25
:10D1F000670083EF9387E9FF93F7F70F0547E3662F
:10D20000F7FE8347F50195EB8947E380F9FE8346F6
:10D21000F401528501474A86A68597000000E78001
:10D2200040B4A167D90748083ECC230A010002CECA
:10D2300097000000E780A0B04DBF639EE7008947DC
:10D24000639EF90093071020231FF50097700000DC
:10D25000E780C0B76DBF0947E39BE7FA8D47E398C6
:10D26000F9FA228597700000E78080DF9797FF1F0B
:10D27000938787CC9C4399E79797FF1F938787B540
:10D280009C4399C703D5040097800000E780A0CE97
:10D29000231F040022855DBF1753FFFFE70223E32E
:10D2A00001113C003ECAB7070B003ECC3C003ECE0D
:10D2B00083C795002A89328593F7F707A384F50081
:10D2C000AE8497F0FFFFE780A0D093170501C187D8
:10D2D000635AF006A1652A849385E502480897D031
:10D2E000FFFFE78060DAA285480897F0FFFFE7803C
:10D2F00060C09797FF1F9387E7AD9C43A9EB01445C
:10D300009375F40F480897F0FFFFE780A0BC935592
:10D31000844093F5F50F480897F0FFFFE78080BB46
:10D320009355044193F5F50F480897F0FFFFE78008
:10D3300060BA014781465008A6854A8597D0FFFF0D
:10D34000E780E0F905611753FFFF670083DA416565
:10D3500085460546A2857D1597500000E78060BD93
:10D3600059DD510597000100E780808F13044006C6
:10D370003344850271B71753FFFFE70243D501110C
:10D38000B70706003EC683C7950021642A8993F734
:10D39000F707A384F500AE8428009305A4040AC40B
:10D3A0000AC897D0FFFFE78020CE300001478146B2
:10D3B000A6854A8597D0FFFFE78060F297E0FFFFE0
:10D3C000E780801513049404480822CC230A010046
:10D3D00002CE97000000E780809605611753FFFF9B
:10D3E000670023D11753FFFFE702C3CCC1642A892A
:10D3F00001449799FF1F9389A9B5130A8002FD1470
:10D4000097E0FFFFE78080C16347A4000145175301
:10D41000FFFF670063CDB307440303A7C90ABA97A8
:10D4200003D707006306970083D72700638427018B
:10D430000504F9B70545E1BF1753FFFFE70283C7AE
:10D440002A8A2E8999C123A0050081498144979A8F
:10D45000FF1F938AAA8F614B97E0FFFFE78040C2CE
:10D4600063C7A4004E851753FFFF6700E3C73384EB
:10D47000640383A70A003E948357040099E763047A
:10D480000900232089008504C1BF4146D2851305C8
:10D49000440097100100E780605975F5A289E5B74F
:10D4A0001753FFFFE70203C139717C083ED4B70769
:10D4B0000A003ED67C083ED883C795002A8A32856A
:10D4C00093F7F707A384F5002E8932C697F0FFFF84
:10D4D000E78000B085676373F5083246AA84328519
:10D4E00097F0FFFFE780A0AC8547AA8963E8A7060D
:10D4F000A16593858504281097D0FFFFE780C0B809
:10D50000268597700000E78040872A8429ED9145A1
:10D51000281097F0FFFFE780E09BA685281097F082
:10D52000FFFFE780209DCE85281097F0FFFFE78062
:10D53000609A014781463010CA85528597D0FFFF17
:10D54000E780E0D9A1679387770448183EDC230A77
:10D55000010202DE97F0FFFFE780607E2161175332
:10D56000FFFF670063B88145281097F0FFFFE78051
:10D570006096A685281097F0FFFFE780A097979701
:10D58000FF1F938767D39C4381CB22856389090062
:10D5900097D00000E78040248345040271B797D0FC
:10D5A0000000E780C022CDBF1753FFFFE70283B022
:10D5B00083C795004111AA8993F7F707A384F50063
:10D5C0003285AE84328A97F0FFFFE78060A08567DE
:10D5D000637FF5022A8997600000E780007A2A8439
:10D5E000914631C58347F50105476387E70291C737
:10D5F0000D476366F704AD461DA893050503032593
:10D600000A00414697100100E78040420DE94101C0
:10D610001753FFFF670043AD9305950803250A00E4
:10D62000414697100100E7806040814669F54A86CF
:10D63000A6854E8597000000E780C081C9BF83257D
:10D640000A001305940897700000E780A02919C10B
:10D65000C146F1BF9797FF1F9387078E9C4399E7B9
:10D660009787FF1F938707779C4399C722859780E9
:10D670000000E780208A69FD8547A30FF40022851A
:10D6800097B00000E7806084228597600000E78003
:10D69000E0734E8581464A86A68597F0FFFFE780B6
:10D6A000607BA1679387570448003EC423020100B2
:10D6B00002C697F0FFFFE780806891BF1753FFFF16
:10D6C000E702639E83C795004111AA8993F7F70784
:10D6D000A384F50032852E89B28A97F0FFFFE78098
:10D6E000208F85676374F50EAA8497600000E78039
:10D6F000C0682A840DED416B014A979BFF1F938BF5
:10D700002B85130C400E7D1B19A833048A0383A7B5
:10D710000B0B3E948357C40163836705050A97E0AA
:10D72000FFFFE780A08EE342AAFE95460DA0835737
:10D73000C501639697029305050303A50A004146B8
:10D7400097100100E780802E994611E181462686D8
:10D75000CA854E8597F0FFFFE780C06F85A883A537
:10D760000A001305040397700000E780A017C14664
:10D7700079FD2285231E940097A00000E780E074C5
:10D78000228597600000E78060649797FF1F93876A
:10D79000A7B29C43A9C323000402228597D00000AE
:10D7A000E78040F04E8581462686CA8597F0FFFFC8
:10D7B000E780406AA1679387070448003EC42302BC
:10D7C000010002C697F0FFFFE78060574101175341
:10D7D000FFFF6700C39089472300F402E1B7397166
:10D7E00006DE22DC4AD8800052D456D25AD026DA3D
:10D7F0004ED65ECE2E8A32892A8B97D0FFFFE780E5
:10D80000E07D0605710541998A8A3301A1402322F2
:10D8100024FC231404FC97D0FFFFE780207C83477F
:10D820009A000605350593F7F7072315A4FCA30412
:10D83000FA004A85232624FC97E0FFFFE780407921
:10D8400093170501C1876340F0025681130104FC60
:10D85000F2506254D2544259B259225A925A025B3F
:10D86000F24B21618280AA844A8597E0FFFFE7801E
:10D870002076AA894A8597E0FFFFE7806075A16559
:10D880009385C5022A89130544FC97C0FFFFE780F2
:10D89000A07F268597C0FFFFE780E073854511C90B
:10D8A0004A86CE8597C0FFFFE780606DAA8B21E98D
:10D8B0008945130544FC97E0FFFFE780A061A6853A
:10D8C000130544FC97E0FFFFE780C062CE85130597
:10D8D00044FC97E0FFFFE780E061CA85130544FC44
:10D8E00097E0FFFFE780006101478146130644FC93
:10D8F000D2855A8597D0FFFFE780609EB9B78145F2
:10D90000130544FC97E0FFFFE780C05CA685130584
:10D9100044FC97E0FFFFE780E05DCE85130544FC03
:10D9200097E0FFFFE780005DCA85130544FC97E0A0
:10D93000FFFFE780205C814497D0FFFFE780006A0B
:10D94000E3D4A4FA83A70B0113971400BA9783D5E5
:10D95000070099C5130544FC97E0FFFFE780805955
:10D960008504D9BF797106D622D44AD000184ECE8C
:10D9700052CC56CA26D25AC8AE893289AA8A97D0C2
:10D98000FFFFE780A0650605690541990A8A330112
:10D99000A140232A24FC231C04FC97D0FFFFE7802E
:10D9A000E06383C7990006052D0593F7F707231D4C
:10D9B000A4FCA384F9004A85232E24FC97E0FFFFF2
:10D9C000E780006193170501C187634FF000528122
:10D9D000130104FDB250225492540259F249624A92
:10D9E000D24A424B45618280AA844A8597E0FFFF74
:10D9F000E780005EA1659385A5022A89130544FD91
:10DA000097C0FFFFE7804068268597C0FFFFE7804B
:10DA1000805C854509C9CA8597C0FFFFE78020590A
:10DA20002A8B29E18945130544FD97E0FFFFE78034
:10DA3000604AA685130544FD97E0FFFFE780804B11
:10DA4000CA85130544FD97E0FFFFE780A04A014720
:10DA50008146130644FDCE85568597D0FFFFE780AB
:10DA60000088B5B78145130544FD97E0FFFFE780C7
:10DA70006046A685130544FD97E0FFFFE7808047D9
:10DA8000CA85130544FD97E0FFFFE780A046814467
:10DA900097D0FFFFE7808054E3DBA4FA83270B01D4
:10DAA00013971400BA9783D5070099C5130544FD51
:10DAB00097E0FFFFE78000448504D9BF1743FFFFCD
:10DAC000E702E36083474500404DD5EFFD575DC455
:10DAD0008346940009476363D70A0346B40085462A
:10DAE00063EEC6088306E40063CA06085C45F9567F
:10DAF0002390D7009787FF1F83C7872599E3A30447
:10DB0000E4009787FF1F9387E72C9C4381E78947B1
:10DB1000A306F4009787FF1F9387077A9C4381E74A
:10DB200089472306F4009705000093854506AA84DB
:10DB30001305040197F00000E7802010FD57231A19
:10DB4000F40281471CDC01489787FF1F23AE871E24
:10DB50009787FF1F9387871F232E040304C08043EA
:10DB600097D0FFFFE780C05161463306C50281456B
:10DB700022859740FFFFE780805881473E85174305
:10DB8000FFFF67000357FD57D5BF1743FFFFE702AD
:10DB900003542A840355450297600000E780E01D86
:10DBA00019E5231E04001743FFFF670083548357C2
:10DBB000E401F5DB930504FF174501001305453526
:10DBC00097E00000E780E014F9BF1743FFFFE7028A
:10DBD00003502E89A16541119385E5032A8436C43B
:10DBE00032C6BE843AC297C0FFFFE780E0491247C1
:10DBF0002285BA8597E0FFFFE780C02D3246228557
:10DC0000B28597E0FFFFE780E02EA2462285B68529
:10DC100097E0FFFFE780002E63030902914522850C
:10DC200097E0FFFFE780C0241146A685971001000A
:10DC3000E78020E241011743FFFF6700834B8945DE
:10DC4000228597E0FFFFE780A02283C7040023001E
:10DC5000F50083C71400A300F500E9BF1743FFFFD9
:10DC6000E702E34683C79500444D054793F7F7075E
:10DC7000A384F5001C42411183C707006367F706C0
:10DC80002E842A89B1C003C7D400630FF702178717
:10DC9000FF1F13072714184305C3A386F40097A09A
:10DCA0000000E780404A83C7D40099E741657D15AD
:10DCB00097400000E780403083D72403918B89C7C9
:10DCC00097E00000E780C0134A85A28597F0FFFF28
:10DCD000E7808010A167C10748003EC4230201000D
:10DCE00002C697F0FFFFE780800541011743FFFF61
:10DCF000670023401743FFFFE702633D03D745005A
:10DD00008D47AA8441112E8432892E8563E3E70270
:10DD100097E0FFFFE780C02BAA8523000900268536
:10DD200097C0FFFFE780A02841011743FFFF67006E
:10DD3000433C97E0FFFFE780A0292AC6228597E0B1
:10DD4000FFFFE780E028B24585472A862300F900D7
:10DD5000268597C0FFFFE7808022F9B7397106DE7C
:10DD600022DC26DA80004ED652D456D24AD85AD077
:10DD70005ECEAE89B284AA8A97D0FFFFE7800025E5
:10DD800006051305250241990A8A3301A140232281
:10DD900024FC231404FC97D0FFFFE780202383C7D3
:10DDA000990006054D0593F7F7072315A4FCA384F6
:10DDB000F9002685232624FC97E0FFFFE780402119
:10DDC00093170501C1876340F0025281130104FCDF
:10DDD000F2506254D2544259B259225A925A025BBA
:10DDE000F24B21618280AA8B03AB040097C0FFFF36
:10DDF000E780601E51E583D7440001498544F1174F
:10DE000093B71700A301F4FC834734FCA165C9C78D
:10DE10009385E504130544FC97C0FFFFE780C02607
:10DE2000A685130544FC97E0FFFFE780A00ADE8586
:10DE3000130544FC97E0FFFFE780C00B834734FCE9
:10DE4000114691E30946DA85130544FC97E0FFFF8C
:10DE5000E78060058144630A0900416B7D1B97D010
:10DE6000FFFFE780A01663CCA4020147814613069A
:10DE700044FCCE85568597C0FFFFE7804046B1B78A
:10DE8000A685130634FC97000000E780E0E6933493
:10DE900015002A8986048DBF9385C504A5BF8327F5
:10DEA000C90013971400BA9783D5070063886501EA
:10DEB000130544FC97E0FFFFE780C003850445B7E6
:10DEC0001743FFFFE702231E79711C103EC4B707FA
:10DED0000F003EC61C103EC883C79500AA8A328533
:10DEE00093F7F707A384F500AE89328497E0FFFF2C
:10DEF000E780000E93170501C187635AF0062A8A4E
:10DF0000228597E0FFFFE780A00C2A895285032B2A
:10DF1000040097C0FFFFE780000C39ED83574400F1
:10DF200081440544F11793B71700A303F10083451B
:10DF30007100DA872287CA8652862800970000007F
:10DF4000E780E0C8014781463000CE85568597C0FE
:10DF5000FFFFE780C038A1679387D70348083ECC0E
:10DF6000230A810026CE97F0FFFFE78040DD456160
:10DF70001743FFFF6700A316A285130671009700E1
:10DF80000000E78060D7AA84094455D13544E300F6
:10DF900055FB4A8597F0FFFFE78000450D4441D9C6
:10DFA000014497D0FFFFE7806002634DA400C16B7E
:10DFB0000144FD1B97D0FFFFE7804001634EA400A2
:10DFC0001544B5B7DC4413171400BA9783D707007C
:10DFD000638327030504F1B7D84493171400BA9755
:10DFE00003D70700631B770123902701268597A09D
:10DFF0000000E78080DB01441DBF050465BF1743B7
:10E00000FFFFE702230B83C7950041112A8A93F78C
:10E01000F707A384F50032852E89328497E0FFFF4D
:10E02000E78000FB93170501C1876353F006AA89B7
:10E03000228597E0FFFFE780A0F92311A1004E851C
:10E04000832A040097C0FFFFE780E0F839E5835793
:10E05000440085440144F11793B71700A300F10071
:10E060000348110003572100D6875285CE862686A5
:10E07000CA8597F0FFFFE7806006A167F1074800B7
:10E080003EC42302910022C697F0FFFFE78020CB19
:10E0900041011743FFFF67002305A2851306110006
:10E0A00097000000E78040C52A84894455D98357EA
:10E0B000210011678544BA97C2071167C18313070E
:10E0C000F7EFE36FF7F89787FF1F9387E7E69C4327
:10E0D00081CB85451305210097500000E78020750E
:10E0E000835521002285814497C0FFFFE78040E5EA
:10E0F00025D923100500228597A00000E78040CD98
:10E1000085B71743FFFFE70203FA83C79500411164
:10E110002A8B93F7F707A384F50032852E8A328481
:10E1200097E0FFFFE780C0EA93170501C1876351BD
:10E13000F006AA8A228597E0FFFFE78060E92A8936
:10E140005685832B040097C0FFFFE780C0E831E5C8
:10E150008357440081440544F11793B71700A30186
:10E16000F10003483100DE875A854A87D686228629
:10E17000D28597F0FFFFE78060F6A167ED074800C2
:10E180003EC42302810026C697F0FFFFE78020BB34
:10E1900041011743FFFF670083F4A2851306310096
:10E1A00097000000E78040B5AA8409445DD99167D3
:10E1B000CA97C2071167C1831307F7EF0544E362EB
:10E1C000F7FACA8597C0FFFFE78080D7014451F96D
:10E1D000814997D0FFFFE78060E063DBA9009848A2
:10E1E00093971900BA9703D7070005EF23902701EB
:10E1F00097D0FFFFE78080DE1544E384A9F62685EB
:10E2000097A00000E780C0BC9787FF1F9387C7D205
:10E210009C430144B9D74A8597500000E780C05815
:10E2200089B785097DB71743FFFFE702A3E8797136
:10E230003E847C083EC82E8AB7071400A1653ECAFA
:10E24000E5057C08AA89080836C4428932C6BA8A1C
:10E25000C6843ECC97C0FFFFE78000E3CA8508086C
:10E2600097E0FFFFE78000C732460808B28597E0D5
:10E27000FFFFE78020C8A246630A09049D450808FD
:10E2800097E0FFFFE780C0BE1D4681459740FFFF36
:10E29000E780E0E663890A089145080897E0FFFFF8
:10E2A000E78000BD1146A68597000100E780607AEF
:10E2B000100801478146D2854E8597C0FFFFE78051
:10E2C000000245611743FFFF670003E2B6850808B7
:10E2D00097E0FFFFE78000C21C400808D843935531
:10E2E000C701858912075183B205D98D97E0FFFFD9
:10E2F000E78040C01C40080883C5870097E0FFFF07
:10E30000E78040BD1C40080883C5A70097E0FFFFD9
:10E31000E78040BC1C40080883C5970097E0FFFFDA
:10E32000E78040BB85BF8945080897E0FFFFE7808D
:10E3300020B483C704002300F50083C71400A300A2
:10E34000F500BDB71743FFFFE702C3D683C79500AB
:10E350004111AA8993F7F707A384F5003285AE84AB
:10E36000328497E0FFFFE780A0C693170501C187BD
:10E37000635DF0042A89032A040097C0FFFFE78049
:10E3800080C519E9835744000548F11793B7170072
:10E39000A307F100814631A81306F100A28597007A
:10E3A0000000E78060951DC51C459DC783D64700CA
:10E3B00001480347F10093078500D2884A86A68565
:10E3C0004E8597000000E78040E641011743FFFFBC
:10E3D000670083D109487DBF1D486DBF1743FFFF0C
:10E3E000E70243CD65715C083EC4B7077B013EC6BA
:10E3F0005C083EC883C795002A8A328593F7F707E1
:10E40000A384F500AE8997E0FFFFE78040BA835709
:10E41000E100E1C78945280097C0FFFFE780C0C63B
:10E420008145280097E0FFFFE780C0AA97C0FFFF63
:10E43000E780A0CC9787FF1F938707E89C4317844A
:10E44000FF1F0344E490AA843334800099C313640B
:10E4500024009787FF1F9387E7979C4399C3136412
:10E4600044009787FF1F938727AD9C4399C313648C
:10E47000840083D504002800014997E0FFFFE7806E
:10E4800060A783D52400280097E0FFFFE78080A6DF
:10E4900083D54400280097E0FFFFE780A0A597D030
:10E4A000FFFFE780A0AE93150501C181280097E02A
:10E4B000FFFFE78020A4A285280097E0FFFFE78008
:10E4C00060A39C446360F902014781463000CE8519
:10E4D000528597C0FFFFE78080E059611743FFFF37
:10E4E000670083C0DC441314490028003E9497E081
:10E4F000FFFFE78060968347440003475400890785
:10E500000607BA978607E36AF5FC835524002800BE
:10E51000814A97E0FFFFE780E09D834544002800A3
:10E5200097E0FFFFE780009B83455400280097E0B9
:10E53000FFFFE780209A8347440063C9FA00814ABD
:10E540008347540063C1FA020509A5BF1C44139711
:10E550005A002800BA9783D50700850A97E0FFFF85
:10E56000E7804099C9BF032BC40093975A00280045
:10E570003E9B83552B00850A97E0FFFFE78080973D
:10E5800083550B00280097E0FFFFE780A0964DBF62
:10E590001743FFFFE702A3B35C4993E717005CC989
:10E5A00097A00000E78020B61743FFFF670063B421
:10E5B0001743FFFFE702A3B12E84814597F0FFFFC9
:10E5C000E780C0E705C583570500FD172310F50058
:10E5D00009C4835725002310F40097000000E7804A
:10E5E00060FB01451743FFFF6700A3B031457DD8AD
:10E5F00023100400C5BF1743FFFFE702A3AB83C787
:10E60000950041112A8A93F7F707A384F500328514
:10E610002E89328497E0FFFFE780809B93170501E6
:10E62000C1876356F006AA89C145228597E0FFFF9E
:10E63000E780A0802A8B4E85832A040097C0FFFFC5
:10E64000E780609931E983574400231101000544B4
:10E65000F11793B71700A300F1008144034811009C
:10E6600003572100D6875285CE862286CA8597F029
:10E67000FFFFE780A0A6A1679387170248003EC46A
:10E680002302810026C697E0FFFFE780406B41012F
:10E690001743FFFF670043A513061100A28597F0FB
:10E6A000FFFFE7806065AA8409E5231101000944A2
:10E6B00075B7930521005A8597000000E78080EF29
:10E6C000835721002A84D9DB9787FF1F9387C7864A
:10E6D0009C4381CB85451305210097500000E780BE
:10E6E0000015835521002685314497C0FFFFE78040
:10E6F00020852DD523100500268597900000E78002
:10E70000206D0144A1BF1743FFFFE702439C411165
:10E710002E896C00AA8402C697F0FFFFE78000D222
:10E720000DC10357050005072310E5009700000001
:10E73000E78040E681473E8541011743FFFF6700C0
:10E74000439B3247954765DBCA8526859730000095
:10E75000E780400DC147E34005FE3244854741460E
:10E760002310F40083570900A685130544002311E4
:10E77000F40097000100E780C02D228545BF1743B4
:10E78000FFFFE702239383C795004111AA8A93F7FD
:10E79000F707A384F5003285AE89328497E0FFFF46
:10E7A000E780008393170501C1876356F0062A8A24
:10E7B000C145228597D0FFFFE7802068AA84528553
:10E7C000032B040097C0FFFFE780E08031E9835707
:10E7D0004400231101008544F11793B71700A300EB
:10E7E000F10001440348110003572100DA875685E0
:10E7F000D2862686CE8597F0FFFFE780208EA16720
:10E800009387070248003EC42302910022C697E086
:10E81000FFFFE780C05241011743FFFF6700C38C31
:10E82000A2851306110097F0FFFFE780E04C2A84D1
:10E8300009E523110100894475B726859305210058
:10E8400097000000E78060ECAA8449FD8355210011
:10E85000228597B0FFFFE780A06E49F5014997C078
:10E86000FFFFE780A077635DA900184893171900A0
:10E87000BA9703D707000DEF035721002390E70055
:10E8800097C0FFFFE7808075630625039777FF1F1A
:10E890009387876A9C4399C70355210097500000CE
:10E8A000E78080F0228597900000E78060521DBFCE
:10E8B000050975B795443DB705C19307F00F630F80
:10E8C000F500C547630CF5009307F5FF05453315C3
:10E8D000F5004205418182800145828041657D15B8
:10E8E0008280B9E91733FFFFE702637E0345060321
:10E8F000328497000000E78060FC9305803EB305FA
:10E90000B502C205C18181CD0357E402854763F892
:10E91000E7001305040197E00000E78020428357D9
:10E92000E40241677D176385E700FD172317F402B2
:10E930001733FFFF6700E37B82801733FFFFE70297
:10E940008376004283C79500444D0349140093F732
:10E95000F707A384F5008347040022091167336990
:10E96000F900A167B347F90041112A8BAE8A63EC25
:10E97000E70E834724001307C00EB91793F7F70F6C
:10E980006373F71003473400C14763EEE70E834714
:10E9900044001307E00793C707086371F70C834926
:10E9A000840083477400A209B3E9F900856763F71F
:10E9B000F90A034A6400834754004E85220A336AE9
:10E9C000FA0097500000E780403B61C12396240382
:10E9D000834B3400137AFA00239A34032388740398
:10E9E0002399440393890401631C090023A60402AC
:10E9F000239804024E8597E00000E78060363DA032
:10EA0000034924004A8597000000E78020EB239704
:10EA1000A402834744004E85A388F402E38D0BFCD7
:10EA2000E30B09FC97E00000E780202F979000009F
:10EA3000E780007381460146D6855A8597E0FFFF3F
:10EA4000E7800058A167938797033EC42302010023
:10EA5000480002C697E0FFFFE780602E41011733B0
:10EA6000FFFF6700C3678544A2862686D6855A8540
:10EA700097E0FFFFE780C054A167938797033EC4E8
:10EA800023029100F1B7BD44C5B79144F1BF1733DC
:10EA9000FFFFE702236201111C08404D3EC2B70789
:10EAA0000F003EC41C083EC62A89AE8997C0FFFFEE
:10EAB000E780A0DA585C1C5C6346B70E6394E500FF
:10EAC00063E2A70E3385A740B3B7A700B305B740ED
:10EAD0001306803E81469D8D97000100E78080B738
:10EAE00093140501C180A1659385C503480097B0C3
:10EAF000FFFFE78060598145480097D0FFFFE7801E
:10EB0000603D83550404480097D0FFFFE780803EB6
:10EB100083552404480097D0FFFFE780A03D81453E
:10EB200089CCC167FD179305F00F6388F400268533
:10EB300097500000E780E0E0AA85480097D0FFFFEB
:10EB4000E780403903554404814501CDC167FD1775
:10EB50009305F00F6307F50097500000E78060DE33
:10EB6000AA85480097D0FFFFE780C036834564043C
:10EB7000480097D0FFFFE780E035834574044800E4
:10EB800097D0FFFFE7800035500001478146CE85D2
:10EB90004A8597B0FFFFE780807405611733FFFF58
:10EBA00067008354814481B71733FFFFE702235284
:10EBB00083C7950093F7F707A384F500970000003B
:10EBC000E78020ED1733FFFF6700A3521733FFFFE5
:10EBD000E702434E83C795004111404D93F7F70775
:10EBE000A384F5002A8A3285B284AE8997D0FFFFCC
:10EBF000E780003E2A8B268597D0FFFFE780403DC7
:10EC00002A89268597D0FFFFE780603A93170B018A
:10EC100063CA0702E177CA97C207C183116763E33A
:10EC2000E70293070910C207C1831307B00F637B84
:10EC3000F70093170901C187AA8A634AF000C54704
:10EC400063FE570141011733FFFF6700E34997B0A7
:10EC5000FFFFE780C028E31725FFD5B763080B0245
:10EC600063060902814463890A02B7077F00231003
:10EC70006405231124057CC0568597000000E780B9
:10EC8000E0C39304803EB304950239A0B7077F0028
:10EC9000232004047CC081440355240497E0000031
:10ECA000E780A0A3A1C497C0FFFFE78000BB269523
:10ECB00093D7F44133379500AE97BA9708DC5CDC04
:10ECC000CE85528597000000E780A0DC99E02322E2
:10ECD0000404A1679387B70348003EC423020100E0
:10ECE00002C697E0FFFFE7808005A9BF8147014882
:10ECF0001CDC232E0403E9B71733FFFFE702233D93
:10ED000097C0FFFFE780C037E1473305F502914523
:10ED100097500000E78000C5E55711C59777FF1FA2
:10ED200023A6A70281473E851733FFFF6700633C98
:10ED300085471777FF1F230DF70082801733FFFFEA
:10ED4000E702E3389777FF1F9387070080433DC0B2
:10ED5000835704046390A70683572404639CB70475
:10ED60003689B28497C0FFFFE78020AF5C5C63C345
:10ED7000B7046395B7001C5C63EEA7028347640485
:10ED800063F3F400A6872303F4048347740463F356
:10ED90009700A687A303F4048357440441677D17B3
:10EDA0006385E70085072312F4043C4481C7CA85C4
:10EDB000268582971733FFFF6700A3339777FF1FDE
:10EDC000938787F89C43014599C303C587008280D8
:10EDD0001733FFFFE702A32F0111B70707003EC655
:10EDE00083C79500584D0AC493F7F7070AC8A38450
:10EDF000F5002A89AE8411CB1C4283C70700230487
:10EE0000F70097900000E7800034216493055402D6
:10EE1000280097B0FFFFE780202797000000E780D9
:10EE200020FAAA85280097D0FFFFE780A00A3000CB
:10EE300001478146A6854A8597B0FFFFE780204AB3
:10EE400013044402480822CC230A010002CE97E0B2
:10EE5000FFFFE780C0EE05611733FFFF67006329FE
:10EE60001733FFFFE702A32601117C003ECAB70754
:10EE700007003ECC7C003ECE83C795002E84AA843A
:10EE800093F7F707A384F500A16593855502480819
:10EE900097B0FFFFE780401F97000000E78040F237
:10EEA000AA85480897D0FFFFE780C00250080147B5
:10EEB0008146A285268597B0FFFFE7804042056125
:10EEC0001733FFFF6700E3229777FF1F9387C7E79A
:10EED0009C43094599C303C5970082809777FF1F1C
:10EEE000938787E69C43094599C303C5D700828071
:10EEF0009777FF1F938747E59C43014599C303C557
:10EF0000A70082801733FFFFE702C31A0111B7077A
:10EF100008003EC683C79500404D0AC493F7F70723
:10EF20000AC8A384F5002A89AE8429C414428547FF
:10EF300003C7060063E0E70A834794000946814956
:10EF40006380C702B307F740A304E400B339F000BD
:10EF500083C716002305F40097900000E780A01EE9
:10EF600003572403058B19C76386090097D0000057
:10EF7000E78000E9216493058402280097B0FFFF31
:10EF8000E780801097000000E78040F4AA85280001
:10EF900097D0FFFFE78000F497000000E78080F53E
:10EFA000AA85280097D0FFFFE780C0F2014781467D
:10EFB0003000A6854A8597B0FFFFE78040321304F2
:10EFC0007402480822CC230A010002CE97E0FFFF1A
:10EFD000E780E0D605611733FFFF6700E3101733C2
:10EFE000FFFFE702C30E01117C003ECAB70708000D
:10EFF0003ECC7C003ECE83C795002E84AA8493F736
:10F00000F707A384F500A16593858502480897B0AA
:10F01000FFFFE780600797000000E78020EBAA85EC
:10F02000480897D0FFFFE780E0EA97000000E780FC
:10F0300060ECAA85480897D0FFFFE780A0E9500858
:10F0400001478146A285268597B0FFFFE7802029EA
:10F0500005611733FFFF6700C3099777FF1F938789
:10F06000A7CE9C43014599C303C5B70082801733DF
:10F07000FFFFE702C3050111B70707003EC683C7BC
:10F080009500404D0AC493F7F7070AC8A384F5001A
:10F090002A89AE8405C81C42054783C707006368F8
:10F0A000F7060347B400630FF700A305F400979039
:10F0B0000000E78040098347B400B9CF97D0FFFF35
:10F0C000E78040BE21649305B400280097B0FFFF9D
:10F0D000E78080FB97000000E78060F8AA852800A1
:10F0E00097D0FFFFE78000DF014781463000A6850B
:10F0F0004A8597B0FFFFE780801E2904480822CC8C
:10F10000230A010002CE97E0FFFFE78040C30561BC
:10F110001733FFFF6700E3FD97D0FFFFE78020BFB5
:10F1200055B71733FFFFE70283FA01117C003ECA8F
:10F13000B70707003ECC7C003ECE83C795002E84E7
:10F14000AA8493F7F707A384F500A165AD054808E5
:10F1500097B0FFFFE78040F397000000E78020F0C2
:10F16000AA85480897D0FFFFE780C0D6500801471E
:10F170008146A285268597B0FFFFE780401605618E
:10F180001733FFFF6700E3F69777FF1F9387C7BB2F
:10F190009C43094599C303C5C70082801733FFFF0D
:10F1A000E702E3F201117C00AE843ECAA165B70715
:10F1B00007002A843ECCD1057C0048083ECE97B09B
:10F1C000FFFFE78060EC97000000E78020FCAA8545
:10F1D000480897D0FFFFE780E0CF500801478146FD
:10F1E000A685228597B0FFFFE780600F0561173382
:10F1F000FFFF670003F01733FFFFE70243ED83C70C
:10F20000950093F7F707A384F50097000000E780C7
:10F2100020F91733FFFF6700C3ED1733FFFFE70245
:10F2200063E983C795000329C501411193F7F707E7
:10F23000A384F5001C4283C90700854763E63707AE
:10F240009777FF1F938747079C432E84AA8485CF17
:10F2500097000000E78080F389476306F5026304A6
:10F2600009028347C9006380370323063901979059
:10F270000000E78040ED83572903898B89C797D029
:10F280000000E780E0B72685A28597000000E780B0
:10F2900020F1A167CD0748003EC42302010002C649
:10F2A00097E0FFFFE780A0A941011733FFFF670048
:10F2B000A3E39777FF1F938727A99C431D4599C315
:10F2C00003C5E70082801733FFFFE70243E0011127
:10F2D000B70707003EC683C79500584D0AC493F789
:10F2E000F7070AC8A384F5002A89AE8415C71C4213
:10F2F00083C7070093968701E18663C406068546A7
:10F300006381D7068346E7006388F6002307F7008A
:10F3100097900000E78020E321649305E400280033
:10F3200097B0FFFFE78040D697000000E780A0F885
:10F33000AA85280097D0FFFFE780C0B90147814622
:10F340003000A6854A8597B0FFFFE78040F9350475
:10F35000480822CC230A010002CE97E0FFFFE78095
:10F36000009E05611733FFFF6700A3D81733FFFF27
:10F37000E702E3D501117C003ECAB70707003ECC87
:10F380007C003ECE83C795002E84AA8493F7F707AE
:10F39000A384F500A165B905480897B0FFFFE78091
:10F3A000A0CE97000000E78000F1AA85480897D01A
:10F3B000FFFFE78020B2500801478146A2852685DD
:10F3C00097B0FFFFE780A0F105611733FFFF6700EB
:10F3D00043D21733FFFFE702E3CDAA840144177934
:10F3E000FF1F1309A996E14997C0FFFFE78040C9B5
:10F3F0006344A400014519A8330534038327090099
:10F400003E95835725006397970011051733FFFF3B
:10F41000670083CD0504C9BF032E8500630A0E1261
:10F420001773FF1F130343B1032303006315030086
:10F4300029436390061203234E01631503001D4305
:10F44000639907101733FFFFE702E3C5C689428AB5
:10F450003E89BA8AB684328BAE8B2A84B5E10355D5
:10F460004E0019E501431A851733FFFF670023C7D4
:10F47000A167A98F116763FBE70097000000E78091
:10F4800080F5814597F0FFFFE780C0120844B70779
:10F4900000E05841F98F18455CC1B707001FF98F8C
:10F4A0001CC55C4991C7610597E00000E780408B6F
:10F4B000E38A09FA228597900000E78060C65DB76D
:10F4C000328597C00000E78040430D4349DD1C446E
:10F4D000116703D54700A167A98F63FBE700970079
:10F4E0000000E78040EF814597F0FFFFE780800C48
:10F4F0000323840093164B01D1828347B300035644
:10F5000063008588FD8BA305F300FD777D8E558E06
:10F51000FD76FD16B204F18E83274301C58E2312BA
:10F5200073012313D3002304530123052301A304F0
:10F530004301BDDF228597B0FFFFE78020CDAA857C
:10F540000844B5D1610597D00000E780207F8DB7D2
:10F550001D431A8582801733FFFFE702A3B50569B3
:10F56000AA84AE89328A0144FD5A7D1997C0FFFFF3
:10F57000E780C0A56347A40001451733FFFF67007C
:10F58000A3B6D84493171400BA9703D70700631F94
:10F5900037032390570163070A00268597900000E0
:10F5A000E780A0809C449DC383D76700B3F7270101
:10F5B000639E3701D2880148814701478146014651
:10F5C0008145268597000000E78040E5050479BF66
:10F5D0001733FFFFE70203AE79711C103EC4B70773
:10F5E0000F003EC61C103EC883C79500AA8A32850C
:10F5F00093F7F707A384F5002E89328497D0FFFF95
:10F60000E780009D93170501C187635AF006AA8918
:10F61000228597D0FFFFE780A09B2A8A4E85032B87
:10F62000040097B0FFFFE780009B39ED835744004B
:10F6300081440544F11793B71700A303F1008345F4
:10F640007100DA872287D2864E86280097E0FFFF76
:10F65000E780E057014781463000CA85568597B05C
:10F66000FFFFE780C0C7A1679387F70348083ECC38
:10F67000230A810026CE97D0FFFFE780406C4561CA
:10F680001733FFFF670043A6A2851306710097E0BA
:10F69000FFFFE7806066AA84094455D1528597E050
:10F6A000FFFFE78060D40D4459D90546D2852685F1
:10F6B00097000000E78060EA2A8451B71733FFFF04
:10F6C000E702E3A0835507000346270041112A847F
:10F6D0002E8532C62EC497E0FFFFE780E0D001C937
:10F6E0003246A245228597000000E78000E74101ED
:10F6F0001733FFFF6700E39F1733FFFFE702A39A6B
:10F7000083C795004111AA8A93F7F707A384F500F0
:10F710003285AE89328497D0FFFFE780608B9317E4
:10F720000501C1876357F00AC1452A8A228597C01F
:10F73000FFFFE78080702A8D228597D0FFFFE7804A
:10F7400020892A89228597D0FFFFE780408693078A
:10F7500005F893F7F70F1307E007AA8B637BF7060B
:10F76000228597D0FFFFE78080842A8C228597D05E
:10F77000FFFFE780C083AA8C5285032B040097B05B
:10F78000FFFFE780408539E98357440023110100DA
:10F790008144F11793B71700A300F1000544034714
:10F7A000110083562100938784005685DA882288C9
:10F7B0005286CE8597F0FFFFE78020A7A167E90773
:10F7C00048003EC42302810026C697D0FFFFE78091
:10F7D000005741011733FFFF6700639013061100C4
:10F7E000A28597E0FFFFE7802051AA8409E5231155
:10F7F000010009446DB7930521006A8597F0FFFF6A
:10F80000E780A0F02A8441FD835521009356C9006A
:10F810001316490185486688E2875E87858A51828A
:10F82000268597000000E78060BF2A848DBF1733CC
:10F83000FFFFE702438783C7950041112A8B93F7A7
:10F84000F707A384F5003285AE89328497C0FFFFA5
:10F85000E780007893170501C1876352F00A2A8A6E
:10F86000228597C0FFFFE780A076AA8A228597C0ED
:10F87000FFFFE780E0752A89228597C0FFFFE780B8
:10F880000073930705F893F7F70F1307E0072A8C27
:10F890006377F706228597C0FFFFE7804071AA8C47
:10F8A000228597C0FFFFE78080702A8D5285832BC9
:10F8B000040097A0FFFFE780007239E583574400FA
:10F8C00085440144F11793B71700A301F1000347E2
:10F8D0003100930784005A85DE882688D6865286B2
:10F8E000CE8597F0FFFFE78040948D4748003EC4E7
:10F8F0002302910022C697D0FFFFE78040444101D8
:10F900001723FFFF6700A37DA2851306310097E050
:10F91000FFFFE780603E2A84894455D99356C90089
:10F920001316490185486A88E6876287858A51826D
:10F93000D68597000000E78060AEAA8449BF1723F0
:10F94000FFFFE70223772A8981440144617A916AA3
:10F95000176BFF1F130B4B5E97B0FFFFE78000682C
:10F9600063C7A40022851723FFFF6700E37783277F
:10F97000090093991400CE9703D50700330745017A
:10F98000420741836364570305C103270B0019C76E
:10F9900085453E8597400000E78060E983270900A0
:10F9A0000504CE972390070085047DB797000000DB
:10F9B000E78060A2832709000504CE972390070003
:10F9C00065D5814597F0FFFFE780C0BEF1BF1723E3
:10F9D000FFFFE702236E83C7950041112A8A93F740
:10F9E000F707A384F50032852E89328497C0FFFF84
:10F9F000E780005E93170501C187635AF004AA8966
:10FA0000832A040097A0FFFFE780E05C31E583577D
:10FA1000440085440144F11793B71700A301F10096
:10FA200003483100D68752850147CE862686CA858F
:10FA300097D0FFFFE780806AA167F50748003EC4C2
:10FA40002302910022C697D0FFFFE780402F41019B
:10FA50001723FFFF67004369A2851306310097E073
:10FA6000FFFFE78060292A8489445DD99767FF1FDB
:10FA70009387874C9C4381CF044997B0FFFFE78071
:10FA8000E055AA85268597400000E78040DA1305F7
:10FA9000040197000000E780C0EA228597800000FB
:10FAA000E78000338144ADBF1723FFFFE702A35F68
:10FAB00083C795004111AA8A93F7F707A384F5003D
:10FAC0003285AE8932842311010097C0FFFFE780A1
:10FAD000205093170501C1876354F0062A8AC14557
:10FAE000228597C0FFFFE7804035AA8B5285032B04
:10FAF000040097A0FFFFE780004E21E983574400F0
:10FB000085440144F11793B71700A300F10003489F
:10FB1000110003572100DA875685D2862686CE85C6
:10FB200097D0FFFFE780805BA1679387270248009B
:10FB30003EC42302910022C697D0FFFFE780202019
:10FB400041011723FFFF67008359A28513061100A7
:10FB500097E0FFFFE780401A2A8489444DD99767D0
:10FB6000FF1F9387673D98433E8901CF044997B0B3
:10FB7000FFFFE780A046AA85268597400000E78022
:10FB800000CB1305040197000000E78080DB97B0ED
:10FB9000FFFFE780A04495443DD9930521005E8591
:10FBA00097F0FFFFE78060B6AA8435F11C48035741
:10FBB000210022852390E70097800000E780402104
:10FBC00083270900A9D70355210097400000E7804B
:10FBD000A0BD35BF1723FFFFE702E34C83C79500A5
:10FBE0004111AA8A93F7F707A384F5003285AE89FD
:10FBF000328497C0FFFFE780A03D93170501C187BE
:10FC00006351F0062A8A228597C0FFFFE780403CB7
:10FC10002A895285032B040097A0FFFFE780A03BB1
:10FC200031E58357440085440144F11793B7170029
:10FC3000A301F10003483100DA8756854A87D2864E
:10FC40002686CE8597D0FFFFE7804049A167F90758
:10FC500048003EC42302910022C697D0FFFFE780F0
:10FC6000000E41011723FFFF67006347A2851306BB
:10FC7000310097E0FFFFE78020082A8489445DD99E
:10FC80009167CA97C2071167C1831307F7EF8544CD
:10FC9000E362F7FA9767FF1F9387072A9843BE8BA3
:10FCA00001CF044997B0FFFFE7804033AA8526853E
:10FCB00097400000E780A0B71305040197000000FB
:10FCC000E78020C897B0FFFFE780403195443DD1E1
:10FCD0001C48228581442390270197800000E780FB
:10FCE000200F83A70B00B9D74A8597400000E78013
:10FCF000A0AB89B71723FFFFE702633D2A844105C4
:10FD0000B28497000000E780C0C311C522859780A8
:10FD10000000E780E00B81460146A685228597809A
:10FD20000000E780C04E1C4C89C7DC4799C3228580
:10FD300082971723FFFF6700C33B9767FF1F9387D7
:10FD4000A7009C43014599C31385070182809767EB
:10FD5000FF1F938767FF884382801723FFFFE70217
:10FD600003379317C600DD8DC2054111C1812A8476
:10FD700032C697C0FFFFE780E01732462285118226
:10FD80009375F60F97C0FFFFE780C014410117235A
:10FD9000FFFF670003361723FFFFE702A3317971E6
:10FDA0003C083ED2B7070C003ED43C083ED683C781
:10FDB0009500AE842A8993F7F707A384F500A1651F
:10FDC00093853504481097A0FFFFE780E02BC165BD
:10FDD000FD150144176AFF1F130A8A17930A400E84
:10FDE000AE892E8B2EC697B0FFFFE78020224205FA
:10FDF000931704014181C183B24563E9A702C1673A
:10FE0000FD176387F500481097C0FFFFE780800E5D
:10FE1000501001478146A6854A8597A0FFFFE780DD
:10FE2000004C45611723FFFF6700032C3307540381
:10FE300083270A0BBA9703D6C701630A3601638A80
:10FE40003501481097000000E78060F1DA8505046D
:10FE500051BFB285EDBF1723FFFFE702C3247971BD
:10FE60007C083EC8B70711003ECA7C083ECC83C759
:10FE70009500AA89328593F7F707A384F5002E89A8
:10FE800097C0FFFFE780C01485676378F504A1651C
:10FE9000AA848905080897A0FFFFE780E01E268551
:10FEA00097400000E78060ED133415000A04A28536
:10FEB000080897C0FFFFE780E001A685080897C003
:10FEC000FFFFE780200325CC014781461008CA8543
:10FED0004E8597A0FFFFE780804045611723FFFF15
:10FEE0006700E31FB30754030327CA0ABA9703D76F
:10FEF0000700631C970003D6270063806505080888
:10FF000097000000E780A0E5DE8505042EC697B0C7
:10FF1000FFFFE780A0104205931704014181C183D0
:10FF2000B245E3E1A7FCC167FD17E38FF5F80808C8
:10FF300097C0FFFFE78000FC41BFB285F9B7C165FC
:10FF4000FD150144176AFF1F130A8A00930A8002F5
:10FF50002E8BAE8B65BF1723FFFFE70243171841B7
:10FF60008347170083460700A207D58FD207D183A6
:10FF70002390F50083472700034717008D45A2070C
:10FF8000D98F91832310F60097C0FFFFE780A0E987
:10FF90001723FFFF6700E3151723FFFFE702831115
:10FFA000C16401441769FF1F130989FA930980028C
:10FFB000FD1497B0FFFFE78060066347A40001458A
:10FFC0001723FFFF67004312330534038327C90A51
:10FFD0003E9583570500E38597FE0504D9BF172397
:10FFE000FFFFE702230D2A8AAE89B284B68A9740C2
:10FFF0000000E78080D819E591473E851723FFFF71
:020000040001F9
:100000006700830E2A894E8597C00000E780E08E46
:100010002A84638E0A048D476DD103570500C547B6
:10002000E31D47FD0347F9018546AD47E317D7FCBC
:100030008347450081CF4146A6855D0597F00000C6
:10004000E780C09E814755D9AD4745BF130965017B
:100050002302E500CA85268597100000E7806062CC
:1000600031C1A547E38B0AF82302040079B705C123
:1000700083570500E39247F94146A685190597F095
:100080000000E780A09A81472DD99947BDB74E85DA
:1000900097000000E78080F02A84954739DD130936
:1000A00055004DBF4146A68523104401231134015C
:1000B0001305190097F00000E780A099228597802A
:1000C0000000E780A0EA81470DBF1723FFFFE7028A
:1000D000030079717C003ECCB7070A003ECE7C005D
:1000E0003ED083C79500B2842E8493F7F707A3848C
:1000F000F5001306A1002A892C0026859700000030
:10010000E780A0E5A16528088D0597A0FFFFE7809F
:10011000A0F790408355A1000355810085469700C4
:100120000000E78000ECAA84AA85280897C0FFFF9A
:10013000E78040DA0356A100835581002808970024
:100140000000E780C0C1300801478146A2854A858A
:1001500097A0FFFFE780A018854748103ED42302F0
:10016000910202D697D0FFFFE78060BD456117235B
:10017000FFFF670003F81723FFFFE70243F57971DC
:100180007C003ECCB7070A003ECE7C003ED083C741
:100190009500B2842E8493F7F707A384F500130625
:1001A000A1002A892C00268597000000E780E0DA6C
:1001B000A16528088D0597A0FFFFE780E0EC90403F
:1001C0008355A10003558100814697000000E78018
:1001D00040E1AA84AA85280897C0FFFFE78080CF66
:1001E0000356A10083558100280897000000E7808E
:1001F00000B7300801478146A2854A8597A0FFFFD6
:10020000E780E00D48102302910202D402D697D075
:10021000FFFFE780C0B245611723FFFF670063ED72
:100220001723FFFFE702A3EA97000000E78060DBE7
:100230001723FFFF6700E3EB9767FF1F938707B163
:10024000884382801723FFFFE70263E88357250076
:100250004111AE842A842307B10017F5FFFF13056F
:1002600025466C002316F10097A0FFFFE780204988
:1002700091C4228597800000E780E0D6FD572310C7
:10028000F400130620028145130554009720FFFF58
:10029000E780E0E641011723FFFF670083E51723AE
:1002A000FFFFE70223E179717C003ECCB7070A002B
:1002B0003ECE7C003ED083C79500AA89AE8493F7DA
:1002C000F7073285A384F5001306A1002C009700E0
:1002D0000000E78080C8035581001144974000006A
:1002E000E780A0A915C50355A100014497B00000FF
:1002F000E780A06011CD0357050083578100454476
:100300006318F700854597000000E780E0F301449B
:10031000216993053900280897A0FFFFE780C0D620
:10032000A285280897C0FFFFE780C0BA0356A10046
:1003300083558100280897000000E78040A230081C
:1003400001478146A6854E8597A0FFFFE78020F9EB
:1003500048104AD42302810202D697D0FFFFE780DB
:10036000009E45611723FFFF670003D81723FFFF97
:10037000E70243D49767FF1F9387079D2A8488432A
:100380002E8915C5035745038357C4016311F7022E
:100390002326050223180502410597D00000E780B7
:1003A000209C6306090097800000E78060DB8144A1
:1003B0009769FF1F9389C9B9130A800297B0FFFF9D
:1003C000E780C0C563C4A4049767FF1F938787A015
:1003D0009C4399C70355C40197200000E780C0BD26
:1003E00063070900228597800000E780C0A01306FC
:1003F000400E814522859720FFFFE78040D0FD57C2
:10040000231EF4001723FFFF670003CE3385440348
:1004100083A7C90A3E95035705008357C401631794
:10042000F700CA8597000000E78000E2850479B7ED
:100430001723FFFFE70203C883C795004111AA896C
:1004400093F7F707A384F5003285AE8497C0FFFFCA
:10045000E78000B885676378F5042A899740000033
:10046000E780A091014401CD83D704003144638823
:100470002701854597000000E78080EF01444E8505
:10048000A2864A86A68597D0FFFFE780A09CA16739
:100490009387170448003EC42302810002C697D008
:1004A000FFFFE780C08941011723FFFF6700C3C337
:1004B0001723FFFFE70203C09767FF1F9387C788D3
:1004C000804329C4014597C00000E780002181478F
:1004D0000148C1641CDC232E040323200404176993
:1004E000FF1F1309E9A601449309400EFD1497B0BC
:1004F000FFFFE780A0B1634FA400814517F5FFFF20
:100500001305857F97A0FFFFE780601F1723FFFF7C
:10051000670083BD330534038327090B3E9583575A
:10052000C50163879700854597000000E78040E498
:10053000050475BF9357050113D78700A380F50005
:1005400093170501C183A1832380E5002381F50072
:10055000A381A50082801723FFFFE70243B7230092
:10056000050083C71500A300F50083C725002301FC
:10057000F50083C73500A301F50083C745002302BA
:10058000F50083C75500A302F50083C765009305F6
:100590009500A30305002303F5002304050032851D
:1005A00097000000E78040F91723FFFF670063B45E
:1005B0001723FFFFE70203B04111E9540DCD85CDAC
:1005C00093F9C5FF2E842A89AA84338AA900B7EA41
:1005D000040063189A020D88854411CCB7E7040023
:1005E0009C5F82972AC622866C003305390197E00A
:1005F0000000E7800046268541011723FFFF6700C2
:10060000A3AE83A78A039104829793170501C18340
:10061000A183A38EF4FE93570501238FF4FEA183DB
:10062000238EA4FEA38FF4FE6DB763E6D5021723D5
:10063000FFFFE702C3A9B28741113686BE8536C6E1
:1006400097E00000E780E040B2464101368517237D
:10065000FFFF670003AA81463685828083870500F5
:100660001387F5003D05FD8793F77708834607005C
:100670007D158606B58FA300F5006307B7007D17CB
:10068000834717009D83DDB782801723FFFFE702B2
:1006900003A4B7E7040083A7070932872A863A85AF
:1006A0008297133515001723FFFF670083A415C138
:1006B00081478DC11723FFFFE70263A1414697E001
:1006C0000000E780003985473E851723FFFF67005C
:1006D00043A281473E8582801DCD1723FFFFE7029D
:1006E000039F414681452A849720FFFFE78020A190
:1006F00041468145130504039720FFFFE78020A0B2
:100700000147C1672322040438C87CC80545172364
:10071000FFFF6700039E0145828081473DCDB5CD37
:100720001723FFFFE702A39AB2842E8913068005E0
:1007300081452A849720FFFFE780609CCA8524C4F6
:10074000268597000000E780C0F641468145228556
:100750009720FFFFE780A09A3044A285228597006A
:100760000000E780C0F293040401A285268597006B
:100770000000E780E0EEA685130504029700000064
:10078000E78000EE228597000000E78020F585478E
:100790003E851723FFFF6700C3953E8582801723A0
:1007A000FFFFE70223914111E9540DCD85CD93F967
:1007B000C5FF2E842A89AA84338AA900B7EA0400D7
:1007C000639844030D88814411CCB7E704009C5F13
:1007D00082972AC622866C003305390197E0000013
:1007E000E7802027268541011723FFFF6700C38F7D
:1007F00083A78A039104829793170501C183A1837C
:10080000A38EF4FE93570501238FF4FEA183238E5C
:10081000A4FEA38FF4FE6DB765CD1723FFFFE7029B
:100820006389B28411E605451723FFFF6700C38B78
:100830002A842E890145EDD93C487848B3E6E70083
:10084000E5D69386F7FFB3B7F6007D17032A440475
:10085000BA9734C87CC863050A06C14913050A0360
:10086000B38949412295637D3601B2862E86A685DD
:1008700097000000E780A0DB7C40BE9464C065B7B1
:10088000CE862E86CE8597000000E78040DAC11420
:10089000D2944E9923220404A2879306040103C72D
:1008A000070003C607038507318FA38FE7FEE39890
:1008B000F6FE3044A285228597000000E78020DD07
:1008C0002699C1493306994063EC9900A9DCA686B4
:1008D000A6851305040397000000E78040D579BF83
:1008E0008147B306F4003307F6000347070083C5CA
:1008F000060085072D8F2380E600E39437FF304400
:10090000A285228597000000E78060D8C1145DBFF2
:10091000014582800DC11713FFFFE702437B1306D9
:10092000800581459710FFFFE780607D054517131F
:10093000FFFF6700037C01458280814749C5C1C52F
:100940001713FFFFE702A378FC4141462E84AA84D7
:100950006399C70413860501A2878146C14503C771
:10096000070003C507038507298F3305D600034514
:1009700005008506298FA38FE7FEE392B6FE30447B
:10098000A285268597000000E78060D02285970029
:100990000000E78060F885473E851713FFFF67007A
:1009A0004375138507031D8E814522959710FFFF20
:1009B000E780E0747C40130700F813060402A29756
:1009C0002388E70251BF3E8582801713FFFFE702AD
:1009D00003706D712E84B284AA8590102800368928
:1009E00097000000E780A0D309EDD55725A050401F
:1009F0000C40280097000000E78040E27DD5FD1400
:100A00002104F5F42C004A8597000000E78020F3CC
:100A1000814761DD3E8551611713FFFF6700636DFC
:100A20001713FFFFE702A36A41112EC432C62C0040
:100A3000054697000000E78080F941011713FFFF8A
:100A40006700236B1713FFFFE702636801112A8415
:100A50002EC602C802CA02CC02CE97E00000E78090
:100A6000402BB2462A86A285080897000000E7803E
:100A700060FB1375F50F05611713FFFF67006367D0
:100A80001713FFFFE702A3647971B2872A84214616
:100A90002308B10013051101BE853AC436C697E09C
:100AA0000000E78000FBB246930591013685970070
:100AB0000000E78060A82285141035460C089700D6
:100AC0000000E78020F62A84224701E921460C1025
:100AD0003A8597E00000E780C0F72285456117134B
:100AE000FFFF670003611713FFFFE702435E7171A9
:100AF000AE84AA850A85328497000000E78060BB37
:100B000011C90A86A685228597000000E78020B8D3
:100B1000814711E1C5473E854D611713FFFF67000F
:100B2000435D1713FFFFE70283571D712A8AB289BD
:100B3000BE8435468547130511012E8CB68A3A8B43
:100B4000C28C468D2308F10097E00000E78060F03A
:100B500010100C085285231F010097000000E78049
:100B6000C0F82A843DEDA1476313FD089307900563
:100B700091E0E5473546E2851305110113990A0115
:100B80002308F1001359090197E00000E78060ECA9
:100B90001357890093978A00D98F90080C085285C3
:100BA000231FF10097000000E78020F42A8415E954
:100BB000A1E49387FA0091831379F9003EC6631389
:100BC00009004149668B8144C14B854DB247639F03
:100BD000970C6A868C0033855C0197E00000E78003
:100BE00040E7228525611713FFFF6700034F930736
:100BF0009004C9F0A547BDBF834701050947C14B14
:100C00002308F10083471105A58FA308F1009387FE
:100C10002400814463E1FB04014714083386E600A5
:100C20008C08B386E400BA95DA9683C6060083C5BD
:100C300005000507AD8E2300D600E390E7FE41478F
:100C4000639CE70490080C08528597000000E78039
:100C5000C0E925D181A0B3069B00BA871008B3056F
:100C6000F60090083E9603C5060003460600850779
:100C70008506298E2380C500E39277FF998F90081F
:100C80000C085285BE9497000000E78000E6894773
:100C9000014749D12A84B1B790083E960346060021
:100CA0001408BE962380C600850759BFB247850445
:100CB0006387971481471808B306F70098083E9792
:100CC0003386F90003470700034606008507318F86
:100CD0002380E600E39177FF90080C085285970087
:100CE0000000E78080E05DF53546E28513051101DF
:100CF0002308B10197E00000E780A0D51397040115
:100D00004183939784002183D98F10180C08528552
:100D1000231FF10097000000E78020DD25FD8147BB
:100D200010183387F9003E96034707000346060074
:100D3000B306FB008507318F2380E600E39277FF3F
:100D400065A81808B306F70098083E973386F9009F
:100D500003470700034606008507318F2380E6001E
:100D6000E3E127FFCA87639E770990080C08528544
:100D700097000000E78060D711FD81479800B30617
:100D8000F700900818103E973E9603470700034669
:100D900006008507318F2380E600E39177FF354613
:100DA000E285130511012308B10197E00000E780F7
:100DB00040CA139704014183939784002183D98FFC
:100DC00010180C085285231FF10097000000E780DF
:100DD000C0D1E31105EC814710183387F9003E9626
:100DE0000347070003460600B306FB008507318F63
:100DF0002380E600E3E227FFC109410BC1BB814725
:100E000085B79408BE9683C6060018083E9723004F
:100E1000D700850789BF638006321713FFFFE702FB
:100E2000032859712A84BE89B28B8547354613053C
:100E300011022E8B468C4289BA8A368A2300F1022F
:100E400097E00000E780E0C010180C1022852317FF
:100E5000010297000000E78040C963180512A1470E
:100E6000631FFC069307900563930900E547354629
:100E7000DA851305110293140A012300F102C180DF
:100E800097E00000E780E0BC93178A0013D7840046
:100E9000D98F90080C1022852317F10297000000CB
:100EA000E780A0C47DE1639209049307FA00BD883E
:100EB000918391E0C144C207C183DE8C814A3EC662
:100EC000414DB24763E2FA0E6286B3854B0188104A
:100ED00097E00000E78080B54DC93D557DA09307A0
:100EE0009004E39609F8A54759B7834701050947D8
:100EF000C14C2300F10283471105B3C7F900A300D9
:100F0000F10293872900814963E1FC0481461810AE
:100F10003306D7008C083387D900B6955697034718
:100F2000070083C5050085062D8F2300E600E390AA
:100F3000D7FE41476390E70690080C102285970082
:100F40000000E78080BA35D189A0B3863A01BA871C
:100F50001010B305F60090083E9603C50600034640
:100F6000060085078506298E2380C500E39297FF3A
:100F70003387EC4090080C102285BA999700000046
:100F8000E780A0B68947014741D165611713FFFF8C
:100F90006700A31490083E96034606001410BE9600
:100FA0002380C600850779B7B247850A93990A015D
:100FB000939D8A0093D909016391570F8547354660
:100FC000DA85130511022300F10293D9890097E015
:100FD0000000E78000A8B3ED3D0190000C102285D1
:100FE0002317B10397000000E78020B059FD814727
:100FF000A68963EA970626860C084A8597E00000D2
:10100000E78020A581471810B306F700100898085C
:101010003E973E9603470700034606008507318F3B
:101020002380E600E3E197FE639FA90590080C107A
:10103000228597000000E78040AB21F98147981096
:10104000B306F700900818183E973E96034707002E
:10105000034606008507318F2380E600E391A7FF52
:101060004109C10CB9BD18089000B306F7003E96BF
:101070003387FC0003470700034606008507318FCE
:101080002380E600B5B798084E97034707001C1069
:10109000CE972380E700850941BF85473546DA852D
:1010A000130511022300F10293D9890097E0000093
:1010B000E780209AB3ED3D0190000C1022852317A4
:1010C000B10397000000E78040A2E31005EC8147E0
:1010D00018089000B306F7003E963387FC000347DC
:1010E0000700034606008507318F2380E600E39161
:1010F000A7FF41460C084A8597E00000E78060950D
:1011000081471810B306F700100898083E973E96DE
:1011100003470700034606008507318F2380E6005A
:10112000E391A7FF90080C10228597000000E7804C
:10113000C09B1DD599BD7D5582801713FFFFE70227
:1011400003F901112A842E8593055100328902C0CA
:1011500002C202C402C69304740097F0FFFFE78046
:10116000A03D1D46A6851305910097E00000E7808D
:10117000408E10088A854A8597000000E780E09637
:1011800019ED93071400180883C6070003460700EB
:1011900085070507B18EA38FD7FEE397F4FE05619F
:1011A0001713FFFF6700E3F41713FFFFE70283F055
:1011B0002E848C414111AA8983871500328991447C
:1011C00063D30700A1449757FF1F9387E70E9C4303
:1011D000A1C7C1CA8D472310F10083C725004A85E6
:1011E0002301F10083C73500A301F10083C7450047
:1011F0002302F10083C75500A302F10083C76500F5
:1012000093059100A30301002303F10023040100CF
:1012100097F0FFFFE78040320C404A860A8597F03E
:10122000FFFFE78080330328040083564400A6882C
:101230001D0881470147E51642868A854E8597003D
:101240000000E780408E2A8919E5A685228597B09F
:10125000FFFFE780E0C14A8541011713FFFF6700E8
:10126000A3E84A860A8597F0FFFFE780002F6DB755
:101270001713FFFFE70203E42E848C414111AA8972
:10128000838715003289914463D30700A14497579F
:10129000FF1F938767029C43A1C7C1C68D472310D8
:1012A000F10083C725004A852301F10083C735007B
:1012B000A301F10083C745002302F10083C7550055
:1012C000A302F10083C7650093059100A303010009
:1012D0002303F1002304010097F0FFFFE780C025FE
:1012E0000C404A860A8597F0FFFFE7800027835667
:1012F0004400032804008A85858EC2061D08C18229
:101300002312D400A68881470147E51642864E8500
:1013100097000000E78060B041011713FFFF6700EE
:10132000A3DC4A860A8597F0FFFFE78000234DBFC4
:101330001713FFFFE702A3D9B335B00001118505EC
:101340002A891315F601336515012308B1009305A9
:10135000110136843AC632C03EC442C297F0FFFF44
:10136000E780801DA2471248425593D68700230B81
:10137000F1009305910193578800A30AD100A30BB4
:10138000F100230C010197F0FFFFE780E01A3247DC
:10139000024603280400B337E00083564400920756
:1013A000914411C2A1444A85A68842860C0897F050
:1013B000FFFFE78040772A8919E5A685228597B047
:1013C000FFFFE780E0AA4A8505611713FFFF67006A
:1013D00043D21713FFFFE702E3CD01113EC6864754
:1013E000B335B0008505AA891315F6015D8D230874
:1013F000B1009305110136843A89B28442C446C2D1
:1014000097F0FFFFE7804013224892481645935714
:101410008800A30AF1009305910193D78800230B5C
:101420000101A30BF100230C110197F0FFFFE780EE
:10143000A0103247104083564400B337E0009207B3
:1014400003280900914891C0A1480C084E859700D7
:101450000000E780809CAA8401E9835544004A8506
:1014600097B0FFFFE780C0A0268505611713FFFF37
:10147000670083C7AA959307F00F1717010013079A
:10148000A7AC6317B50013C5F7FF1375F50F82807E
:1014900005058346F5FFB58FBA9783C70700D5B713
:1014A0000357450014419307F00F17160100130668
:1014B000A6A9369742074183139506014181631B14
:1014C000E500AD8FB29703C50700130515F313357B
:1014D00015008280850603C5F6FFA98FB29783C7E2
:1014E0000700D9BF1713FFFFE70263BEB287368438
:1014F0002E86BA86AA853E85BA8497F0FFFFE780DC
:101500006052634F0500228597E00000E78060800D
:101510002A86A686A285268597F0FFFFE780805061
:101520001713FFFF6700E3BC1713FFFFE70283B841
:101530005D712A8BAE8A171501001305659E2C007C
:10154000B284368ABA893E8997F0FFFFE780C04FA0
:101550002A845DE134104146DA85280097F0FFFFC8
:10156000E780404C2A8449E98547A303F100A6C2DD
:10157000930771002408BEC4A68685470D462C1823
:10158000281002DC02DED6C0BEC697F0FFFFE7805F
:1015900000442A8435E183477102A6860D4693F7FD
:1015A000F7072300FA00C1473EDE2C1889472810B0
:1015B00026DCA303F10097F0FFFFE78040412A8477
:1015C00005ED4146A6854E8597D00000E78060482E
:1015D0008D47A6860D462C182810A303F10097F01E
:1015E000FFFFE780C03E2A8401E94146A6854A857F
:1015F00097D00000E780E045228561611713FFFF67
:10160000670083AE1713FFFFE70263AC97F7000094
:10161000938707EF984383C7470079712A89AE847F
:1016200017150100130545900C083AC42306F10074
:1016300097F0FFFFE78040412A8405ED14104146F2
:10164000CA85080897F0FFFFE780C03D2A8415E1AE
:10165000140815462C00081097F0FFFFE780803C27
:101660002A8401E921462C08268597D00000E780CE
:10167000403E228545611713FFFF670083A71713BC
:10168000FFFFE702C3A497F70000938767E79C4733
:101690007971AA842E8417150100130565890C0839
:1016A0003EC697F0FFFFE780203A0DE9141041464F
:1016B000A685080897F0FFFFE780C03605E114080B
:1016C00011466C00081097F0FFFFE780A03519E580
:1016D0008347F10193F7F7032300F40045611713E3
:1016E000FFFF670003A11713FFFFE702439E368841
:1016F000A14881470147E54697F0FFFFE780A042F8
:101700001713FFFF6700E39E1713FFFFE702239CF9
:101710003688A14881470147E54697F0FFFFE780FB
:10172000C06F1713FFFF6700C39C1713FFFFE7028B
:10173000039A01112A842E850C0832C697F0FFFF08
:10174000E780803009ED3247970601009386C67C1A
:101750001008C145228597000000E780E0D80561A8
:101760001713FFFF6700E3981713FFFFE7022396A5
:101770004111C1472EC032C48A8509463EC23EC6C9
:1017800097F0FFFFE780A02441011713FFFF6700D8
:1017900043961713FFFFE70283934111AE861306AA
:1017A0001009AA850A8502C002C202C402C697F0C7
:1017B000FFFFE780202741011713FFFF67006393B6
:1017C0001713FFFFE702A390328797060100938665
:1017D000A6762E869305000297000000E780C0D011
:1017E0001713FFFF6700E3901713FFFFE702238E35
:1017F0007971C1472ACC2ED032D42C080D4628004E
:101800003ECE3ED23ED602C402C602C802CA97F0FD
:10181000FFFFE780C01B45611713FFFF6700638D63
:101820001713FFFFE702A38A0111AA842E8417056C
:1018300001001305E5708A8597F0FFFFE780C0205F
:1018400015E514084146A6850A8597F0FFFFE78055
:10185000601D09ED8347E1010347F101A207D98F1C
:10186000CA07C9836177D98F2310F4000561171364
:10187000FFFF6700038815CD1713FFFFE7022385DD
:101880009747FF1F9387075190439745FF1F938505
:10189000A5501745FF1F1305E54B97D00000E780C3
:1018A00000C51745FF1F1305E54A1713FFFF670023
:1018B00043841745FF1F1305E54982808DCD17131B
:1018C000FFFFE702C3809747FF1F9387A74C94430E
:1018D00001112E840A869745FF1F9385E54B97D00B
:1018E0000000E78040C60A85029401450561171390
:1018F000FFFF670003807D5582801703FFFFE7022B
:10190000037D97D00000E78080D19747FF1F23A376
:10191000A74817F5FFFF1305E5C997B00000E7805A
:10192000C0741703FFFF6700C37C1747FF1F13072F
:10193000A7489317150008433E95FD572310F5005F
:1019400082801703FFFFE70283782A84084009E5B5
:101950001703FFFF6700E3791C4158401CC0631365
:10196000E5005CC08347550023200500F99BA302D6
:10197000F50097A0FFFFE780207CC9BF1703FFFF9A
:10198000E70243739747FF1F9387074598432A84CD
:1019900011CB8347350093F7070289C7035505002C
:1019A000894502971305440197B00000E780403B4A
:1019B000835504000355E40097300000E780A00C35
:1019C000485819C597A0FFFFE7800077232A040233
:1019D0001305840397000000E780E0F68144B149D5
:1019E0009790FFFFE780C06D63CBA402834734006C
:1019F0002320040493F727FCA301F40000489790E8
:101A0000FFFFE780E06C13161500814522859700E3
:101A1000FFFFE780C06E1703FFFF6700E36CB3872B
:101A200034030329040385043E994A859700000086
:101A3000E78060F12304090065B78347350093F719
:101A4000070299E3014582808357E500E39CB7FED6
:101A5000C167FD176316F60005458280054599A804
:101A60001703FFFFE702A36693170601C187B2843D
:101A70002A8401496359F002835705009DCB014533
:101A80006367F600034584003E953325A600137571
:101A9000F50F0DA01C4813171900BA9783D707003C
:101AA000E38E97FA05099790FFFFE7806062E343B2
:101AB000A9FE01451703FFFF6700A3631703FFFF9C
:101AC000E702435FAE89AA849790FFFFE780005644
:101AD0002A8497D0FFFFE780A02EAA86014713062D
:101AE000840197050000938585E41745FF1F1305C2
:101AF000E52C9790FFFFE780801C2A8925C98C443C
:101B00001304C50022859E0593F5050897A0FFFFE5
:101B1000E780403CCC4083877400E18163DD0704AB
:101B200093E50508228597A0FFFFE780A03A0D46C0
:101B300093854400228597A0FFFFE780C03683D5B8
:101B40000400228597A0FFFFE780E03D83D52400B5
:101B5000228597A0FFFFE780003D03D6490083A5BB
:101B60000900228597A0FFFFE780E0334A8517032D
:101B7000FFFF6700635793F5F5076DB71703FFFF86
:101B8000E702E35401112A84328532C697A0FFFF91
:101B9000E780E0279780FFFFE780603483570400E9
:101BA0001747FF1F1307C73A3246231BF10093075D
:101BB00000F8A30DF1001C471843231AA1008983E4
:101BC000858BB307F740B28548083ECE231C010041
:101BD000230D010097000000E78080EE05611703E8
:101BE000FFFF670003511703FFFFE702A34C00410B
:101BF00001453DC49304C40026853289AE8997A06F
:101C0000FFFFE780C02495452A8A2685035B0401EF
:101C100097A0FFFFE7802021268597A0FFFFE780A0
:101C2000603E8D45AA8A268597A0FFFFE780A01F0A
:101C3000268597A0FFFFE780E03C5C48420A135AE4
:101C40000A01D2975CC423186401814763983A0162
:101C500046054D81330625419337160013F5F70FDE
:101C60001703FFFF670043481703FFFFE702A34383
:101C700089692A8BAE8B328AB68A81440144314C01
:101C8000FD199790FFFFE780A04363CDA4009790D4
:101C9000FFFFE780E045018D33B5AA001703FFFF82
:101CA0006700E3433389840383270B003E9963175E
:101CB0000A008347890085043E94E1B703560A0071
:101CC000DE854A8533F6C90097000000E780E0F121
:101CD0006DD10545E1B71703FFFFE702433F01114F
:101CE0002A847C000355E5003ECAB70707003ECCB6
:101CF0007C003ECE97200000E78020082A89854599
:101D0000480897A0FFFFE78020399945480897A029
:101D1000FFFFE780E015AA844A8597200000E7804E
:101D2000A0082380A4009747FF1F938767229C4346
:101D30004166130606F09396870113D78701558FE6
:101D400093D68700F18E558FA207B706FF00F58F57
:101D5000D98F11462C00138514003EC497D0000083
:101D6000E78020CF5008A382040089452285970090
:101D70000000E780E0E019C9AA851305840397A055
:101D8000FFFFE780E0313C4085073CC00561170359
:101D9000FFFF670003361703FFFFE7024333979007
:101DA000FFFFE780E0342A8405049790FFFFE78077
:101DB00020333305A402F14791453305F5029720FE
:101DC0000000E78020BA11E565551703FFFF6700A3
:101DD00043329747FF1F23A9A7FE9790FFFFE78095
:101DE00020312A8405049790FFFFE780602F330598
:101DF000A4028945060597200000E780A0B669D5B2
:101E00009747FF1F23AAA7FA9790FFFFE780402E6E
:101E10002A8405049790FFFFE780802C3304A402F6
:101E20009747FF1F239C87F89790FFFFE780402C80
:101E30002A849790FFFFE780A02A93071400338538
:101E4000A7029747FF1F239CA7F6970701009387D8
:101E5000E7D21747FF1F2327F7F60145BDB7170342
:101E6000FFFFE7022325AA842E8901449749FF1F1B
:101E70009389090E130A80069790FFFFE78040269A
:101E80006347A40001451703FFFF6700E3253305FF
:101E9000440383A709024A86A6853E959700000061
:101EA000E780E0B919E10504C1BF0545E9BF1703A3
:101EB000FFFFE702431FAA8A2E8BB28B368C3A8A29
:101EC000814401448149974CFF1F938C6C08130D8A
:101ED00080069790FFFFE780A02063C9A40011E06F
:101EE00085494E851703FFFF6700631F3389A403ED
:101EF00083A70C025E86D6853E994A85970000002E
:101F0000E780E0B31DC19790FFFFE780601E0544A6
:101F1000636D4501D2866286DA8513050903970051
:101F20000000E780A0D411C1854985045DB717037F
:101F3000FFFFE7022318C16441112A890144974930
:101F4000FF1F9389E900130A8006FD1436C632C4C8
:101F50002EC29790FFFFE780A01892452246B24616
:101F60006348A400014541011703FFFF6700C31741
:101F70003305440383A709023E9509C6834735000C
:101F8000C18B9DC791C68347350093F707028DC368
:101F9000630699008357E500639C270103570500FA
:101FA00001CB63E7E50083478500BA97E3CDF5FAF7
:101FB000050469BF1703FFFFE702C30FC1642A8945
:101FC00001449749FF1F9389A9F8130A8006FD145D
:101FD0009790FFFFE780C0106346A4001703FFFF40
:101FE000670083103305440383A709023E95835796
:101FF000E500638A970063049900639627019700C0
:102000000000E780E0970504E1B71703FFFFE70250
:10201000030989692A8AAE8A328BB68B8144174CB0
:10202000FF1F130CECF2930C8006314DFD199790B5
:10203000FFFFE780E00A63C6A4001703FFFF670005
:10204000C3093389940383270C028355CA015A8636
:102050003E994A8597000000E780609E31C1814D1E
:1020600015A03384AD038327090303D60B00D6855F
:1020700033F6C9003E94228597000000E780E0B661
:1020800009E9850D9790FFFFE7808003E3CBADFC66
:1020900001A8228597000000E780E08A230404005D
:1020A000850471B71703FFFFE702E3FF4169AA8ABE
:1020B000014A174BFF1F130BABE97D19C14B054CB0
:1020C0009790FFFFE780C0016346AA001703FFFF58
:1020D0006700E30093098006B3073A0383290B02E4
:1020E000BE9983D7E900638E270163842A01639A2E
:1020F000570103A4890301E84E8597000000E7809B
:10210000C0BD050A75BF835704016399770993041D
:10211000C400268597A0FFFFE78060D385452A8D00
:102120002685835C040197A0FFFFE780C0CF26854A
:1021300097A0FFFFE780A0E762056185635905046A
:102140008D45268597A0FFFFE780E0CD8945268550
:1021500097A0FFFFE78020CD8945268597A0FFFF48
:10216000E78060CC8545268597A0FFFFE780E0CC1F
:1021700083470500094793F7F707639AE7009945F6
:10218000268597A0FFFFE78040CBA3028501484842
:10219000337D2D01231894016A9548C40040A1BFE6
:1021A0001703FFFFE702A3F237E404008327041DAF
:1021B00082979747FF1F83C7A7C61715FF1F1305F1
:1021C000E535A300F5008327441C82978327841CF0
:1021D00081461306F00F8145014582971703FFFFE3
:1021E000670023F11747FF1F130787B3184397456D
:1021F000FF1F83C5E5C29747FF1F9387E7C083464C
:102200008703034697036397D5009747FF1F2389EA
:10221000C7C0828083C587010347A7036317B60041
:102220009747FF1F238EE7BE828003C6870163178F
:10223000C7009747FF1F2385D7BE828083C68701CB
:10224000130750026319D700930760021747FF1F57
:102250002308F7BC828083C68701130660026315DA
:10226000D60093077002DDB783C7870155BF974734
:10227000FF1F938767B9D44B0947638DE60817039F
:10228000FFFFE702C3E41749FF1F130929B53E8486
:1022900083470900918B9DCFB7E4040083A7041DF9
:1022A000829783A7441C1745FF1F1305A5B3829788
:1022B00083A7841C81461746FF1F0346A6B48145A9
:1022C0000145829721C583470900ED9B1747FF1FF2
:1022D0002306F7B08347040093F7F70F85CB9147A8
:1022E0001747FF1F232CF7B297000000E78080EB11
:1022F00097000000E78040EFB7E70400BC4F41467D
:1023000091451745FF1F0345A5B082971703FFFFAF
:10231000670023DE82801703FFFFE70243DB8D4760
:1023200041116306F504C5476308F502854763104C
:10233000F5029747FF1F2387A7AEB7E70400BC4B02
:10234000930500101745FF1F034585AC8297410197
:102350001703FFFF6700E3D985471747FF1F2303D4
:10236000F7ACB7E70400BC4B93050020E1BF9747EB
:10237000FF1F938767A9D44B1147638DE600B7E72A
:10238000040083A7071D8297B7E70400BC4B9305A1
:1023900000044DBF05491747FF1F232127A983C705
:1023A000070032C62E8493F7F70FD5D3B7E40400A5
:1023B00083A7041D7D141374F40F8297E37689FCC0
:1023C000B245994703C61500E3F0C7FCFC44090673
:1023D0001745FF1F130545A58297BC4893050008C4
:1023E0001745FF1F0345C5A2829779BF1703FFFF5B
:1023F000E702E3CD1747FF1F130707A14047184B1C
:102400001C409746FF1F23A7F6A06316E40017475A
:10241000FF1F2323F7A0130584FE9790FFFFE7809B
:1024200000AA035564FF9780FFFFE780807297A0A2
:10243000FFFFE78060D01703FFFF670083CB170320
:10244000FFFFE702C3C89747FF1F9387E79BD84B5F
:10245000DC4789C797000000E78080F98547174768
:10246000FF1F232DF79A9747FF1F9387678B9C4386
:10247000930500021745FF1F0345859983C787030E
:102480001747FF1F230EF798B7E70400BC4B82974E
:102490001703FFFF6700E3C59747FF1F23A8A79611
:1024A00082801703FFFFE702E3C037E404007C4C9F
:1024B000A1451745FF1F0345A59582977C48A14577
:1024C0001745FF1F0345C5949744FF1F9384C4938A
:1024D0008297DC4489EB97000000E78080D91703DE
:1024E000FFFF670063C003D567FF9780FFFFE780AA
:1024F0004066AA896DD1D84891476310F7027C4C99
:1025000091451745FF1F0345A59082977C4891454B
:102510001745FF1F0345C58F829703A9490103D4BF
:1025200009018947B7E904001747FF1F2328F78EE1
:1025300083A7091D21044204829783C784011715CC
:10254000FF1F1305A5FD61191717FF1FA308F7FC4F
:1025500083A7491C418082979747FF1F2384078CDC
:1025600083A7C91C814609469375F40F4A85829753
:1025700011E99747FF1F83C7279B89C79700FF1F54
:10258000E7802066B7E70400BC4F2146A145174508
:10259000FF1F0345E587829799B71703FFFFE702FF
:1025A00003B393F7052001112E8481CF970000001B
:1025B000E78020E91345042005611703FFFF67004A
:1025C00043B393F70510A9CF9744FF1F9384C483A7
:1025D000DC4897000000E78020C11737FF1F130772
:1025E0002774184383C78401034787036318F700E0
:1025F000DC4489C797000000E78080DF85471747E4
:10260000FF1F232DF780B7E70400BC4B93050002A2
:102610001735FF1F0345C57F82971345041069BF17
:1026200093F70508BDC79737FF1F83C7F77FE917E3
:1026300019469735FF1F9385457F1305D10093F405
:10264000F70F1739FF1F0349297E97C00000E78065
:10265000404093970401C1831737FF1F1307477D3D
:10266000231DF100231CF1009737FF1F9387C779C3
:102670003ACE3ACAD8432306010009CBDC4393156E
:10268000890154080D46E1856800829713450408C6
:1026900025B793F72500A5C39737FF1F9387C77604
:1026A000D84B89476306F7029737FF1F83C7077325
:1026B00013F7270011EF918B99CFB7E70400BC4FB8
:1026C0001306000A89451735FF1F03456574829775
:1026D00013452400D5B59737FF1F938767649C4344
:1026E00083C787031737FF1F230CF772970000007B
:1026F000E78060DBF1BF93F7050281CB9700000014
:10270000E78060DA1345040245BD93F7850081CB6D
:1027100097000000E780E0D21345840071BD93F775
:10272000150081CB97000000E780A0B4134514008A
:1027300061B593F7450081CB97000000E78060B357
:102740001345440095BD93F7050495C39737FF1FC4
:1027500083C7876B91CB97000000E780A0A49147C7
:102760001737FF1F232CF76A13450404B1B593F7FD
:1027700005010145E38207E49737FF1F9387C76888
:10278000D84B91476310F7049737FF1F938707656E
:102790009C4313D727008583D98F858B91E7B7E7B3
:1027A000040083A7071D8297B7E70400FC4F9145FB
:1027B0001735FF1F0345C565829785471737FF1FEC
:1027C000232EF76413450401C5BB9737FF1F238DE4
:1027D000A77482801703FFFFE702638F9737FF1FFD
:1027E00023AA07629737FF1F23A80762854717347C
:1027F000FF1F1304E4521737FF1F2321F7621C4009
:1028000083C787031737FF1F230CF7609790FFFFDD
:10281000E780409329C59717FF1F23A5A7D01C4029
:10282000170500001305A5D783C787031737FF1FB8
:102830002308F75E1717FF1FA302F7CE9737FF1F76
:10284000A384075CB7E7040083A70708829797373C
:10285000FF1F238FA75A1703FFFF67008389B7C79E
:10286000898E938767ED1717FF1F232DF7CA45BF82
:102870001737FF1F03474759795555E79737FF1F0C
:102880009387875803C7170005079736FF1FA38D47
:10289000E65603C717008D463377D7029736FF1FDA
:1028A000A384E65683C617001737FF1F1307474751
:1028B000184393F6F60FA9EE834787031737FF1FD8
:1028C0002300F75685471737FF1F230FF752973717
:1028D000FF1F9387A7509C430145998BA9E717F3E6
:1028E000FEFFE702C37E37E404007C48C14517358C
:1028F000FF1F0345E55182973C4885451735FF1F6B
:10290000034505518297014517F3FEFF6700637E7B
:1029100083C7170085466395F6008347970379BF01
:102920008347A70361BF82809737FF1F83C7C74DC7
:10293000A1CF17F3FEFFE702837937E4040097374E
:10294000FF1F2383074C7C4885451735FF1F034530
:10295000254C82977C4C91451735FF1F0345454B0D
:1029600082977C4891451735FF1F0345654A82973A
:102970003C48C1451735FF1F0345854982970145EE
:1029800017F3FEFF6700E3767955828017F3FEFFA9
:10299000E702E3732A84035565FF9780FFFFE78012
:1029A000401B9737FF1F93872746D847BE841DEFEC
:1029B0009790FFFFE78080779C48232004009DEBE1
:1029C0009737FF1F23AA87449737FF1F23A4874405
:1029D000B7E70400BC4B89451735FF1F0345454346
:1029E0008297014517F3FEFF6700A370630A870013
:1029F000184375BF80C39737FF1F23AF8740C9BFF8
:102A00007955CDB717F3FEFFE702636C9737FF1FC9
:102A10009387C751884323260500232405005105C9
:102A200097A00000E780C03317F3FEFF6700636CD8
:102A300017F3FEFFE702A3691734FF1F1304044FC7
:102A40001C40411199CF9C472302B5002AC61CC1E6
:102A500097000000E78040FB1C409C4B99C3324527
:102A60008297410117F3FEFF6700A36817F3FEFF8B
:102A7000E702E3654111444D328532842EC69790BA
:102A8000FFFFE780C0522AC422859790FFFFE780AE
:102A9000205403A84400630C0800B2458357440047
:102AA0001840224683D54500AA8626850298410112
:102AB00017F3FEFF6700E36317F3FEFFE7022361EE
:102AC000404D1DC808C09705000093856503130598
:102AD000440197A00000E78040169737FF1F9387B7
:102AE000E7449C43014589E79737FF1F23A08744AC
:102AF00017F3FEFF6700E35F7D55DDBF17F3FEFFB1
:102B0000E702E35C011168009305F00F02C602C8FA
:102B100002CA02CC02CE97000000E780A0F1056156
:102B200017F3FEFF6700E35C9737FF1F93870740AB
:102B30009C43D847A1679D076319F70217F3FEFF6F
:102B4000E702E358011132859790FFFFE7802046A6
:102B5000230AA1008145680097000000E78080ED0E
:102B6000056117F3FEFF6700C35882809737FF1F88
:102B70009387C73B9C43D847A16793877703631923
:102B8000F70217F3FEFFE702835401113285979095
:102B9000FFFFE780C041230AA1008145680097003C
:102BA0000000E78020E9056117F3FEFF670063542A
:102BB00082809737FF1F938767379C43D847954795
:102BC0006316F70417F3FEFFE70263500111328525
:102BD00032849790FFFFE780803D230AA100228581
:102BE0009790FFFFE780C03E83574400231BA1005E
:102BF00081453ECC1C4068003ECE97000000E78037
